:020000040800F2
:1000000000060020E1010008E3010008E301000808
:10001000E3010008E3010008E3010008E301000830
:10002000E3010008E3010008E3010008752F000860
:10003000E3010008E3010008E3010008E301000810
:10004000E3010008E3010008E3010008E301000800
:10005000E3010008E30100081D32000845320008F2
:100060006D32000895320008BD320008E301000837
:10007000E3010008E3010008E3010008E3010008D0
:10008000E3010008E3010008E3010008E3010008C0
:10009000E3010008E3010008E3010008E53200087D
:1000A000E3010008E3010008E3010008E3010008A0
:1000B000B9330008E3010008E3010008E301000888
:1000C000E3010008E3010008E3010008E301000880
:1000D000E3010008E3010008E3010008E301000870
:1000E00049330008E3010008E3010008E3010008C8
:1000F000E3010008E3010008E3010008E301000850
:10010000E3010008E3010008E3010008E30100083F
:10011000E3010008E3010008E3010008E30100082F
:10012000E3010008E3010008E3010008E30100081F
:10013000E3010008E3010008E3010008E30100080F
:10014000E3010008E3010008E30100082927000893
:10015000E3010008E3010008E3010008E3010008EF
:10016000E3010008E3010008E3010008E3010008DF
:10017000E3010008E3010008E3010008E3010008CF
:10018000E3010008E3010008E3010008E3010008BF
:10019000E3010008E3010008E3010008E3010008AF
:1001A000E3010008E3010008E3010008E30100089F
:1001B000E3010008E3010008E3010008E30100088F
:1001C000E3010008E3010008E3010008E30100087F
:1001D000E3010008E3010008E3010008E30100086F
:1001E00002E000F000F8FEE772B6374880F30888B6
:1001F000364880F3098836483649086040F20000E6
:10020000CCF200004EF63471CEF200010860BFF36C
:100210004F8FBFF36F8F40F20000C0F2F0004EF638
:100220008851CEF200010860BFF34F8FBFF36F8F8C
:100230004FF00000E1EE100A4EF63C71CEF20001E4
:100240000860062080F31488BFF36F8F01F034FF3D
:1002500002F02EFE4FF055301F491B4A91423CBF21
:1002600041F8040BFAE71D49184A91423CBF41F896
:10027000040BFAE71A491B4A1B4B9A423EBF51F83E
:10028000040B42F8040BF8E700201849184A914281
:100290003CBF41F8040BFAE701F012FF02F05CFEEC
:1002A000144C154DAC4203DA54F8041B8847F9E7A7
:1002B00000F042F8114C124DAC4203DA54F8041B22
:1002C0008847F9E701F0FABE00060020002200206E
:1002D0000000000808ED00E00000002000060020FB
:1002E0008837000800220020402200204022002001
:1002F000602E0020E0010008E0010008E001000895
:10030000E00100082DE9F04F2DED108AC1F80CD066
:10031000C3689D46BDEC108ABDE8F08F002383F3CF
:1003200011882846A047002001F074FAFEE701F08A
:1003300003FA00DFFEE7000038B500F0BFFB01F074
:100340008BFE054601F0AEFE0446C8B90E4B9D4239
:1003500018D001339D4218BF044641F2883504BFCE
:1003600001240025002001F081FE0CB100F074F89A
:1003700000F002FD284600F0C3F800F06DF8F9E740
:100380000025EFE70546EDE7010007B008B500F0EE
:1003900067FBA0F120035842584108BD07B541F260
:1003A0001203022101A8ADF8043000F077FB03B07E
:1003B0005DF804FB38B5302383F3118817480368D0
:1003C0000BB101F0F3FA164A144800234FF47A7186
:1003D00001F0E2FA002383F31188124C236813B171
:1003E0002368013B2360636813B16368013B63606A
:1003F0000D4D2B7833B963687BB9022000F026FCE1
:10040000322363602B78032B07D163682BB902205A
:1004100000F01CFC4FF47A73636038BD402200206A
:10042000B50300086023002058220020084B1870F4
:1004300003280CD8DFE800F008050208022000F0CD
:10044000FDBB022000F0F0BB024B00225A60704757
:100450005822002060230020244B254A10B51C465A
:100460001968013140D004339342F9D16268214BBD
:100470009A4239D9204B9B6803F1006303F580331E
:100480009A4231D2002000F033FB0220FFF7CEFF6A
:100490001A4B1A6C00221A64196E1A66196E596C7E
:1004A0005A64596E5A665A6E5A6942F080025A610D
:1004B0005A6922F080025A615A691A6942F0005260
:1004C0001A611A6922F000521A611B6972B64FF064
:1004D000E0233021C3F8084DD4E9003281F31188BC
:1004E0009D4683F30888104710BD00BF0000010837
:1004F00020000108FFFF0008002200200038024011
:100500002DE9F04F93B0AA4B00902022FF210AA8BA
:100510009D6800F0DBFBA74A1378A3B9A648012128
:1005200003601170302383F3118803680BB101F06D
:100530003DFAA24AA04800234FF47A7101F02CFA48
:10054000002383F31188009B13B19D4B009A1A601E
:100550009C4A009C1378032B1EBF00231370984AFB
:100560004FF0000A18BF5360D3465646D1460120CB
:1005700000F064FB24B1924B1B68002B00F0118249
:10058000002000F06DFA0390039B002BF2DB0120AA
:1005900000F04AFB039B213B162BE8D801A252F83E
:1005A00023F000BF0106000829060008BD06000868
:1005B0006F0500086F0500086F0500084707000871
:1005C000170900083108000893080008BB08000854
:1005D000E10800086F050008F30800086F0500082F
:1005E00065090008A10600086F050008A9090008B0
:1005F0000D060008A10600086F0500089308000812
:100600000220FFF7C3FE002840F0F581009B022185
:10061000BAF1000F08BF1C4605A841F21233ADF82D
:10062000143000F03BFAA2E74FF47A7000F018FAA9
:10063000071EEBDB0220FFF7A9FE0028E6D0013FF2
:10064000052F00F2DA81DFE807F0030A0D101336F8
:1006500005230593042105A800F020FA17E054486B
:100660000421F9E758480421F6E758480421F3E744
:100670004FF01C08404600F03DFA08F104080590D0
:10068000042105A800F00AFAB8F12C0FF2D10120DC
:1006900000FA07F747EA0B0B5FFA8BFB4FF00009F4
:1006A00000F060FB26B10BF00B030B2B08BF0024FE
:1006B000FFF774FE5BE746480421CDE7002EA5D086
:1006C0000BF00B030B2BA1D10220FFF75FFE0746B7
:1006D00000289BD0012000F00BFA0220FFF7A6FEB5
:1006E00000261FFA86F8404600F012FA044690B140
:1006F0000021404600F01CFA01360028F1D1BA462C
:10070000044641F21213022105A8ADF814303E460A
:1007100000F0C4F92BE70120FFF788FE2546244BA3
:100720009B68AB4207D9284600F0E4F9013040F05D
:1007300067810435F3E7234B00251D70204BBA4633
:100740005D603E46ACE7002E3FF460AF0BF00B035C
:100750000B2B7FF45BAF0220FFF768FE322000F026
:100760007FF9B0F10008FFF651AF18F003077FF4EE
:100770004DAF0F4A926808EB050393423FF646AF30
:10078000B8F5807F3FF742AF124B0193B84523DDA8
:100790004FF47A7000F064F90390039A002AFFF690
:1007A00035AF019B039A03F8012B0137EDE700BF3A
:1007B000002200205C23002040220020B503000816
:1007C000602300205822002004220020082200205C
:1007D0000C2200205C220020C820FFF7D7FD07462E
:1007E00000283FF413AF1F2D11D8C5F12002424558
:1007F0000AAB25F0030028BF424683490192184402
:1008000000F03EFA019A8048FF2100F05FFA4FEABB
:10081000A8037D490193C8F38702284600F05EFAD9
:10082000064600283FF46DAF019B05EB830537E7D3
:100830000220FFF7ABFD00283FF4E8AE00F0A4F97A
:1008400000283FF4E3AE0027B846704B9B68BB42DC
:1008500018D91F2F11D80A9B01330ED027F003039C
:1008600012AA134453F8203C05934046042205A9DC
:1008700000F0ACFA04378046E7E7384600F03AF972
:100880000590F2E7CDF81480042105A800F006F9E0
:1008900006E70023642104A8049300F0F5F800287B
:1008A0007FF4B4AE0220FFF771FD00283FF4AEAE36
:1008B000049800F051F90590E6E70023642104A8AC
:1008C000049300F0E1F800287FF4A0AE0220FFF7C7
:1008D0005DFD00283FF49AAE049800F04DF9EAE778
:1008E0000220FFF753FD00283FF490AE00F05CF9C2
:1008F000E1E70220FFF74AFD00283FF487AE05A993
:10090000142000F057F904210746049004A800F0D1
:10091000C5F83946B9E7322000F0A2F8071EFFF605
:1009200075AEBB077FF472AE384A926807EB0903D5
:1009300093423FF66BAE0220FFF728FD00283FF4FC
:1009400065AE27F003074F44B9453FF4A9AE4846CA
:1009500000F0D0F80421059005A800F09FF809F1F7
:100960000409F1E74FF47A70FFF710FD00283FF417
:100970004DAE00F009F9002844D00A9B01330BD09A
:1009800008220AA9002000F0A9F900283AD0202264
:10099000FF210AA800F09AF9FFF700FD1C4800F0BB
:1009A0003FFF13B0BDE8F08F002E3FF42FAE0BF0E9
:1009B0000B030B2B7FF42AAE0023642105A80593BB
:1009C00000F062F8074600287FF420AE0220FFF70F
:1009D000DDFC804600283FF419AEFFF7DFFC41F252
:1009E000883000F01DFF059800F0EEF9464600F053
:1009F000B9F93C46BBE5064652E64FF0000905E66C
:100A0000BA467EE637467CE65C22002000220020C3
:100A1000A086010070B50F4B1B780133DBB2012BB0
:100A20000C4611D80C4D29684FF47A730E6AA2FB5C
:100A30000332014622462846B047844204D1074B80
:100A400000221A70012070BD4FF4FA7000F0E8FE29
:100A50000020F8E710220020082600209423002020
:100A600007B50023024601210DF107008DF807307C
:100A7000FFF7D0FF20B19DF8070003B05DF804FB3D
:100A80004FF0FF30F9E700000A4608B50421FFF7F0
:100A9000C1FF80F00100C0B2404208BD30B4054C37
:100AA0002368DD69044B0A46AC460146204630BC4B
:100AB000604700BF08260020A086010070B501F045
:100AC000D1F9094E094D30800024286833888342CB
:100AD00008D901F0C1F92B6804440133B4F5803F13
:100AE0002B60F2D370BD00BF962300206823002046
:100AF00001F066BA00F1006000F5803000687047D0
:100B000000F10060920000F5803001F0F1B90000C2
:100B1000054B1A68054B1B889B1A834202D9104467
:100B200001F09AB900207047682300209623002026
:100B300038B5084D044629B128682044BDE838403E
:100B400001F0AAB92868204401F08EF90028F3D0FA
:100B500038BD00BF6823002010F003030AD1B0F5B0
:100B6000047F05D200F10050A0F51040D0F8003805
:100B7000184670470023FBE700F10050A0F5104035
:100B8000D0F8100A70470000064991F8243033B1BC
:100B90000023086A81F824300822FFF7B1BF012042
:100BA000704700BF6C230020014B1868704700BFDE
:100BB000002004E070B5194B1D68194B0138C5F3CE
:100BC0000B0408442D0C04221E88A6420BD15C683D
:100BD0000A46013C824213460FD214F9016F4EB10E
:100BE00002F8016BF6E7013A03F10803ECD1814208
:100BF0000B4602D22C2203F8012B0A4A0524168840
:100C0000AE4204D1984284BF967803F8016B013C50
:100C100002F10402F3D1581A70BD00BF002004E0B5
:100C20009C34000888340008022802BF024B4FF4AD
:100C300000129A61704700BF00040240022802BF00
:100C4000014B20229A61704700040240022801BF34
:100C5000024A536983F02003536170470004024045
:100C600070B504464FF47A764CB1412C254628BF26
:100C7000412506FB05F000F0D3FD641BF4E770BDD1
:100C800010B50023934203D0CC5CC4540133F9E780
:100C900010BD000010B5013810F9013F3BB191F9CA
:100CA00000409C4203D11AB10131013AF4E71AB174
:100CB00091F90020981A10BD1046FCE70346024641
:100CC000D01A12F9011B0029FAD1704702440346D9
:100CD000934202D003F8011BFAE770472DE9F8436D
:100CE0001F4D144695F824200746884652BBDFF86E
:100CF00070909CB395F824302BB92022FF214846F0
:100D00002F62FFF7E3FF95F82400C0F10802A2422A
:100D100028BF2246D6B24146920005EB8000FFF77D
:100D2000AFFF95F82430A41B1E44F6B2082E1744DA
:100D30009044E4B285F82460DBD1FFF725FF00285A
:100D4000D7D108E02B6A03EB82038342CFD0FFF7B1
:100D50001BFF0028CBD10020BDE8F8830120FBE772
:100D60006C230020024B1A78024B1A70704700BFA8
:100D7000942300201022002010B5104C104800F0E1
:100D8000B5F821460E4800F0DDF82468626DD2F80F
:100D9000043843F00203C2F804384FF47A70FFF7C6
:100DA0005FFF0849204600F0D3F9626DD2F804389D
:100DB00023F00203C2F8043810BD00BF68350008F4
:100DC00008260020703500087047000030B5094D36
:100DD0000A4491420DD011F8013B5840082340F3DA
:100DE0000004013B2C4013F0FF0384EA5000F6D1CD
:100DF000EFE730BD2083B8ED02684368114301601E
:100E000003B118477047000013B5446BD4F894340D
:100E10001A681178042915D1217C022912D1197977
:100E2000128901238B4013420CD101A904F14C001B
:100E300001F0FAFED4F89444019B2179024620681F
:100E400000F0D0F902B010BD143001F07DBE0000FA
:100E50004FF0FF33143001F077BE00004C3001F04A
:100E60004FBF00004FF0FF334C3001F049BF00008E
:100E7000143001F04BBE00004FF0FF31143001F090
:100E800045BE00004C3001F01BBF00004FF0FF32A8
:100E90004C3001F015BF00000020704710B5D0F8AD
:100EA00094341A6811780429044617D1017C022968
:100EB00014D15979528901238B4013420ED1143039
:100EC00001F0DEFD024648B1D4F894444FF480733B
:100ED00061792068BDE8104000F072B910BD0000D3
:100EE000406BFFF7DBBF0000704700007FB5124B7F
:100EF000036000234360C0E90233012502260F4B43
:100F0000057404460290019300F18402294600967C
:100F10004FF48073143001F08FFD094B0294CDE93A
:100F2000006304F523724FF48073294604F14C00EA
:100F300001F056FE04B070BDBC340008E10E00089C
:100F4000090E00080B68302282F311880A7903EB3E
:100F5000820290614A79093243F822008A7912B1FB
:100F600003EB820398610223C0F8941403740020F9
:100F700080F311887047000038B5037F044613B131
:100F800090F85430ABB9201D01250221FFF734FF42
:100F900004F1140025776FF0010100F069FC84F87A
:100FA000545004F14C006FF00101BDE8384000F0EE
:100FB0005FBC38BD10B5012104460430FFF71CFFAB
:100FC0000023237784F8543010BD000038B5044660
:100FD0000025143001F048FD04F14C00257701F0A4
:100FE00017FE201D84F854500121FFF705FF20460D
:100FF000BDE83840FFF752BF90F8443003F060037B
:10100000202B07D190F84520212A4FF0000303D868
:101010001F2A06D800207047222AFBD1C0E90E33D0
:1010200003E0034A82630722C2630364012070471E
:101030001122002037B5D0F894341A6811780429A9
:1010400004461AD1017C022917D11979128901238A
:101050008B40134211D100F14C05284601F098FE57
:1010600058B101A9284601F0DFFDD4F89444019B52
:1010700021790246206800F0B5F803B030BD0000C9
:10108000F0B500EB810385B09E6904460D46FEB1C4
:10109000302383F3118804EB8507301D0821FFF707
:1010A000ABFEFB685B691B6806F14C001BB101904D
:1010B00001F0C8FD019803A901F0B6FD024648B150
:1010C000039B2946204600F08DF8002383F3118806
:1010D00005B0F0BDFB685A691268002AF5D01B8A7A
:1010E000013B1340F1D104F14402EAE7093138B57C
:1010F00050F82140DCB1302383F31188D4F89424D4
:101100001368527903EB8203DB689B695D6845B124
:1011100004216018FFF770FE294604F1140001F065
:10112000B9FC2046FFF7BAFE002383F3118838BDCF
:101130007047000001F018B8012303700023C0E9D4
:101140000133C36183620362C36243620363704716
:1011500038B50446302383F311880025C0E90355D0
:10116000C0E90555416001F00FF80223237085F3B3
:101170001188284638BD000070B500EB8103054694
:101180005069DA600E46144618B110220021FFF7AC
:101190009DFDA06918B110220021FFF797FD31468F
:1011A0002846BDE8704001F0B9B80000826802F03E
:1011B000011282600022C0E90422826101F03AB982
:1011C000F0B400EB81044789E4680125A4698D40EF
:1011D0003D43458123600023A2606360F0BC01F0C1
:1011E00055B90000F0B400EB81040789E4680125DB
:1011F00064698D403D43058123600023A2606360E4
:10120000F0BC01F0CFB9000070B502230025044600
:101210000370C0E90255C0E90455C564856180F8D2
:10122000345001F017F863681B6823B12946204643
:10123000BDE87040184770BD0378052B10B5044613
:101240000AD080F850300523037043681B680BB147
:10125000042198470023A36010BD000001780529F0
:1012600006D190F85020436802701B6803B11847FC
:101270007047000070B590F83430044613B1002375
:1012800080F8343004F14402204601F0F5F8636838
:101290009B68B3B994F8443013F0600535D0002151
:1012A000204601F095FB0021204601F087FB636892
:1012B0001B6813B1062120469847062384F8343072
:1012C00070BD204698470028E4D0B4F84A30E26B5D
:1012D0009A4288BFE36394F94430E56B002B4FF0EA
:1012E000300380F20381002D00F0F280092284F89F
:1012F000342083F311880021D4E90E232046FFF720
:1013000071FF002383F31188DAE794F8452003F096
:101310007F0343EA022340F20232934200F0C58089
:1013200021D8B3F5807F48D00DD8012B3FD0022BB8
:1013300000F09380002BB2D104F14C02A263022290
:10134000E2632364C1E7B3F5817F00F09B80B3F5CE
:10135000407FA4D194F84630012BA0D1B4F84C3092
:1013600043F0020332E0B3F5006F4DD017D8B3F568
:10137000A06F31D0A3F5C063012B90D8636894F8B7
:1013800046205E6894F84710B4F848302046B047CD
:10139000002884D04368A3630368E3631AE0B3F5CD
:1013A000106F36D040F6024293427FF478AF5C4B28
:1013B000A3630223E3630023C3E794F84630012BC1
:1013C0007FF46DAFB4F84C3023F00203C4E90E553E
:1013D000A4F84C30256478E7B4F84430B3F5A06F36
:1013E0000ED194F8463084F84E30204600F08AFF43
:1013F00063681B6813B101212046984703232370BB
:101400000023C4E90E339CE704F14F03A3630123D7
:10141000C3E72378042B10D1302383F311882046AF
:10142000FFF7C4FE85F311880321636884F84F50E9
:1014300021701B680BB12046984794F84630002B6A
:10144000DED084F84F300423237063681B68002BC0
:10145000D6D0022120469847D2E794F848301D069E
:1014600003F00F0120460AD500F0F8FF012804D050
:1014700002287FF414AF2B4B9AE72B4B98E700F030
:10148000DFFFF3E794F84630002B7FF408AF94F8C1
:10149000483013F00F01B3D01A06204602D501F0F0
:1014A000ABFAADE701F09EFAAAE794F84630002BBC
:1014B0007FF4F5AE94F8483013F00F01A0D01B066E
:1014C000204602D501F084FA9AE701F077FA97E70F
:1014D000142284F8342083F311882B462A462946A7
:1014E0002046FFF76DFE85F31188E9E65DB1152210
:1014F00084F8342083F311880021D4E90E23204698
:10150000FFF75EFEFDE60B2284F8342083F311889A
:101510002B462A4629462046FFF764FEE3E700BF34
:10152000EC340008E4340008E834000838B590F8DA
:1015300034300446002B3ED0063BDAB20F2A34D8B2
:101540000F2B32D8DFE803F0373131082232313146
:101550003131313131313737C56BB0F84A309D42C6
:1015600014D2C3681B8AB5FBF3F203FB12556DB9A5
:10157000302383F311882B462A462946FFF732FE93
:1015800085F311880A2384F834300EE0142384F89C
:101590003430302383F3118800231A46194620463D
:1015A000FFF70EFE002383F3118838BD036C03B1EF
:1015B00098470023E7E70021204601F009FA0021BF
:1015C000204601F0FBF963681B6813B10621204631
:1015D00098470623D7E7000010B590F83430142B55
:1015E000044629D017D8062B05D001D81BB110BD51
:1015F000093B022BFBD80021204601F0E9F900212C
:10160000204601F0DBF963681B6813B10621204610
:101610009847062319E0152BE9D10B2380F83430C5
:10162000302383F3118800231A461946FFF7DAFDA9
:10163000002383F31188DAE7C3689B695B68002B9A
:10164000D5D1036C03B19847002384F83430CEE73A
:1016500000230375826803691B6899689142FBD275
:101660005A68036042601060586070470023037539
:10167000826803691B6899689142FBD85A680360C5
:10168000426010605860704708B50846302383F305
:1016900011880B7D032B05D0042B0DD02BB983F3C0
:1016A000118808BD8B6900221A604FF0FF338361F7
:1016B000FFF7CEFF0023F2E7D1E9003213605A6052
:1016C000F3E70000FFF7C4BF054BD9680875186839
:1016D00002681A60536001220275D860FEF712BEDC
:1016E0009823002030B50C4BDD684B1C87B00446B6
:1016F0000FD02B46094A684600F04EF92046FFF706
:10170000E3FF009B13B1684600F050F9A86907B0E9
:1017100030BDFFF7D9FFF9E79823002089160008AC
:10172000044B1A68DB6890689B68984294BF00205D
:101730000120704798230020084B10B51C68D8681A
:1017400022681A60536001222275DC60FFF78EFF69
:1017500001462046BDE81040FEF7D4BD9823002086
:1017600038B5074C074908480123002523706560F8
:1017700001F046FB0223237085F3118838BD00BFBA
:1017800000260020F43400089823002000F044B91B
:10179000034A516853685B1A9842FBD8704700BFF0
:1017A000001000E08B60022308618B8208467047BE
:1017B0008368A3F1840243F8142C026943F8442C93
:1017C000426943F8402C094A43F8242CC26843F884
:1017D000182C022203F80C2C002203F80B2C044ACC
:1017E00043F8102CA3F12000704700BF1D03000830
:1017F0009823002008B5FFF7DBFFBDE80840FFF79E
:1018000061BF0000024BDB6898610F20FFF75CBFEF
:1018100098230020302383F31188FFF7F3BF0000E3
:1018200008B50146302383F311880820FFF75AFFDB
:10183000002383F3118808BD064BDB6839B1426889
:1018400018605A60136043600420FFF74BBF4FF0ED
:10185000FF307047982300200368984206D01A682A
:101860000260506099611846FFF72CBF7047000076
:1018700038B504460D462068844200D138BD03685F
:1018800023605C608561FFF71DFFF4E710B5036816
:101890009C68A2420CD85C688A600B604C60216036
:1018A000596099688A1A9A604FF0FF33836010BDBF
:1018B0001B68121BECE700000A2938BF0A2170B52B
:1018C00004460D460A26601901F094FA01F080FAE8
:1018D000041BA54203D8751C2E460446F3E70A2EC6
:1018E00004D9BDE87040012001F0CABA70BD000003
:1018F000F8B5144B0D46D96103F1100141600A2A75
:101900001969826038BF0A22016048601861A8180E
:10191000144601F061FA0A2701F05AFA431BA34268
:10192000064606D37C1C281901F064FA2746354682
:10193000F2E70A2F04D9BDE8F840012001F0A0BA6F
:10194000F8BD00BF98230020F8B506460D4601F00B
:101950003FFA0F4A134653F8107F9F4206D12A469A
:1019600001463046BDE8F840FFF7C2BFD169BB6809
:10197000441A2C1928BF2C46A34202D92946FFF746
:101980009BFF224631460348BDE8F840FFF77EBF83
:1019900098230020A823002010B4C0E903230023CB
:1019A0005DF8044B4361FFF7CFBF000010B5194C41
:1019B000236998420DD0D0E90032816813605A60E3
:1019C0009A680A449A60002303604FF0FF33A361D2
:1019D00010BD2346026843F8102F536000220260B6
:1019E00022699A4203D1BDE8104001F0FDB9936825
:1019F00081680B44936001F0EBF92269E169926818
:101A0000441AA242E4D91144BDE81040091AFFF774
:101A100053BF00BF982300202DE9F047DFF8BC80BA
:101A200008F110072C4ED8F8105001F0D1F9D8F871
:101A30001C40AA68031B9A423ED81444D5E90032E0
:101A40004FF00009C8F81C4013605A60C5F80090B8
:101A5000D8F81030B34201D101F0C6F989F31188EA
:101A6000D5E9033128469847302383F311886B6901
:101A7000002BD8D001F0ACF96A69A0EB04094A4503
:101A800082460DD2022001F0FBF90022D8F8103076
:101A9000B34208D151462846BDE8F047FFF728BFBA
:101AA000121A2244F2E712EB090938BF4A462946C6
:101AB0003846FFF7EBFEB5E7D8F81030B34208D050
:101AC0001444211AC8F81C00A960BDE8F047FFF7CC
:101AD000F3BEBDE8F08700BFA823002098230020B4
:101AE00000207047FEE70000704700004FF0FF3015
:101AF0007047000002290CD0032904D001290748AF
:101B000018BF00207047032A05D8054800EBC20023
:101B10007047044870470020704700BFCC3500086C
:101B2000202200208035000870B59AB0054608468E
:101B300001A9144600F0C2F801A8FFF7BFF8431C42
:101B40005B00C5E900340022237003236370C6B232
:101B500001AB02341046D1B28E4204F1020401D826
:101B60001AB070BD13F8011B04F8021C04F8010C34
:101B70000132F0E708B5302383F311880348FFF7FB
:101B800059FA002383F3118808BD00BF08260020FE
:101B900090F8443003F01F02012A07D190F8452045
:101BA0000B2A03D10023C0E90E3315E003F06003D4
:101BB000202B08D1B0F848302BB990F84520212AC5
:101BC00003D81F2A04D8FFF717BA222AEBD0FAE766
:101BD000034A82630722C26303640120704700BF87
:101BE0001822002007B5052917D8DFE801F01916DB
:101BF00003191920302383F31188104A0190012121
:101C0000FFF7BAFA01980E4A0221FFF7B5FA0D481C
:101C1000FFF7DCF9002383F3118803B05DF804FBC0
:101C2000302383F311880748FFF7A6F9F2E7302342
:101C300083F311880348FFF7BDF9EBE7203500086F
:101C4000443500080826002038B50C4D0C4C0D49D1
:101C50002A4604F10800FFF767FF05F1CA0204F104
:101C600010000949FFF760FF05F5CA7204F118007A
:101C70000649BDE83840FFF757BF00BFD02A002013
:101C800020220020003500080A350008153500081C
:101C900070B5044608460D46FFF710F8C6B2204658
:101CA000013403780BB9184670BD32462946FEF759
:101CB000F1FF0028F3D10120F6E700002DE9F047FD
:101CC00005460C46FEF7FAFF2C49C6B22846FFF738
:101CD000DFFF08B10C36F6B229492846FFF7D8FFD6
:101CE00008B11036F6B2632E0BD8DFF89080DFF81B
:101CF0009090244FDFF898A02E7846B92670BDE862
:101D0000F08729462046BDE8F04701F09FBB252E0D
:101D100030D1072241462846FEF7BCFF80B91A4B56
:101D2000224603F1100153F8040B42F8040B8B42D6
:101D3000F9D119889B781180937007351334DBE74C
:101D4000082249462846FEF7A5FF98B90F4BA21C6A
:101D5000197809090232C95D02F8041C13F8011B45
:101D600001F00F015345C95D02F8031CF0D118348E
:101D70000835C1E704F8016B0135BDE7EC35000813
:101D80001535000808360008F4350008107AFF1FE2
:101D90001C7AFF1FBFF34F8F024AD368DB03FCD4CA
:101DA000704700BF003C024008B5094B1B7873B96F
:101DB000FFF7F0FF074B1A69002ABFBF064A5A60B7
:101DC00002F188325A601A6822F480621A6008BDF3
:101DD0002E2D0020003C02402301674508B50B4B27
:101DE0001B7893B9FFF7D6FF094B1A6942F00042FE
:101DF0001A611A6842F480521A601A6822F48052FA
:101E00001A601A6842F480621A6008BD2E2D002004
:101E1000003C02400B28F0B516D80C4C0C49237836
:101E20007BB90C4D0E460C234FF0006255F8047B35
:101E300046F8042B013B13F0FF033A44F6D101238B
:101E4000237051F82000F0BD0020FCE7602D002039
:101E5000302D00201C360008014B53F8200070473D
:101E60001C3600080C2070470B2810B5044601D919
:101E7000002010BDFFF7CEFF064B53F82430184466
:101E8000C21A0BB90120F4E712680132F0D1043B09
:101E9000F6E700BF1C3600080B2810B5044621D811
:101EA000FFF778FFFFF780FF0F4AF323D360C300EB
:101EB000DBB243F4007343F002031361136943F48C
:101EC00080331361FFF766FFFFF7A4FF074B53F85A
:101ED000241000F0D9F8FFF781FF2046BDE810403C
:101EE000FFF7C2BF002010BD003C02401C360008B6
:101EF000F8B512F00103144642D18218B2F1016F15
:101F000057D82D4B1B6813F0010352D02B4DFFF710
:101F10004BFFF323EB60FFF73DFF40F20127032C5B
:101F200015D824F001046618244C401A40F2011719
:101F3000B142236900EB010524D123F001032361A1
:101F4000FFF74CFF0120F8BD043C0430E7E78307AE
:101F5000E7D12B6923F440732B612B693B432B6141
:101F600051F8046B0660BFF34F8FFFF713FF036850
:101F70009E42E9D02B6923F001032B61FFF72EFF6E
:101F80000020E0E723F44073236123693B4323618E
:101F90000B882B80BFF34F8FFFF7FCFE2D8831F8A5
:101FA000023BADB2AB42C3D0236923F001032361EE
:101FB000E4E71846C7E700BF00380240003C024093
:101FC000084908B50B7828B11BB9FFF7EDFE0123CE
:101FD0000B7008BD002BFCD0BDE808400870FFF76F
:101FE000FDBE00BF2E2D002010B50244064BD2B21C
:101FF000904200D110BD441C00B253F8200041F8BB
:10200000040BE0B2F4E700BF502800400F4B30B59E
:102010001C6F240407D41C6F44F400741C671C6FED
:1020200044F400441C670A4C236843F48073236023
:102030000244084BD2B2904200D130BD441C00B2E1
:1020400051F8045B43F82050E0B2F4E70038024056
:10205000007000405028004007B5012201A900206F
:10206000FFF7C2FF019803B05DF804FB13B5044607
:10207000FFF7F2FFA04205D0012201A90020019440
:10208000FFF7C4FF02B010BD70470000034B1A6891
:102090001AB9034AD2F874281A607047642D0020D8
:1020A0000030024008B5FFF7F1FF024B1868C0F39B
:1020B000407008BD642D002070470000FEE700005E
:1020C0000A4B0B480B4A90420BD30B4BDA1C121AEB
:1020D000C11E22F003028B4238BF00220021FEF70E
:1020E000F5BD53F8041B40F8041BECE7C8370008A3
:1020F000602E0020602E0020602E002070B5D0E9F8
:1021000015439E6800224FF0FF3504EB4213510146
:10211000D3F800090028BEBFD3F8000940F0804082
:10212000C3F80009D3F8000B0028BEBFD3F8000B9A
:1021300040F08040C3F8000B013263189642C3F8A8
:102140000859C3F8085BE0D24FF00113C4F81C38FB
:1021500070BD0000890141F02001016103699B0607
:10216000FCD41220FFF714BB10B5054C2046FEF737
:10217000E3FF4FF0A0436365024BA36510BD00BFB2
:10218000682D00207036000870B50378012B0546D5
:1021900050D12A4B446D98421BD1294B5A6B42F0C7
:1021A00080025A635A6D42F080025A655A6D5A692C
:1021B00042F080025A615A6922F080025A610E216F
:1021C00043205B6900F022FC1E4BE3601E4BC4F809
:1021D00000380023C4F8003EC02323606E6D4FF426
:1021E0000413A3633369002BFCDA012333610C2051
:1021F000FFF7CEFA3369DB07FCD41220FFF7C8FAE9
:102200003369002BFCDA0026A6602846FFF776FF2C
:102210006B68C4F81068DB68C4F81468C4F81C68FC
:102220004BB90A4BA3614FF0FF336361A36843F0DE
:102230000103A36070BD064BF4E700BF682D0020CA
:10224000003802404014004003002002003C30C02F
:10225000083C30C0F8B5446D054600212046FFF724
:1022600079FFA96D00234FF001128F68C4F834384C
:102270004FF00066C4F81C284FF0FF3004EB431207
:1022800001339F42C2F80069C2F8006BC2F8080926
:10229000C2F8080BF2D20B686A6DEB65636210231B
:1022A0001361166916F01006FBD11220FFF770FAC1
:1022B000D4F8003823F4FE63C4F80038A36943F46B
:1022C000402343F01003A3610923C4F81038C4F875
:1022D00014380A4BEB604FF0C043C4F8103B084B76
:1022E000C4F8003BC4F81069C4F80039EB6D03F181
:1022F000100243F48013EA65A362F8BD4C3600086F
:1023000040800010426D90F84E10D2F8003823F44F
:10231000FE6343EA0113C2F8003870472DE9F84321
:1023200000EB8103456DDA68166806F00306731E3C
:10233000022B05EB41130C4680460FFA81F94FEA58
:1023400041104FF00001C3F8101B4FF0010104F1E0
:10235000100398BFB60401FA03F391698EBF334EA0
:1023600006F1805606F5004600293AD0578A04F156
:102370005801490137436F50D5F81C180B43C5F875
:102380001C382B180021C3F8101953690127611E4E
:10239000A7409BB3138A928B9B08012A88BF5343A3
:1023A000D8F85C20981842EA034301F1400205EB9B
:1023B0008202C8F85C00214653602846FFF7CAFE37
:1023C00008EB8900C3681B8A43EA845348346401DC
:1023D0001E432E51D5F81C381F43C5F81C78BDE8A4
:1023E000F88305EB4917D7F8001B21F40041C7F823
:1023F000001BD5F81C1821EA0303C0E704F13F03D2
:1024000005EB83030A4A5A6028462146FFF7A2FEDD
:1024100005EB4910D0F8003923F40043C0F8003927
:10242000D5F81C3823EA0707D7E700BF0080001063
:1024300000040002826D1268C265FFF75FBE0000F3
:102440005831436D49015B5813F4004004D013F434
:10245000001F0CBF02200120704700004831436D6F
:1024600049015B5813F4004004D013F4001F0CBF63
:10247000022001207047000000EB8101CB68196A3F
:102480000B6813604B6853607047000000EB8103DA
:1024900030B5DD68AA691368D36019B9402B84BFD1
:1024A000402313606B8A1468426D1C44013CB4FBEA
:1024B000F3F46343033323F0030302EB411043EAD5
:1024C000C44343F0C043C0F8103B2B6803F0030340
:1024D000012B09B20ED1D2F8083802EB411013F4E7
:1024E000807FD0F8003B14BF43F0805343F000538B
:1024F000C0F8003B02EB4112D2F8003B43F004432A
:10250000C2F8003B30BD00002DE9F041244D6E6D56
:1025100006EB40130446D3F8087BC3F8087B380762
:102520000AD5D6F81438190706D505EB84032146D9
:10253000DB6828465B689847FA071FD5D6F8143839
:10254000DB071BD505EB8403D968CCB98B69488AB6
:102550005A68B2FBF0F600FB16228AB91868DA68EE
:1025600090420DD2121AC3E90024302383F311885C
:102570000B482146FFF78AFF84F31188BDE8F081FC
:10258000012303FA04F26B8923EA02036B81CB680F
:10259000002BF3D021460248BDE8F041184700BFA8
:1025A000682D002000EB810370B5DD68436D6C6918
:1025B0002668E6604A0156BB1A444FF40020C2F870
:1025C00010092A6802F00302012A0AB20ED1D3F8D8
:1025D000080803EB421410F4807FD4F8000914BFFC
:1025E00040F0805040F00050C4F8000903EB421264
:1025F000D2F8000940F00440C2F80009D3F83408CA
:10260000012202FA01F10143C3F8341870BD19B96F
:10261000402E84BF4020206020682E8A8419013C0F
:10262000B4FBF6F440EAC44040F000501A44C6E758
:102630002DE9F8433B4D6E6D06EB40130446D3F88D
:102640000889C3F8088918F0010F4FEA40171AD01B
:10265000D6F81038DB0716D505EB8003D9684B692F
:102660001868DA68904230D2121A4FF000091A60E6
:10267000C3F80490302383F3118821462846FFF7DE
:1026800091FF89F3118818F0800F1CD0D6F83438E8
:102690000126A640334216D005EB84036D6DD3F8B6
:1026A0000CC0DCF814200134E4B2D2F800E005EBF1
:1026B00004342F445168714515D3D5F8343823EAD2
:1026C0000606C5F83468BDE8F883012303FA04F26E
:1026D0002B8923EA02032B818B68002BD3D0214660
:1026E00028469847CFE7BCF81000AEEB01038342C1
:1026F00028BF0346D7F8180980B2B3EB800FE2D8A1
:102700009068A0F1040959F8048FC4F80080A0EB88
:1027100009089844B8F1040FF5D818440B449060A8
:102720005360C7E7682D00202DE9F74FA24C656D77
:102730006E69AB691E4016F480586E6107D0204662
:10274000FEF762FD03B0BDE8F04F00F047BC002E7D
:1027500012DAD5F8003E98489B071EBFD5F8003E18
:1027600023F00303C5F8003ED5F8043823F0010335
:10277000C5F80438FEF772FD370505D58E48FFF71A
:10278000BDFC8D48FEF758FDB0040CD5D5F80838CF
:1027900013F0060FEB6823F470530CBF43F410538F
:1027A00043F4A053EB6031071BD56368DB681BB9AA
:1027B000AB6923F00803AB612378052B0CD1D5F866
:1027C000003E7D489A071EBFD5F8003E23F0030364
:1027D000C5F8003EFEF742FD6368DB680BB1764842
:1027E0009847F30274D4B70227D5D4F85490DFF891
:1027F000C8B100274FF0010A09EB4712D2F8003B9D
:1028000003F44023B3F5802F11D1D2F8003B002B05
:102810000DDA62890AFA07F322EA0303638104EB03
:102820008703DB68DB6813B1394658469847A36DC8
:1028300001379B68FFB29F42DED9F00617D5676D5E
:102840003A6AC2F30A1002F00F0302F4F012B2F572
:10285000802F00F08580B2F5402F08D104EB830370
:102860000022DB681B6A07F5805790426AD130036B
:10287000D5F8184813D5E10302D50020FFF744FE30
:10288000A20302D50120FFF73FFE630302D5022019
:10289000FFF73AFE270302D50320FFF735FE750345
:1028A0007FF550AFE00702D50020FFF7C1FEA1077A
:1028B00002D50120FFF7BCFE620702D50220FFF718
:1028C000B7FE23077FF53EAF0320FFF7B1FE39E7E0
:1028D000636DDFF8E4A0019300274FF00109A36DB9
:1028E0009B685FFA87FB9B453FF67DAF019B03EB3F
:1028F0004B13D3F8001901F44021B1F5802F1FD1FB
:10290000D3F8001900291BDAD3F8001941F09041DF
:10291000C3F80019D3F800190029FBDB5946606D94
:10292000FFF718FC218909FA0BF321EA030323813D
:1029300004EB8B03DB689B6813B1594650469847FC
:102940000137CCE7910708BFD7F80080072A98BF66
:1029500003F8018B02F1010298BF4FEA182884E7BF
:10296000023304EB830207F580575268D2F818C08F
:10297000DCF80820DCE9001CA1EB0C0C00218842EB
:102980000AD104EB830463689B699A6802449A60E5
:102990005A6802445A606AE711F0030F08BFD7F87B
:1029A00000808C4588BF02F8018B01F1010188BFCE
:1029B0004FEA1828E3E700BF682D0020436D03EBC2
:1029C0004111D1F8003B43F40013C1F8003B7047BC
:1029D000436D03EB4111D1F8003943F40013C1F802
:1029E00000397047436D03EB4111D1F8003B23F4EC
:1029F0000013C1F8003B7047436D03EB4111D1F860
:102A0000003923F40013C1F80039704700F1604326
:102A100003F561430901C9B283F80013012200F0F4
:102A20001F039A4043099B0003F1604303F5614390
:102A3000C3F880211A60704730B5039C01720433DB
:102A400004FB0325C0E90653049B03630021059B97
:102A5000C160C0E90000C0E90422C0E90842C0E941
:102A60000A11436330BD0000416A0022C0E904112D
:102A7000C0E90A22C2606FF00101FEF7F9BE000052
:102A8000D0E90432934201D1C2680AB9181D7047D7
:102A90000020704703691960C2680132C260C269D0
:102AA000134482690361934224BF436A0361002196
:102AB000FEF7D2BE38B504460D46E3683BB1626905
:102AC000131D1268A3621344E362002007E0237A17
:102AD00033B929462046FEF7AFFE0028EDDA38BDAF
:102AE0006FF00100FBE70000C368C269013BC360EF
:102AF0004369134482694361934224BF436A43613B
:102B000000238362036B03B11847704770B530230D
:102B1000044683F31188866A3EB9FFF7CBFF05466A
:102B200018B186F31188284670BDA36AE26A13F8CB
:102B3000015BA362934202D32046FFF7D5FF002337
:102B400083F31188EFE700002DE9F84F04460E46A5
:102B5000174698464FF0300989F311880025AA4698
:102B6000D4F828B0BBF1000F09D141462046FFF749
:102B7000A1FF20B18BF311882846BDE8F88FD4E976
:102B80000A12A7EB050B521A934528BF9346BBF1D7
:102B9000400F1BD9334601F1400251F8040B43F8B2
:102BA000040B9142F9D1A36A40334036A362403509
:102BB000D4E90A239A4202D32046FFF795FF8AF30D
:102BC0001188BD42D8D289F31188C9E730465A46E8
:102BD000FEF756F8A36A5B445E44A3625D44E7E7F0
:102BE00010B5029C0172043303FB0421C0E90613F3
:102BF0000023C0E90A33039B0363049BC460C0E95C
:102C00000000C0E90422C0E90842436310BD00008F
:102C1000026AC260426AC0E904220022C0E90A22B4
:102C20006FF00101FEF724BED0E904239A4201D1DE
:102C3000C26822B9184650F8043B0B607047002365
:102C40001846FAE7C368C2690133C3604369134495
:102C500082694361934224BF436A43610021FEF7C6
:102C6000FBBD000038B504460D46E3683BB123695F
:102C70001A1DA262E2691344E362002007E0237A8E
:102C800033B929462046FEF7D7FD0028EDDA38BDD6
:102C90006FF00100FBE7000003691960C268013AA8
:102CA000C260C269134482690361934224BF436ACC
:102CB000036100238362036B03B118477047000070
:102CC00070B530230D460446114683F31188866A99
:102CD0002EB9FFF7C7FF10B186F3118870BDA36A44
:102CE0001D70A36AE26A01339342A36204D3E169CF
:102CF00020460439FFF7D0FF002080F31188EDE76C
:102D00002DE9F84F04460D46904699464FF0300A9B
:102D10008AF311880026B346A76A4FB94946204670
:102D2000FFF7A0FF20B187F311883046BDE8F88F88
:102D3000D4E90A073A1AA8EB0607974228BF1746B4
:102D4000402F1BD905F1400355F8042B40F8042B04
:102D50009D42F9D1A36A4033A3624036D4E90A23E5
:102D60009A4204D3E16920460439FFF795FF8BF3BB
:102D700011884645D9D28AF31188CDE729463A46CB
:102D8000FDF77EFFA36A3B443D44A3623E44E5E772
:102D9000D0E904239A4217D1C3689BB1836A8BB1EF
:102DA000043B9B1A0ED01360C368013BC360C36928
:102DB0001A44836902619A4224BF436A0361002373
:102DC00083620123184670470023FBE700F030B907
:102DD0004FF08043586A70474FF080430022586399
:102DE0001A610222DA6070474FF080430022DA60F5
:102DF000704700004FF0804358637047FEE70000C3
:102E000070B51B4B01630025044686B0586085628F
:102E10000E4600F0BFF804F11003C4E904334FF08C
:102E2000FF33C4E90635C4E90044A560E562FFF755
:102E3000CFFF2B460246C4E9082304F134010D4AB2
:102E4000256580232046FEF7ADFC0123E0600A4A99
:102E50000375009272680192B268CDE90223074BB4
:102E60006846CDE90435FEF7C5FC06B070BD00BF6D
:102E7000002600207C36000881360008FD2D000861
:102E8000024AD36A1843D062704700BF98230020DB
:102E90004B6843608B688360CB68C3600B69436198
:102EA0004B6903628B6943620B68036070470000E3
:102EB00008B5264B26481A6940F2FF110A431A61E9
:102EC0001A6922F4FF7222F001021A611A691A6B60
:102ED0000A431A631A6D0A431A651E4A1B6D11468E
:102EE000FFF7D6FF02F11C0100F58060FFF7D0FF6D
:102EF00002F1380100F58060FFF7CAFF02F15401CA
:102F000000F58060FFF7C4FF02F1700100F58060FA
:102F1000FFF7BEFF02F18C0100F58060FFF7B8FFFC
:102F200002F1A80100F58060FFF7B2FF02F1C401D1
:102F300000F58060FFF7ACFF02F1E00100F5806072
:102F4000FFF7A6FFBDE8084000F0EEB800380240E9
:102F5000000002408836000808B500F059FAFEF774
:102F6000FFFBFFF793F8BDE80840FEF76DBE0000D9
:102F700070470000EFF3098305494A6B22F0010214
:102F80004A63683383F30988002383F31188704709
:102F900000EF00E0302080F3118862B60C4B0D4A40
:102FA000D96821F4E0610904090C0A43DA60D3F816
:102FB000FC20094942F08072C3F8FC200A6842F004
:102FC00001020A602022DA7783F82200704700BFEE
:102FD00000ED00E00003FA05001000E010B530231A
:102FE00083F311880E4B5B6813F4006314D0F1EE89
:102FF000103AEFF30984683C4FF08073E361094BAA
:10300000DB6B236684F30988FEF78AFB10B1064B5D
:10301000A36110BD054BFBE783F31188F9E700BFFF
:1030200000ED00E000EF00E02F030008320300088D
:103030000F4B1A6C42F001021A641A6E42F0010240
:103040001A660C4A1B6E936843F0010393604FF0BD
:10305000804353229A624FF0FF32DA6200229A6173
:103060005A63DA605A6001225A611A60704700BFE1
:1030700000380240002004E04FF0804208B511699A
:10308000D3680B40D9B2C9439B07116107D53023E0
:1030900083F31188FEF77AFB002383F3118808BDC0
:1030A0001F4B1A696FEAC2526FEAD2521A611A694B
:1030B000C2F308021A614FF0FF301A695A69586169
:1030C00000215A6959615A691A6A62F080521A627B
:1030D0001A6A02F080521A621A6A5A6A58625A6A66
:1030E00059625A6A1A6C42F080521A641A6E42F09F
:1030F00080521A661A6E0B4A106840F48070106095
:10310000186F00F44070B0F5007F1EBF4FF48030A0
:1031100018671967536823F40073536000F054B9BB
:103120000038024000700040334B4FF080521A6468
:10313000324A4FF4404111601A6842F001021A60AD
:103140001A689107FCD59A6822F003029A602A4B0C
:103150009A6812F00C02FBD1196801F0F9011960AC
:103160009A601A6842F480321A601A689203FCD599
:103170005A6F42F001025A671F4B5A6F9007FCD5F5
:103180001F4A5A601A6842F080721A601B4A5368DC
:103190005904FCD5184B1A689201FCD5194A9A605B
:1031A000194B1A68194B9A42194B21D1194A1168C7
:1031B000194A91421CD140F205121A60144A136850
:1031C00003F00F03052BFAD10B4B9A6842F0020271
:1031D0009A609A6802F00C02082AFAD15A6C42F4FA
:1031E00080425A645A6E42F480425A665B6E70475F
:1031F00040F20572E1E700BF003802400070004075
:103200000854400700948838002004E0116400202E
:10321000003C024000ED00E041C20F41074A08B502
:10322000536903F00103536123B1054A13680BB1DD
:1032300050689847BDE80840FFF7D0BE003C014009
:10324000E02D0020074A08B5536903F002035361DB
:1032500023B1054A93680BB1D0689847BDE8084090
:10326000FFF7BCBE003C0140E02D0020074A08B536
:10327000536903F00403536123B1054A13690BB189
:1032800050699847BDE80840FFF7A8BE003C0140E0
:10329000E02D0020074A08B5536903F00803536185
:1032A00023B1054A93690BB1D0699847BDE808403E
:1032B000FFF794BE003C0140E02D0020074A08B50E
:1032C000536903F01003536123B1054A136A0BB12C
:1032D000506A9847BDE80840FFF780BE003C0140B7
:1032E000E02D0020164B10B55C6904F478725A6129
:1032F000A30604D5134A936A0BB1D06A98476006B7
:1033000004D5104A136B0BB1506B9847210604D5B6
:103310000C4A936B0BB1D06B9847E20504D5094A70
:10332000136C0BB1506C9847A30504D5054A936CF8
:103330000BB1D06C9847BDE81040FFF74FBE00BFFF
:10334000003C0140E02D0020194B10B55C6904F4ED
:103350007C425A61620504D5164A136D0BB1506D5B
:103360009847230504D5134A936D0BB1D06D984748
:10337000E00404D50F4A136E0BB1506E9847A104B8
:1033800004D50C4A936E0BB1D06E9847620404D5F5
:10339000084A136F0BB1506F9847230404D5054AB0
:1033A000936F0BB1D06F9847BDE81040FFF716BE82
:1033B000003C0140E02D002008B5FFF75DFEBDE8B0
:1033C0000840FFF70BBE0000062108B50846FFF7CE
:1033D0001DFB06210720FFF719FB06210820FFF738
:1033E00015FB06210920FFF711FB06210A20FFF734
:1033F0000DFB06211720FFF709FB06212820FFF708
:1034000005FBBDE8084007211C20FFF7FFBA0000BC
:1034100008B5FFF745FE00F00BF8FDF78BFEFDF752
:1034200063FDFFF7A5FDBDE80840FFF7CFBC000036
:103430000023054A19460133102BC2E9001102F19D
:103440000802F8D1704700BFE02D0020034611F8B4
:10345000012B03F8012B002AF9D1704753544D3347
:1034600032463F3F3F0053544D33324634307800AC
:1034700053544D3332463432780053544D33324630
:103480003434365858000000012033000010410049
:1034900001105A000310590007103100000000000D
:1034A0005C340008130400006634000819040000AE
:1034B00070340008210400007A3400080000000085
:1034C000650E0008510E00088D0E0008790E0008E8
:1034D000850E0008710E00085D0E0008490E0008F8
:1034E000990E00080000000001000000000000002C
:1034F00063300000F0340008F02300200026002094
:103500004172647550696C6F740025424F4152449A
:10351000252D424C002553455249414C25000000C1
:10352000020000000000000081100008ED100008FB
:1035300040004000A02A0020B02A00200200000025
:10354000000000000300000000000000311100082E
:103550000000000010000000C02A00200000000051
:103560000100000000000000682D002001010200A1
:10357000E51B0008F51A0008911B0008751B0008E0
:10358000430000008835000809024300020100C022
:1035900032090400000102020100052400100105A7
:1035A000240100010424020205240600010705820B
:1035B000030800FF09040100020A000000070501DA
:1035C00002400000070581024000000012000000D8
:1035D000D4350008120110010200004009124157C1
:1035E00000020102030100000403090425424F41C7
:1035F000524425006F6D6E69627573663470726F28
:103600002D626473686F740030313233343536376D
:103610003839414243444546000000000040000064
:1036200000400000004000000040000000000100D9
:103630000000020000000200000002000000020082
:103640000000020000000200000002000000000074
:10365000751200082D150008D9150008400040001B
:10366000C82D0020C82D002001000000D82D00200A
:103670008000000040010000030000006D61696EE1
:103680000069646C650000000001804200000000D9
:10369000AAAAAAAA00010040FFFF00000000000043
:1036A00000A00A004005000100000000AAAAAAAA82
:1036B00040020001CFFF00000000000000000000F9
:1036C0000000000000000000AAAAAAAA0000000052
:1036D000FFFF0000000000000000000000000000EC
:1036E00000000000AAAAAAAA00000000FFFF000034
:1036F00000000000000000000000000000000000CA
:10370000AAAAAAAA00000000FFFF00000000000013
:10371000000000000000000000000000AAAAAAAA01
:1037200000000000FFFF000000000000000000009B
:103730000000000000000000AAAAAAAA00000000E1
:10374000FFFF00000000000000000000000000007B
:10375000000000000A00000000000000030000005C
:103760000000000000000000000000000000000059
:103770000000000000000000000000000000000049
:1037800000000000000000008300000000000000B6
:1037900000000F0000000000FF009600000000087D
:1037A000009600000000080004000000E835000852
:1037B0000000000000000000000000000000000009
:1037C0000000000000000000FFFFFFFFFFFFFFFF01
:1037D000FFFFFFFFFFFFFFFFFFFFFFFFFFFFFFFFF9
:1037E000FFFFFFFFFFFFFFFFFFFFFFFFFFFFFFFFE9
:1037F000FFFFFFFFFFFFFFFFFFFFFFFFFFFFFFFFD9
:10380000FFFFFFFFFFFFFFFFFFFFFFFFFFFFFFFFC8
:020000040801F1
:1000000000060020A9120108497A0A08A5790A0801
:10001000117A0A08A5790A08DD790A08AB120108E5
:10002000AB120108AB120108AB120108250F0D0835
:10003000AB120108AB120108AB120108AB120108A8
:10004000AB120108AB120108AB120108AB12010898
:10005000AB120108AB120108BD1A0D08E51A0D0814
:100060000D1B0D08351B0D085D1B0D08E1BF0C08AD
:1000700009C00C0835C00C0861C00C088DC00C0804
:10008000B5C00C08E1C00C0865BF0C08AB12010834
:10009000AB120108AB120108AB120108851B0D0859
:1000A000A91C0D08AD1C0D08C11C0D08C51C0D08B0
:1000B000C91C0D08DD1C0D08F11C0D08AB12010850
:1000C000AB1201086DC60C0815C80C08AB1201086C
:1000D000AB120108591C0D08AB1201086D1C0D086C
:1000E000E91B0D08AB120108AB120108151D0D0824
:1000F000191D0D082D1D0D08311D0D080DC10C0811
:10010000AB120108AB120108051D0D08AB12010866
:10011000811C0D08AB120108AB120108AB120108DB
:1001200039C10C0861C10C088DC10C08B9C10C089B
:10013000E5C10C08AB120108AB120108AB120108B3
:10014000AB120108AB120108AB12010851160D08E1
:100150000DC20C0839C20C0865C20C08951C0D08AC
:10016000AB120108AB120108AB120108AB12010877
:10017000AB120108AB120108AB120108AB12010867
:10018000AB120108AB120108AB120108AB12010857
:10019000AB120108AB120108AB120108AB12010847
:1001A000AB120108AB120108AB120108AB12010837
:1001B000AB120108AB120108AB120108AB12010827
:1001C000AB120108AB120108AB120108AB12010817
:1001D000AB120108AB120108AB120108AB12010807
:1001E000C5350108816B01085D9E0108DDFD010830
:1001F000ED4602080DC10208C1480408790F06083F
:100200008115060815870608FDEE0608C1F60608E2
:10021000F9F90608855F070825800708193E0808D0
:10022000E9B7080841C50808396B0A08DD700A08F3
:10023000A19B0B08D5FD0B08ED240C08153B0C0801
:10024000BD6A0C089D710C08000000000000000051
:1002500081F0004102E000BF83F0004330B54FEA77
:1002600041044FEA430594EA050F08BF90EA020FE4
:100270001FBF54EA000C55EA020C7FEA645C7FEA77
:10028000655C00F0E2804FEA5454D4EB5555B8BF9A
:100290006D420CDD2C4480EA020281EA030382EA0B
:1002A000000083EA010180EA020281EA0303362D9D
:1002B00088BF30BD11F0004F4FEA01314FF4801C70
:1002C0004CEA113102D0404261EB410113F0004F82
:1002D0004FEA03334CEA133302D0524263EB430339
:1002E00094EA050F00F0A780A4F10104D5F1200ED7
:1002F0000DDB02FA0EFC22FA05F2801841F1000132
:1003000003FA0EF2801843FA05F359410EE0A5F105
:1003100020050EF1200E012A03FA0EFC28BF4CF036
:10032000020C43FA05F3C01851EBE37101F00045EC
:1003300007D54FF0000EDCF1000C7EEB00006EEBF9
:100340000101B1F5801F1BD3B1F5001F0CD3490883
:100350005FEA30004FEA3C0C04F101044FEA4452DA
:1003600012F5800F80F09A80BCF1004F08BF5FEA61
:10037000500C50F1000041EB045141EA050130BD41
:100380005FEA4C0C404141EB0101013C28BFB1F553
:10039000801FE9D291F0000F04BF01460020B1FA9E
:1003A00081F308BF2033A3F10B03B3F120020CDA71
:1003B0000C3208DD02F1140CC2F10C0201FA0CF04F
:1003C00021FA02F10CE002F11402D8BFC2F1200CB4
:1003D00001FA02F120FA0CFCDCBF41EA0C0190406A
:1003E000E41AA2BF01EB0451294330BD6FEA0404B3
:1003F0001F3C1CDA0C340EDC04F11404C4F120029E
:1004000020FA04F001FA02F340EA030021FA04F3AF
:1004100045EA030130BDC4F10C04C4F1200220FA06
:1004200002F001FA04F340EA0300294630BD21FA44
:1004300004F0294630BD94F0000F83F4801306BF0A
:1004400081F480110134013D4EE77FEA645C18BFFE
:100450007FEA655C29D094EA050F08BF90EA020F95
:1004600005D054EA000C04BF1946104630BD91EA8D
:10047000030F1EBF0021002030BD5FEA545C05D190
:100480004000494128BF41F0004130BD14F58004CF
:100490003CBF01F5801130BD01F0004545F0FE4143
:1004A00041F470014FF0000030BD7FEA645C1ABF78
:1004B000194610467FEA655C1CBF0B46024650EAAF
:1004C000013406BF52EA033591EA030F41F40021DB
:1004D00030BD00BF90F0000F04BF0021704730B561
:1004E0004FF4806404F132044FF000054FF0000136
:1004F00050E700BF90F0000F04BF0021704730B5F7
:100500004FF4806404F1320410F0004548BF4042CB
:100510004FF000013EE700BF42004FEAE2014FEA20
:1005200031014FEA02701FBF12F07F4393F07F4FFB
:1005300081F06051704732F07F4208BF704793F0FE
:100540007F4F04BF41F40021704730B54FF4607411
:1005500001F0004521F000411CE700BF50EA010214
:1005600008BF704730B54FF000050AE050EA0102BD
:1005700008BF704730B511F0004502D5404261EB2D
:1005800041014FF4806404F132045FEA915C3FF46E
:10059000D8AE4FF003025FEADC0C18BF03325FEA0B
:1005A000DC0C18BF033202EBDC02C2F1200300FABC
:1005B00003FC20FA02F001FA03FE40EA0E0021FAE1
:1005C00002F11444BDE600BF70B54FF0FF0C4CF4CF
:1005D000E06C1CEA11541DBF1CEA135594EA0C0F81
:1005E00095EA0C0F00F0DEF82C4481EA030621EABC
:1005F0004C5123EA4C5350EA013518BF52EA0335F7
:1006000041F4801143F4801338D0A0FB02CE4FF0A8
:100610000005E1FB02E506F00042E0FB03E54FF0D8
:100620000006E1FB03569CF0000F18BF4EF0010ED0
:10063000A4F1FF04B6F5007F64F5407404D25FEACC
:100640004E0E6D4146EB060642EAC62141EA55517F
:100650004FEAC52040EA5E504FEACE2EB4F1FD0CC1
:1006600088BFBCF5E06F1ED8BEF1004F08BF5FEA3F
:10067000500E50F1000041EB045170BD06F00046F1
:1006800046EA010140EA020081EA0301B4EB5C049E
:10069000C2BFD4EB0C0541EA045170BD41F4801196
:1006A0004FF0000E013C00F3AB8014F1360FDEBFBB
:1006B000002001F0004170BDC4F10004203C35DA97
:1006C0000C341BDC04F11404C4F1200500FA05F31A
:1006D00020FA04F001FA05F240EA020001F00042BB
:1006E00021F0004110EBD37021FA04F642EB060131
:1006F0005EEA430E08BF20EAD37070BDC4F10C045B
:10070000C4F1200500FA04F320FA05F001FA04F21E
:1007100040EA020001F0004110EBD37041F100010A
:100720005EEA430E08BF20EAD37070BDC4F1200515
:1007300000FA05F24EEA020E20FA04F301FA05F27D
:1007400043EA020321FA04F001F0004121FA04F225
:1007500020EA020000EBD3705EEA430E08BF20EAF5
:10076000D37070BD94F0000F0FD101F0004640002F
:1007700041EB010111F4801F08BF013CF7D041EAB1
:10078000060195F0000F18BF704703F000465200B5
:1007900043EB030313F4801F08BF013DF7D043EA86
:1007A0000603704794EA0C0F0CEA135518BF95EA3C
:1007B0000C0F0CD050EA410618BF52EA4306D1D1C3
:1007C00081EA030101F000414FF0000070BD50EAE2
:1007D000410606BF1046194652EA430619D094EA6C
:1007E0000C0F02D150EA013613D195EA0C0F05D156
:1007F00052EA03361CBF104619460AD181EA0301AA
:1008000001F0004141F0FE4141F470014FF0000061
:1008100070BD41F0FE4141F4780170BD70B54FF0FC
:10082000FF0C4CF4E06C1CEA11541DBF1CEA13557C
:1008300094EA0C0F95EA0C0F00F0A7F8A4EB05045E
:1008400081EA030E52EA03354FEA013100F0888055
:100850004FEA03334FF0805545EA131343EA12631E
:100860004FEA022245EA111545EA10654FEA0026D3
:100870000EF000419D4208BF964244F1FD0404F58C
:10088000407402D25B084FEA3202B61A65EB0305E8
:100890005B084FEA32024FF480104FF4002CB6EBA5
:1008A000020E75EB030E22BFB61A754640EA0C0025
:1008B0005B084FEA3202B6EB020E75EB030E22BF65
:1008C000B61A754640EA5C005B084FEA3202B6EBA6
:1008D000020E75EB030E22BFB61A754640EA9C0065
:1008E0005B084FEA3202B6EB020E75EB030E22BF35
:1008F000B61A754640EADC0055EA060E18D04FEAF3
:10090000051545EA16754FEA06164FEAC30343EA92
:1009100052734FEAC2025FEA1C1CC0D111F4801F5F
:100920000BD141EA00014FF000004FF0004CB6E758
:1009300011F4801F04BF01430020B4F1FD0C88BFF7
:10094000BCF5E06F3FF6AFAEB5EB030C04BFB6EB02
:10095000020C5FEA500C50F1000041EB045170BDF5
:100960000EF0004E4EEA113114EB5C04C2BFD4EB22
:100970000C0541EA045170BD41F480114FF0000EA6
:10098000013C90E645EA060E8DE60CEA135594EA22
:100990000C0F08BF95EA0C0F3FF43BAF94EA0C0F25
:1009A0000AD150EA01347FF434AF95EA0C0F7FF49A
:1009B00025AF104619462CE795EA0C0F06D152EAEE
:1009C00003353FF4FDAE1046194622E750EA4106D2
:1009D00018BF52EA43067FF4C5AE50EA41047FF4E3
:1009E0000DAF52EA43057FF4EBAE12E74FF0FF3C48
:1009F00006E000BF4FF0010C02E000BF4FF0010C19
:100A00004DF804CD4FEA410C7FEA6C5C4FEA430C91
:100A100018BF7FEA6C5C1BD001B050EA410C0CBFE0
:100A200052EA430C91EA030F02BF90EA020F002042
:100A3000704710F1000F91EA030F58BF994208BFA9
:100A400090422CBFD8176FEAE37040F00100704766
:100A50004FEA410C7FEA6C5C02D150EA013C07D1BD
:100A60004FEA430C7FEA6C5CD6D152EA033CD3D008
:100A70005DF8040B704700BF8446104662468C4602
:100A80001946634600E000BF01B5FFF7B7FF002835
:100A900048BF10F1000F01BD4DF808EDFFF7F4FF5E
:100AA0000CBF012000205DF808FB00BF4DF808EDE9
:100AB000FFF7EAFF34BF012000205DF808FB00BF0C
:100AC0004DF808EDFFF7E0FF94BF012000205DF82E
:100AD00008FB00BF4DF808EDFFF7CEFF94BF0120E3
:100AE00000205DF808FB00BF4DF808EDFFF7C4FFDC
:100AF00034BF012000205DF808FB00BF4FEA410C25
:100B00007FEA6C5C02D150EA013C0AD14FEA430C07
:100B10007FEA6C5C02D152EA033C02D14FF0000044
:100B200070474FF0010070474FEA410212F5001282
:100B300015D211D56FF47873B3EB625212D94FEA24
:100B4000C12343F0004343EA505311F0004F23FA0E
:100B500002F018BF404270474FF00000704750EA63
:100B6000013005D111F0004008BF6FF00040704720
:100B70004FF00000704700BF4A0011D212F500127A
:100B800011D20DD56FF47873B3EB62520ED44FEAE5
:100B9000C12343F0004343EA505323FA02F0704765
:100BA0004FF00000704750EA013002D14FF0FF30A3
:100BB00070474FF0000070474FEA4102B2F1E04346
:100BC00024BFB3F5001CDCF1FE5C0DD901F0004C34
:100BD0004FEAC0024CEA5070B2F1004F40EB830084
:100BE00008BF20F00100704711F0804F21D113F1B0
:100BF0003872BCBF01F00040704741F480114FEAE9
:100C00005252C2F11802C2F1200C10FA0CF320FA71
:100C100002F018BF40F001004FEAC1234FEAD3238E
:100C200003FA0CFC40EA0C0023FA02F34FEA4303F8
:100C3000CCE77FEA625307D150EA01331EBF4FF081
:100C4000FE4040F44000704701F0004040F0FE409C
:100C500040F40000704700BF80F0004002E000BF99
:100C600081F0004142001FBF5FEA410392EA030F97
:100C70007FEA226C7FEA236C6AD04FEA1262D2EBE1
:100C80001363C1BFD218414048404140B8BF5B42E6
:100C9000192B88BF704710F0004F40F4000020F07F
:100CA0007F4018BF404211F0004F41F4000121F095
:100CB0007F4118BF494292EA030F3FD0A2F10102DF
:100CC00041FA03FC10EB0C00C3F1200301FA03F11D
:100CD00000F0004302D5494260EB4000B0F5000F40
:100CE00013D3B0F1807F06D340084FEA310102F1FF
:100CF0000102FE2A51D2B1F1004F40EBC25008BFB1
:100D000020F0010040EA03007047490040EB00007A
:100D1000013A28BFB0F5000FEDD2B0FA80FCACF17B
:100D2000080CB2EB0C0200FA0CF0AABF00EBC250A8
:100D300052421843BCBFD0401843704792F0000F96
:100D400081F4000106BF80F400000132013BB5E7E9
:100D50004FEA41037FEA226C18BF7FEA236C21D05F
:100D600092EA030F04D092F0000F08BF08467047C4
:100D700090EA010F1CBF0020704712F07F4F04D192
:100D8000400028BF40F00040704712F100723CBFA5
:100D900000F50000704700F0004343F0FE4040F4CF
:100DA000000070477FEA226216BF08467FEA23638D
:100DB0000146420206BF5FEA412390EA010F40F478
:100DC000800070474FF0000304E000BF10F00043C4
:100DD00048BF40425FEA000C08BF704743F09643AB
:100DE00001464FF000001CE050EA010208BF7047C6
:100DF0004FF000030AE000BF50EA010208BF70474D
:100E000011F0004302D5404261EB41015FEA010C61
:100E100002BF84460146002043F0B64308BFA3F159
:100E20008053A3F50003BCFA8CF2083AA3EBC2533B
:100E300010DB01FA02FC634400FA02FCC2F120025A
:100E4000BCF1004F20FA02F243EB020008BF20F091
:100E50000100704702F1200201FA02FCC2F12002F7
:100E600050EA4C0021FA02F243EB020008BF20EAEC
:100E7000DC7070477BB972B90029BEBF00204FF00B
:100E8000004106E008BF00281CBF6FF000414FF092
:100E9000FF3000F007BAADF1080C6DE904CE00296F
:100EA00009DB002B1ADB00F095F8DDF804E0DDE942
:100EB000022304B07047404261EB4101002B1BDB71
:100EC00000F088F8DDF804E0DDE9022304B04042D8
:100ED00061EB4101524263EB43037047524263EBC3
:100EE000430300F077F8DDF804E0DDE9022304B005
:100EF000404261EB41017047524263EB430300F013
:100F000069F8DDF804E0DDE9022304B0524263EB46
:100F10004303704753B94AB9002908BF00281CBFD2
:100F20004FF0FF314FF0FF3000F0BCB9ADF1080CCD
:100F30006DE904CE00F04EF8DDF804E0DDE90223AF
:100F400004B07047430803F05533C01A830803F018
:100F5000333300F03330184400EB101000F00F3042
:100F600000EB002000EB0040000E704707EE900AF7
:100F7000F5EEC07AF1EE10FA01D400F00BB8F1EE04
:100F8000677A08B517EE900A00F004F8404261EB6A
:100F9000410108BDD0B5FFF7BFFA0C4B0022064651
:100FA0000F46FFF711FBFFF7E7FD0446FFF792FA44
:100FB000074B0022FFF708FB02460B463046394636
:100FC000FFF74AF9FFF7D8FD2146D0BD0000F03DFC
:100FD0000000F0412DE9F047089D04468E46002BA5
:100FE0004DD18A42944669D9B2FA82F252B101FADD
:100FF00002F3C2F1200120FA01F10CFA02FC41EAED
:10100000030E94404FEA1C48210CBEFBF8F61FFA71
:101010008CF708FB16E341EA034306FB07F199420C
:101020000AD91CEB030306F1FF3080F01F819942BF
:1010300040F21C81023E63445B1AA4B2B3FBF8F099
:1010400008FB103344EA034400FB07F7A7420AD920
:101050001CEB040400F1FF3380F00A81A74240F248
:1010600007816444023840EA0640E41B00261DB1B3
:10107000D4400023C5E900433146BDE8F0878B42E8
:1010800009D9002D00F0EF800026C5E900013046A7
:101090003146BDE8F087B3FA83F6002E4AD18B4281
:1010A00002D3824200F2F980841A61EB030301202B
:1010B0009E46002DE0D0C5E9004EDDE702B9FFDE17
:1010C000B2FA82F2002A40F09280A1EB0C014FEAC2
:1010D0001C471FFA8CFE0126200CB1FBF7F307FB1F
:1010E000131140EA01410EFB03F0884208D91CEBC2
:1010F000010103F1FF3802D2884200F2CB8043465F
:10110000091AA4B2B1FBF7F007FB101144EA01443D
:101110000EFB00FEA64508D91CEB040400F1FF31CC
:1011200002D2A64500F2BB800846A4EB0E0440EABA
:1011300003409CE7C6F12007B34022FA07FC4CEAC3
:10114000030C20FA07F401FA06F31C43F9404FEAB6
:101150001C4900FA06F3B1FBF9F8200C1FFA8CFECB
:1011600009FB181140EA014108FB0EF0884202FA1F
:1011700006F20BD91CEB010108F1FF3A80F08880E0
:10118000884240F28580A8F102086144091AA4B29D
:10119000B1FBF9F009FB101144EA014100FB0EFE1E
:1011A0008E4508D91CEB010100F1FF346CD28E454D
:1011B0006AD90238614440EA0840A0FB0294A1EBDE
:1011C0000E01A142C846A64656D353D05DB1B3EB3B
:1011D000080261EB0E0101FA07F722FA06F3F1406B
:1011E0001F43C5E9007100263146BDE8F087C2F112
:1011F0002003D8400CFA02FC21FA03F3914001438A
:101200004FEA1C471FFA8CFEB3FBF7F007FB1036C2
:101210000B0C43EA064300FB0EF69E4204FA02F46E
:1012200008D91CEB030300F1FF382FD29E422DD9C1
:10123000023863449B1B89B2B3FBF7F607FB1633F6
:1012400041EA034106FB0EF38B4208D91CEB010176
:1012500006F1FF3816D28B4214D9023E6144C91AF6
:1012600046EA004638E72E46284605E70646E3E606
:101270001846F8E64B45A9D2B9EB020864EB0C0E10
:101280000138A3E74646EAE7204694E74046D1E71F
:10129000D0467BE7023B614432E7304609E76444CD
:1012A000023842E7704700BF02E000F000F8FEE7B6
:1012B00072B6374880F30888364880F30988364884
:1012C0003649086040F20000CCF200004EF634715E
:1012D000CEF200010860BFF34F8FBFF36F8F40F273
:1012E0000000C0F2F0004EF68851CEF20001086016
:1012F000BFF34F8FBFF36F8F4FF00000E1EE100A86
:101300004EF63C71CEF200010860062080F314888E
:10131000BFF36F8FBFF064FEBEF0CAFE4FF05530D2
:101320001F491B4A91423CBF41F8040BFAE71D4993
:10133000184A91423CBF41F8040BFAE71A491B4A8C
:101340001B4B9A423EBF51F8040B42F8040BF8E7DE
:1013500000201849184A91423CBF41F8040BFAE7B3
:10136000BFF042FEBEF0F8FE144C154DAC4203DA5D
:1013700054F8041B8847F9E702F096F8114C124D17
:10138000AC4203DA54F8041B8847F9E7BFF02ABEE1
:1013900000060020002200200000010808ED00E007
:1013A0000000002000060020D0C00F08002200200E
:1013B000502C0020502C0020605C0120E00101082E
:1013C0004802010848020108480201082DE9F04FCF
:1013D0002DED108AC1F80CD0C3689D46BDEC108A73
:1013E000BDE8F08F002383F311882846A047002032
:1013F000BEF0E4FBFEE7BEF041FA00DFFEE70000CE
:1014000001F0FF01102A2BDB10F0070F08D010F8B5
:10141000013B013A8B422DD010F0070F42B3F6D1B9
:10142000F0B441EA012141EA014122F007047FF0D2
:1014300000070023F0E80256083C85EA010586EA29
:10144000010685FA47F5A3FA87F586FA47F6A5FA65
:1014500087F68EB9EED1F0BC01F0FF0102F0070271
:1014600032B110F8013B013A83EA010313B1F8D11C
:101470000020704701387047002D06BF35460338FD
:10148000073815F0010F07D1013015F4807F02BF36
:10149000013015F4C03F0130F0BC0138704700BF87
:1014A00010F8012B11F8013B012A28BF9A42F7D00E
:1014B000D01A7047034613F8012B002AFBD1181AE3
:1014C0000138704738B50022002304460D46FFF767
:1014D000EDFA28B920462946BDE8384000F00AB8A0
:1014E000204605F1004100F005F8404261EB410162
:1014F00038BD00BFD0B50C4B002206460F46FFF7A3
:1015000063F8FFF739FB0446FEF7E4FF074B0022C0
:10151000FFF75AF802460B4630463946FEF79CFE66
:10152000FFF72AFB2146D0BD0000F03D0000F0414E
:10153000036800221B6818477FB5039140210546C8
:1015400083F058FE039A18B90124204604B070BDF8
:10155000134E039296F9B234002BF5D064F048FF95
:10156000437A039A53B964F043FF847A039A2CB9FF
:101570000C4B4021284683F045FEE6E7D6F8643E52
:10158000B6F9B414B3F906309942DDDD064B009389
:101590004021064B284683F035FE0024D5E700BFE6
:1015A000584C002044980D0863980D0851980D0878
:1015B0002DE9F0430D46B5B02021044683F01AFE14
:1015C000002800F0B6805C4E96F9B234ABB1D6F884
:1015D000642EB6F9B434B2F90A1003F10A0291424A
:1015E00003DD40F28D32934207DC544B2A46202122
:1015F000204683F007FE002098E096F9A134022BE4
:1016000005D14F4B2A462021204683F0FBFDB6F83A
:101610007434DFF86C81A3F57A739BB241F65832CB
:10162000934210D808F5804706F59C62D7F8A43E8F
:1016300092ED007AD3ED097AB4EEE77AF1EE10FA82
:1016400003DD404BD2E7404BD0E706F2E44292ED97
:10165000007AD3ED0B7AB4EEE77AF1EE10FAF0DC13
:10166000B6F9AE34002B01DC384BBFE70021602215
:1016700003A80DF108090291C3F07EFC34486422EE
:1016800049468AF0F7FA40B9324BCDF800902A4625
:101690002021204683F0B6FDADE764F0A9FE2021AD
:1016A00065F0AAFE08B92C4BA0E72C480FF06CFEA1
:1016B000012806D1D7F8B00E8AF0CCFF98B10128E6
:1016C00015D0002160221CA81B91C3F055FC2449B1
:1016D000D7F8AC0E64231BAA8AF08CF9E8B91BABCF
:1016E0000093204BD3E7204B0093204BCFE796F895
:1016F000783E83B11E48192150F042F958B108F5DF
:1017000000581B48D8F88C64192150F05FF98642C4
:10171000D7DD184BE8E7184BE6E71849D7F8A40ED1
:1017200064231BAA87F026F80028D8D035B0BDE87E
:10173000F0830120FAE700BF584C002070980D0894
:1017400083980D08BB980D08AB980D08D5980D0827
:101750004C8500205EF30D08EA980D08D48E002019
:1017600063990D0867990D082E990D0809990D08C0
:10177000883B00204D990D083E990D0879990D0878
:10178000582C002007B504488CF0E6FA00F0010060
:1017900003B05DF804FB00BFE07A00202DE9F043C0
:1017A000DFF844910446D9F874020368A5B01B69B8
:1017B0000D469847804615F0BFF800210746602285
:1017C0000CA80B91C3F0D8FB64230BAA4146384602
:1017D00014F0BAFB064648B93A4A0BAB29462046F4
:1017E00083F018FF304625B0BDE8F083A9F54E60C0
:1017F00070F090FDB8F1000F03D194F91E30012B69
:101800000AD1314812F086F880B9304A294620467C
:1018100083F000FF0026E5E710F0060FE2D0A9F5FF
:10182000405012F077F808B9294AEFE703A9384683
:1018300014F0BCF928B19DF80D305B0601D5254A9E
:10184000E4E7DFF8A880D8ED007AF5EEC07AF1EE93
:1018500010FA4FF00003C5DD089309930A930DF1C8
:10186000200907AB019305AA06AB04A9CDF80090A7
:10187000384614F07DFD48462FF0F8FFD8ED007A89
:10188000B4EEE70AF1EE10FA01DB134ABEE79DED74
:10189000057AF4EEC77AF1EE10FA01D80F4AB5E7EF
:1018A0009DED047AF4EEC77AF1EE10FA01D80C4AF5
:1018B000ACE79DED067AF4EEC77AF1EE10FA91D816
:1018C000084AA3E780990D08582C002089990D0833
:1018D000A0990D08C6990D08D4990D08E9990D082D
:1018E000FF990D08159A0D08585C0020285100201A
:1018F00008B5064B93F88D329B0704D5044A83F054
:1019000089FE002008BD0120FCE700BF585C0020D4
:101910002C9A0D0870B50C4C0546D4F87402036877
:101920005B690E46984710B10124204670BDA4F5AE
:10193000405012F001F804460028F5D1034A314620
:10194000284683F067FEF0E7585C00203C9A0D08BB
:101950002DE9F046464ED6F8983293F8CB509BB01E
:1019600081468A4665B9434B1B68986A03685B6B7E
:101970009847044640B9404A5146484683F04AFEDB
:1019800028461BB0BDE8F08664F032FD202165F0EA
:1019900033FD58B164F02CFD1F2165F02DFD88B397
:1019A000364A5146484683F035FE002496F86A329E
:1019B00003F01403142B05D1314A5146484683F0F5
:1019C00029FE00245146484684F0FEFC002188424E
:1019D0004FF0600202A808BF0C460191C3F0CCFA98
:1019E000D6F89802036801AA1B6864219847054647
:1019F00080B9244A01AB5146484683F00BFE2C4681
:101A00002546BDE764F0F4FCA52165F0F5FC00284F
:101A1000C6D1CBE7002CF3D0D9F808303BB9D9F8C0
:101A2000003051465B6B484698470446E8E751460C
:101A30004846FFF7BDFD514607464846FFF758FFA9
:101A40003840C4B251464846FFF776FD514604403F
:101A50004846FFF75FFF51460440484683F002FEC8
:101A600051460440484684F0C7FC0440C8E700BF24
:101A7000585C002060910020509A0D08679A0D086C
:101A8000819A0D08999A0D0808B5FFF761FF054A7C
:101A900092F8681260F3041182F86812024A907199
:101AA00008BD00BF585C00203D930020F7B50546F7
:101AB0000F4683F0DBFB044678B10221284683F011
:101AC00099FB064648B115488CF046F9C205C0F3AB
:101AD0000723C0F3002403D53446204603B0F0BDED
:101AE0009B07F9D50D488CF045F90D4B03F654636F
:101AF000D3ED007AF8EEE77A30EE670ADFED097A87
:101B0000B0EEC00AB4EEE70AF1EE10FAE4DD064BDF
:101B10003A460221284683F075FBDEE7E07A002092
:101B2000586C00200000C842A49A0D08F8B504467D
:101B30000F4683F04DFE10210546204683F05AFBE8
:101B400058B12046FFF71EFE064630B9044B3A4610
:101B50001021204683F056FB35462846F8BD00BFCD
:101B6000B89A0D0870B505460E4683F0EBFA0446A8
:101B700078B18021284683F03DFB50B1074B93F8A4
:101B8000353843B1064B32468021284683F03AFB74
:101B90000024204670BD0446FBE700BF585C0020CF
:101BA000CC9A0D0838B50D4D0446D5F8B00E8AF024
:101BB00051FD012810D0D5F8B00E8AF04BFD022857
:101BC00004D02046BDE8384083F0BEBA04480FF088
:101BD000DBFB0128F5D138BD0020FCE7586C002064
:101BE000D48E0020F0B5134C04F5005385B0D3F823
:101BF0005C2E0092D3F8602E0192D3F8642E0292EC
:101C0000D3F8683E03936A4606460F4684F08EFB7F
:101C100039460546304683F04FFB04F540542840D2
:101C200094F8683260F3C303C3F3C00084F86832E9
:101C300005B0F0BD582C00202DE9F8430646274892
:101C4000DFF8A890DFF8A8800F4670F063FB044629
:101C5000D9F8740203681B699847054630B914F037
:101C6000060F03D1D9F8A832022B09D139463046E4
:101C700083F0F4FB054618B9002488F807400AE011
:101C800039463046FFF78AFD04460028F4D02DB9C6
:101C9000012388F807302046BDE8F8830821304644
:101CA00083F0A8FA0028F3D00D4822F01DFB00288D
:101CB000EED00C4B93F81424B02101FB023203F553
:101CC0000053B2F81E22B3F9A2349A42E0DD064B6B
:101CD0003A460821304683F095FACDE7784F002048
:101CE000782D0020582C0020E09A0D08585C002028
:101CF0003D9300202DE9F3410E46054614F01CFEED
:101D0000804613F015FF044640B9464A0121284693
:101D100083F080FC204602B0BDE8F081424FD7F846
:101D20007402036831469B699847044658B9D7F84E
:101D3000740203685B6C98473C4A034601212846BD
:101D400083F068FCE6E7AB68002BE3D0102128465F
:101D500083F050FA20B3D8ED937A98ED920A20EEF2
:101D6000270AC0F011FEDFED327AA7F5805320EE8E
:101D7000270AB3F97434DFED2F7A20EE270A07EE35
:101D8000903AF8EEE77AB4EEE70AF1EE10FA07DDE2
:101D9000294B01221021284683F034FA0024B9E7A8
:101DA0004021284683F026FA38B3012E1ED0232E78
:101DB0001CD0042E1AD02148D0F8643EB3F9083064
:101DC00000EE103AA0F50050B8EEC00A00F09EFBFD
:101DD000B5EEC00AF1EE10FA0FDD194B00930122A7
:101DE000184B4021284683F00DFAD7E7D7F8740244
:101DF0000368DB6B98470028DDD0134B1B68D86A5B
:101E00000368DB6998470128014604D10F4A284638
:101E100083F000FCC2E73146284602B0BDE8F0413D
:101E200083F09EBFF09A0D08585C0020019B0D08BE
:101E3000E02E65420000C842159B0D08584C00205A
:101E400063980D081D9B0D0860910020299B0D08CB
:101E500070B505460E46FFF7A1FC084B0446D87145
:101E600031462846FFF756FD31460028284608BF70
:101E7000002484F037F9204070BD00BF3D9300205E
:101E80002DE9F0414E4F3B78002B40F096804D4CB1
:101E9000D4F8985295F8CB5001263E701DB13B7096
:101EA0002846BDE8F08184F04FFB054630B9464A2C
:101EB0003870137843F001031370F1E758F008FC11
:101EC000314657F0F1FBA4F5405006F061FA3F4B64
:101ED0001E710B264AF072FC013E4AF025FC16F0FA
:101EE000FF06F7D13A4800F037FF14F025FDD0F88F
:101EF0000022C4F8C02290F87C32DA074DD414F0E6
:101F000099F858F0E5FB3C2158F07AF90023C4F821
:101F1000803200212E482F4E00F0A4FF2C4811F0F3
:101F2000F9FC01462C488FF081FD2C4B1B68D86AC8
:101F3000036801211B689847D4F8980203689B6ADC
:101F400098470121D4F898028EF090FD58F0C0FB1C
:101F50008046D4F8740203681B68984796F83424C6
:101F60000146404657F07CFDA6F5005006F002FA07
:101F700054F0D4FA53F014FE00233B7095F09AFD10
:101F8000B4F86A3206F5005623F4087343F02003D0
:101F9000C6F8BC0EA4F86A3282E79B07B9D4314672
:101FA0000B4804F0E5FF0E488BF0E4FEDFED0D7A00
:101FB00020EE270A84EDA00AABE7002570E700BFFA
:101FC000502C0020585C00205C9300203D930020A2
:101FD000582C0020584C0020C4580020609100204C
:101FE000E07A00200AD7233C2DE9F043374DD5F89D
:101FF000983293F8CB3087B0002B64D062B10129BE
:1020000001D0232908D195F96832002B04DB002484
:10201000204607B0BDE8F08384F04CFB044600285E
:10202000F5D014F089FC07461AF0FCFD80463846CE
:1020300013F088FAD8B198F92430022B17D1002672
:102040004FF00009F1B203AA38460191CDF80C9087
:10205000CDF81090CDF8149013F012FE019918B13C
:1020600003AA40461AF0DCFA0136032EEAD11848DA
:10207000012106F073FD1648012106F045FD0021FF
:10208000D5F898028EF0F2FC124832F011F958F0AF
:102090001FFB002157F008FB0F4B1B68D86A036831
:1020A00000211B68984795F86A32D5F874120B48DE
:1020B0006FF3451385F86A320B1A594259413C3087
:1020C00093F0F0FBA4E70124A2E700BF585C0020D6
:1020D000582C00206C860020609100200888002089
:1020E00010B5064CD4F8740203685B6A984718B1BF
:1020F000D4F8983293F8CB0010BD00BF585C002094
:1021000030B52DED028B89B00C46B0EE408AFFF75A
:10211000E7FF0546002838D0B4EE488AF1EE10FA01
:102120007CBFDFED1C8ADFED1C7A226863689FEDBF
:102130001A0A68BFDFED198A029278BF68EE288A12
:1021400002A878BF68EEA78AD4ED027A0393F1EE75
:10215000677ACDED047A2EF08BFFB4EE488A002228
:102160000123F1EE10FACDE900238DED050ACDED46
:10217000060A9FED0A0A0A488DED071AF0EE680A72
:1021800068BF134605A90DF0DDF9284609B0BDEC7E
:10219000028B30BDE02E65420000C8420000000006
:1021A000788D002007B50191FFF79AFF30B10199B2
:1021B000044803B05DF804EB00F0F4BA03B05DF836
:1021C00004FB00BF582C0020014870F02FBA00BF5C
:1021D000784F002008B500F5405090F86832C3F3FE
:1021E00040128A420BD061F3451380F8683231B156
:1021F00058F06EFABDE808400F2158F001B808BD4C
:1022000070B500F540560546D6F8A8328B420C460C
:1022100011D0012910D0022915D051B958F058FA1F
:102220001B2157F0EDFF0D4A062105F541505BF0EB
:10223000F5FCC6F8A84270BD58F04AFA1A2157F0CA
:10224000DFFF074AF0E7012100F00CFE58F040FAEA
:102250001D2157F0D5FF034AE6E700BF949B0D0808
:10226000A99B0D08A49B0D0810B500F540520C4623
:1022700092F88D3203F00101A14209D064F300030A
:1022800082F88D32DB0704D405F072FC024B9C729D
:1022900010BD05F039FEF9E73D93002000F54050F0
:1022A00090F88D3261F3410380F88D32014B197340
:1022B000704700BF3D93002000F5405090F86A320F
:1022C00043F0040380F86A327047000010B50446FA
:1022D00054F024F904F54052436FD2F8982204F5E3
:1022E0008044D360D4F8A42E9366D4F8AC2EC2F800
:1022F000FC32D4F8A40E03685B6D9847D4F8A40EA2
:102300000368BDE810409B6D1847000070B52DEDC7
:10231000028B00F540550446D5F8983293F8CB303F
:10232000002B74D095F96832002B70DB00F5A043C8
:1023300093F83839002B6AD1D5F8740203685B69C9
:102340009847002863D1334BD3F8740203681B68A5
:1023500098470B285BD004F580469FED2F7AD6F87E
:10236000AC3ED3EDDB7AF0EEE77AF4EEC77AF1EE2D
:1023700010FA4CD5D5F8980244305AF063FE034663
:10238000DFED260A93ED000A9F20B7EE001A2BF02E
:10239000EFFBB5EEC00AF1EE10FA38DD04F59D4012
:1023A00008308BF0F3FCDFED1E7AB0EEC00AB4EE1D
:1023B000E70AF1EE10FA2AD504F58054D6F8A40EF7
:1023C000D4F8083607EE903A0368D3F89830B8EEA0
:1023D000E78A984738EE400ADFED127AB0EEC00A7D
:1023E000B4EEE70AF1EE10FA11D5D4F80C3640F24B
:1023F000E63203F2F313934209D8BDEC028BD5F811
:1024000098029FED090ABDE870408BF01FBFBDEC3C
:10241000028B70BD585C00200000003400000000FA
:10242000000070420000FA430AD7233C08B500F5CB
:102430004050D0F8980203681B699847F6EE007A7E
:1024400020EE270AB5EEC00AF1EE10FA48BF9FED64
:10245000010A08BD0000000038B52DED028B00F523
:1024600080450446D5F8A43EDFED110A93ED370A06
:1024700004F540547120B7EE001A2BF079FBD4F824
:102480009802D5F8AC5E03681B69B0EE408A9847A5
:1024900038EE400ABDEC028BDFED067A05F50575D6
:1024A000284620EE270ABDE838407BF015BF00BF64
:1024B0000000000000007A4400F5A050D0ED985ACA
:1024C000D2ED007AD0ED9B6A91ED006A26EEE77AB4
:1024D00067EEA57AA6EE257AE6EE267A81ED007AF9
:1024E000C2ED007A7047000000F50050B0F91C3DC5
:1024F00033B9B0F9AE040028B8BF404280B270478B
:1025000083EAE370A0EBE370F8E7000070B52DED0F
:10251000028B00F5405382B093F88D1211F0010642
:10252000044605D09FED2E0A02B0BDEC028B70BDB3
:102530008DED010A63F05CFF037F002BF2D0DFED2D
:10254000298ADFED270A9DED010AB0EE681A4E20B8
:102550002BF00EFB04F500554FF4C8723146B5F967
:10256000B604B0EE408A2BF041FBA5F8B604204635
:1025700010F054FFB5F9B63407EE900AB8EEE77ADA
:1025800007EE903AF8EEE77A77EE676AB4EEE68AFD
:10259000F1EE10FA0DD52046FFF7A6FF07EE900AE0
:1025A00038EE668AB8EEE70A20EE088A88EE260A38
:1025B000BAE777EE877AB4EEE78AF1EE10FAB1DD8A
:1025C000B5F9AE3400EE103A38EE678AB8EEC00ABC
:1025D00078EEE77A20EE088A88EE270AA4E700BFA3
:1025E0000000000000007A4400207047002070477F
:1025F0007047000000F513500430704700487047E2
:1026000014CC0D0800F54050D0F8740203681B6824
:1026100018470000034808603521117008221A602D
:10262000704700BFAC9F0D0800F54050D0F8740211
:1026300003681B6D1847000000F54050D0F8740285
:102640000368DB6C1847000000F5405300F5B34009
:10265000D3F8743258301B1A584258417047000062
:1026600010B500F540500C46D0F8740203681B6E9C
:10267000984707EE900A9FED057AF8EE677A0120F9
:1026800067EE877AC4ED007A10BD00BF0AD7233CFD
:1026900010B500F540500C46D0F874020368DB6DAD
:1026A000984707EE900A9FED057AF8EEE77A012049
:1026B00067EE877AC4ED007A10BD00BF0AD7233CCD
:1026C00010B500F540500C46D0F8740203685B6EFC
:1026D0009847DFED047A20EE270A012084ED000AF6
:1026E00010BD00BF0AD7233C69F012BA12F008B837
:1026F00065F068BF53F05CBE28F0C4BE57F056B911
:1027000018F02EB866F0DEBA63F0CCBA61F0D4BB34
:1027100010F04ABB10F076BF06F068BC11F0EEBFB7
:1027200005F078BA05F064B905F08AB805F064BF21
:102730006AF0A2BF0FF0C6BCFFF7E8BD10F072BC94
:1027400010F0BABE03F000BB10F0F8BB10F072BB83
:1027500063F09CBD4BF064BA23F074B805F084BEFE
:1027600002F076BD66F0BEBA10F0C2BE06F0F6BB4F
:1027700004F0EABB06F042BD05F0F4B806F040B93B
:1027800005F0C4BF10F09CBA06F0E2B8FFF79EBD9A
:1027900029F06ABA05F034BC0AF02EBA0AF018B96A
:1027A0000AF0ACB81FB500F540530446D3F87402E4
:1027B000039103685B6A984760B1DFED070A0399EC
:1027C000002304F5C2400093B0EE600A1A462030A0
:1027D0000CF00EFD04B010BD0000000010B52DED92
:1027E000028B00F540530446D3F8740203685B6A19
:1027F000B0EE408A984720B90024BDEC028B2046F9
:1028000010BD9FED080A04F5C24028EE000A2030F2
:102810000BF0B8FF04460028EED003480121FFF773
:10282000D9FCEAE70000C842582C00200A4A92F975
:102830006822002A0B4605DA00228A604A600A6094
:102840000120704700F58040D0F8A42E783207CAE6
:1028500083E80700F4E700BF585C002038B54D4B13
:10286000044640F8043B69F073FA04F1100017F0D5
:10287000FBFB04F1680053F029FB04F5907021F094
:1028800043FC04F58C6016F029F904F2845019F029
:1028900051FC04F6C80028F03BFC04F5666069F0C2
:1028A00035F804F573604EF091FF04F58F5056F043
:1028B0004BFE04F5975014306FF00EF804F5985065
:1028C000103066F09BF804F59A500C3081F0CCFE85
:1028D00004F59B50083053F0BBFE04F59C500C30BF
:1028E0006AF014FC04F5805300252B4A83F8B0539A
:1028F00004F59D53103304F59E50136049F088FD94
:1029000004F5A0502946103012F002FB04F5D35014
:1029100018307BF01FFF04F5FB501C307EF0C4FE26
:1029200004F50250143080F0F9FF04F503503830FC
:1029300081F02EFC04F50550103012F0EBF804F590
:102940000A5030307CF07EFC04F50C5013490830FE
:102950004DF058FD04F50C5020306FF07FFB04F56E
:102960000F501C3082F01CFA04F5005304F511508E
:1029700083F834540A4D0C3082F034FB2B6813B1C9
:10298000084895F065F8204607494DF03BFD2C605E
:10299000204638BD60970E08F09C0020782D0F0867
:1029A00020940020B89B0D0868960E0810B510F012
:1029B000A9FC63F01DFD0368BDE810405B68184783
:1029C000FFF7F4BF10B5044606F0B6F8204610F045
:1029D000CBFF204605F06EFF204605F0F7FF2046AE
:1029E00004F0FCF82046BDE8104004F063BA000093
:1029F000FFF7E8BF70B500F54B550435044628468F
:102A000017F00CFA1AF00EF990F9213093B390F800
:102A100040337BB304F5405304F28456D3F8980254
:102A200044305AF00FFB0346DFED130A93ED000A22
:102A30009F20B7EE001A2BF09BF894F9B835012BC4
:102A4000284608BF86ED0E0A002116F07BFFDFED59
:102A50000B7A04F2DC7494ED287A20EE270ADFED7D
:102A6000087AA7EE270A304684ED280ABDE87040B0
:102A700019F0E8BF70BD00BF00000000CDCCCC3D18
:102A80006666663FFFF7B6BF10B50121044610F039
:102A9000A7FF60B1114BD3F8740203689B6A984793
:102AA00028B9204602F0E2FA204602F0EFFA4FF48D
:102AB0000011204610F094FF18B12AF0EBFA28F02C
:102AC000F7F94FF48021204610F08AFF28B12AF050
:102AD000E1FABDE8104028F0EFB810BD585C0020C6
:102AE000FFF7D2BF70B500F580450446D5F8A40EB7
:102AF0009FED560A86B06C302EF0BAFA04F5A0505D
:102B000003A910308DED030ACDED040A8DED051AF1
:102B100012F0AAF80221204610F062FF70B10121E4
:102B2000204610F05DFF48B9494BD3F874020368A2
:102B30009B6A984710B9204602F098FA0121204676
:102B400010F04EFF48B9424BD3F8740203689B6AF9
:102B5000984710B9204602F099FA0121204610F05A
:102B60003FFF10B9204602F0E9FA04F54056D6F8C6
:102B7000980203685B6C98474021204610F030FFB4
:102B800060B104F58F50019056F0A4F804F580531D
:102B9000019893F910330BB156F0DEF94FF48061D0
:102BA000204610F01DFF18B104F58F5056F02CF997
:102BB0002021204610F014FF48B1D6F874020368B3
:102BC0001B69984718B3D5F8AC0E87F04FFE8021EB
:102BD000204610F005FF38B32AF05CFA28F090F890
:102BE0001021204610F0FCFE18B1D5F8A40E84F098
:102BF000E1FC4FF40041204610F0F2FE18B304F55A
:102C00009E40443006B0BDE8704066F09DB9204655
:102C10000DF0A8F90028D6D1D6F8740203685B69D4
:102C200098470028CFD0D2E74FF48021204610F0FB
:102C3000D7FE0028D0D14FF40021204610F0D0FE5E
:102C40000028C9D1CCE706B070BD00BFE02E6542B8
:102C5000585C0020FFF746BF10B50121044610F074
:102C6000BFFE10B1204602F069FA8021204610F024
:102C7000B7FE58B14FF48021204610F0B1FE28B9BC
:102C80002AF008FABDE8104028F016B810BD000080
:102C9000FFF7E2BF10B5044605F084FA204605F0C0
:102CA000D5F8204605F0C4FA204611F04DFD204627
:102CB000BDE8104003F06EBFFFF7ECBF70B54FF6F4
:102CC000FF71044610F08CFE04F5405528B1D5F88C
:102CD00068220721204602F061FAD5F8983293F86D
:102CE000CB306BB92046FFF7E7FAD5F8980204F528
:102CF0000053026893F80415166A93F8CA24B04783
:102D000065F08AF964F03CFE204611F00FFD95F85D
:102D100068320F4A04F58044DB43D4F8A45EC3F361
:102D2000C01353712B681E6F53F0F8FB53F060F81B
:102D30002846B047D4F8AC4E53F0F0FB04F50574C8
:102D400053F056F82046BDE870407BF02BB900BF29
:102D50003D930020FFF7B2BF70B500F5805606F531
:102D6000826300F54054D3F85022C4F8AC22D3F863
:102D70005C32C4F8B0320546D6F8100600F58C4037
:102D800050302AF0C9FED4F8AC32C4F8B832D4F8C6
:102D9000B032C4F8B402C4F8BC324FF6FF71284612
:102DA00010F01EFE38B1D6F8102628460921BDE8DD
:102DB000704002F0CBB970BD30B500F54053D3F888
:102DC000A842002C4CD093F86922D10748D56FF364
:102DD000000283F8692200F50052012CD2F85C1E33
:102DE000D2F8605EB1F908400BBFD3EDAC5AD3ED19
:102DF000AF5AD3EDAB7AD3EDAE7A07EE104AB5F900
:102E0000084006EE904A0CBFF8EEE66AF8EEE66A75
:102E1000B8EEC77A25EEE66A00F5A050A7EE276A5D
:102E200067EEA67AD0ED986AE7EE257A90ED9B7A68
:102E300027EE877AA6EE267ABDEEC77A17EE103A0D
:102E40000B8190ED987AD2F8603E67EE877A90ED2C
:102E50009B7AE6EE477AFDEEE77A17EE902A1A8122
:102E600030BD000038B505462DED028B00F540540D
:102E700071B1284610F0F6F8D4F8B4321B1A03F2F8
:102E8000F31340F2E63293420CD8BDEC028B38BD0E
:102E9000D4F8A832022BF8D110F0C8F8B0F57A7F38
:102EA000E7D2F2E7C4F8B40200F58C405030642356
:102EB00090FBF3F308EE103ADFED097AB8EEC88A1A
:102EC00028EE278AB0EE480ABFF0A4FB84EDAE0AD4
:102ED000B0EE480ABFF0F4FC84EDAF0AD5E700BFBE
:102EE00035FA8E3C00F5A0500121103013F09CBC47
:102EF000FFF7F8BF10B5044610F096FA10212046EF
:102F000010F06EFD70B1204601F0FEFF4FF400118D
:102F1000204610F065FD28B92AF0BCF8BDE8104045
:102F200027F0C6BF10BD0000FFF7E4BFF8B50446A8
:102F3000254606F097F8224B45F83C3B214BA4650B
:102F4000C4E91734204BC4E91934204BE36604F17B
:102F5000800018F02BFD04F19C0018F027FD04F10F
:102F6000B80018F023FD4FF6FF76194BC4F8CC30AB
:102F7000A4F8D06004F1D40018F018FD4FF0FF372A
:102F8000144B1549C4F8307128461D604DF03AFACB
:102F9000A4F87870A4F8946004F5A27018F006FD07
:102FA00004F5B07018F002FD04F5BE7018F0FEFCD8
:102FB000002384F89031C4F8B4312046F8BD00BF36
:102FC000E8F90D08992701089D270108A1270108A4
:102FD0000000FFFF0C93002090660E0810B5044619
:102FE00006F040F80A4B23600123A38704F1400058
:102FF00018F0DCFC04F1500018F0D8FC04F160007B
:1030000018F0D4FC04F1700018F0D0FC204610BD7C
:10301000BC020E082DE9F043044689B0FFF71EFC00
:10302000A94B236004F51350303004F5005502F02D
:10303000EBF904F512533833C5F8703E062385F8D2
:10304000743E4FF07C5805A904F5395704F53A5001
:10305000CDF814805AF0F2F807F1580093F0FAFB1B
:1030600004F59D460023083685F8B03E04F53B572D
:10307000192304A985F8BC3EC5F8B86E07F108000D
:10308000CDF810805AF0DAF807F1200093F0E2FB57
:103090004FF00108182304F53C5085F8043F04F56F
:1030A0003E5785F8F88EC5F8006F184465F0B8F8FB
:1030B000384682F053F806AE844BC5F8803F31465F
:1030C000381D8DF818804DF0D1FF384638304AF061
:1030D00065FD04F53F50383082F02AF87C4BC5F886
:1030E000F83F04F540507B4D0695314610305AF0BC
:1030F000A5F804F5405031461C3006955AF09EF86C
:1031000004F5405006953146283004F540555AF0F4
:1031100095F804F54159704B2B6409F1140093F0B4
:1031200099FB04F54358F83708F11C083846143762
:103130005EF08AFFB845F9D10723C5F800320023B5
:10314000A5F804324FF4CB7018F0ECFFC5F8FC0181
:1031500004F54850083093F07DFB04F549500C30DD
:1031600093F078FB5D4B1A680AB9C3F8009004F538
:10317000C6485B4B2B6408F1080804F54950C5F8B4
:103180007482383083F0B6FA564B07934FF07E576F
:10319000554BC5F8AC72C5F8B8720694009304F5A7
:1031A0004B5096E80C004FF40071043016F07CFA96
:1031B00004F56050383073F067F904F59C4003A9BA
:1031C000583003975AF078F804F59C4003A96C3006
:1031D00003975AF033F804F59C40783018F0E6FB7A
:1031E00004F5804303F688620026166056609660F8
:1031F00003F6946204F59D4016605660966004F5EF
:10320000A0521032C3F8A02E002283F8C12E4FF432
:103210000041443017F02AF804F59E40443065F030
:103220003BFD04F59F40483071F032F804F5A040B2
:1032300004F5A04504304EF04FF82C4B6B60284647
:103240002B4B2C491830186005F138094DF0DAF88D
:10325000FF2385F8483085F85030274948464DF01F
:10326000D1F8264B1F6817B1254894F0F1FBC3F83D
:10327000009004F5A04004F5B14909F174095830F3
:1032800054F0B6FA1F4948464DF0BCF805F6F40371
:1032900048465E601C494DF0B5F81C4B1C48186050
:1032A00004F5B24210323B464FF0140C9FB20CFBB7
:1032B00007010133097C0029F8D1164B1F80164BFA
:1032C0001F686FB31548D0E7E0A30D08409B0D08B9
:1032D000809B0D080000A040C0B90E086497002034
:1032E00060A40D0895270108D0A30D08909B0D0838
:1032F000F89C002014CC0E08042C0F08889D002098
:10330000CC9B0D08EC670F082C680F08DC9300209D
:1033100094E70D08DA93002098930020ED9B0D08A8
:1033200004F5B240042114301A605AF031FA04F561
:10333000B24003A94D4B03933C3059F07FFF04F595
:10334000B2405C3005F08EFE494BC5F85C3904F59F
:10335000B3401C3005F086FE04F5B749454BC5F86F
:103360009C3904F5B34009F130095830FFF7DEFD10
:10337000484605F077FE404BC5F8B03B09F13C00EC
:103380008FF07AFD3D4BC5F8EC3B04F5C04004F5E9
:10339000C0455C3005F066FE394BEB6504F5C14075
:1033A00085F898701C3005F05DFE364BC5F89C30F2
:1033B00004F5C140583005F055FE334BC5F8147183
:1033C00004F5C240C5F8D830203005F04BFE2F4B35
:1033D000C5F8203104F5C240C5F85C71643005F0D1
:1033E00041FE2B4BC5F8643104F5C3402C3005F089
:1033F00039FE284BC5F8AC3104F5C340683005F000
:1034000031FE254BC5F8E83104F5C440C5F86062CB
:10341000C5F864627C30FFF7E1FD404605F022FE0E
:103420001E4BC5F8083304F5C640443005F01AFEBB
:103430001B4BC5F8443304F5C740A5F8807314301E
:10344000FFF7CCFD174BC5F89433012385F81D34E5
:1034500005F2244504F5C8402E606E60AE60303041
:103460000AF04CFA204609B0BDE8F083CDCC4C3DC3
:10347000D8F50D0880F60D0890FA0D0824FB0D080C
:10348000E0FB0D0884FC0D08C8FE0D086CFF0D085C
:1034900000000E089C000E0840010E0820040E08D3
:1034A000C0050E0878030E0838B5054B1C68236864
:1034B0000A461D68034B01462046A847002038BD38
:1034C00060910020582C002038B5037904463BB9A0
:1034D00005682DB1284626F063FD284618F024FE25
:1034E000204638BD314B324A70B5036000F5A04329
:1034F00000F5BE45C3F8B02B2E4AC3F8EC2B0446AA
:1035000005F59070FFF7E0FF05F58C7004F5BD45FB
:10351000FFF7DAFF05F1E400FFF7D6FF05F1DC0065
:10352000FFF7D2FF04F54053234AD3F8FC011A6495
:1035300008B118F0FDFD214B236004F5005393F80A
:10354000EC2042B9D3F8E8502DB1284626F028FDEA
:10355000284618F0E9FD04F59A500C3081F098F8EF
:1035600004F59850103065F061FA04F6E46504F64D
:103570008466B54204D0183D284626F067F9F8E77E
:103580000F4BC4F8C83804F6282059F037FA04F66F
:10359000FC1059F033FA04F65C1059F02FFA04F5D8
:1035A000136059F02BFA204670BD00BFE0A30D0850
:1035B00090FA0D08507E0F08C0B90E0860970E08EB
:1035C000BC580E0810B593F085FD064C064B1860EC
:1035D0002046FFF71FFD2046044A0549BDE810407C
:1035E000BEF0F2BE582C00206091002068F100204F
:1035F000E53401080120704790F89C308B4286BF6B
:10360000283150F8210000207047000090F89C30CD
:103610008B4286BF283150F82100002070470000FF
:10362000FA207047014B93F87A047047584C0020F9
:10363000034BD3F8A802431E58425841704700BFBD
:10364000585C0020034BD3F8A802831E584258410F
:10365000704700BF585C0020034BD3F8980208B1B4
:103660008DF000BB01487047585C00204CA40D0849
:1036700038B5C36A374D43F4E052C262026B42F47C
:10368000E0520263426B42F4E0524263D5F8AC2E42
:103690000446E2B143F4F843C362D5F8AC0E86F0B9
:1036A000A5FC38B1236B43F480432363636B43F47D
:1036B00080436363D5F8AC0E86F0BAFD38B1236B56
:1036C00043F400532363636B43F400536363224B5F
:1036D0001D6845B1192128464EF052F918B1E36A28
:1036E00043F48073E3621D4B93F8783E6BB1236B18
:1036F00043F48073236345B1192128464EF078F9CD
:1037000018B1636B43F480736363154B93F8F0381F
:10371000013B012B0BD8D4E90B2343F48003236333
:10372000636B42F4800243F48003E2626363E36A02
:1037300043F08043E362236B43F080432363094BF0
:10374000D3F8983293F8C1301BB9636B43F08043D0
:10375000636338BD586C0020E8930020584C00206B
:10376000587C0020585C002013B54FF44470CDE91C
:10377000002118F0D1FC044628B1DDE9002161F0F8
:103780006FFB024B2360204602B010BDA4A60D08BB
:1037900000207047704700000320704708207047E2
:1037A000014B93F87C047047584C0020034B93F96D
:1037B000FB04003818BF0120704700BF584C0020A0
:1037C000014B93F97E047047584C0020704700006D
:1037D0007047000008B50C4BD3F8AC0E70B910233D
:1037E0000A4AD2F8982243F0400022B192F8CB2046
:1037F0000AB143F0C00040F0010008BD86F0F6FBBE
:103800000028ECD01823EBE7586C0020585C00200F
:1038100038B5C5780B46352D044628BF35253522E9
:1038200000211846C1F0A8FB2A4604F10C01BDE8AE
:103830003840C1F057BB00001FB5184C94F89E12D9
:1038400004F5A87011F050F978B194F89E1204F5BF
:10385000A87011F04BF940B194F89E1204F5A870CD
:1038600004B0BDE8104011F043B900230193029366
:10387000039313F061F801A912F03EFE20B101A8F4
:103880002DF0F4FF04B010BD22F01AF890F8F432D5
:10389000B02202FB030090ED3B0AF3E7584C0020F6
:1038A00008B50D4BD3F89802A8B1443059F0CAFBC3
:1038B000034693ED000ADFED090A9F20B7EE001AD8
:1038C0002AF056F9DFED067A20EE270ABDEEC00A8F
:1038D00010EE103A18B208BD585C0020000000003D
:1038E0000000C8422DE9F04FDFF8D880344F8DB08A
:1038F0000446042508F5005617F8019BB8F9D4349E
:1039000009F1FF3A43FA0AF3D90742D5207C5BF06C
:103910004FF98346207C5CF04FF800F121039B4572
:1039200005D2207C0DB0BDE8F04F5AF097BBBAF13C
:10393000030F2ED8DFE80AF00234393ED6F8A40E81
:1039400003689B68984700F194035A69D3F800A074
:10395000D3F804E0D8681969D3F818C008925A6AF5
:103960001B6ACDF82520CDF8293062222123CDE92C
:10397000003206900791207CCDF80CA0192303AAF1
:10398000C221CDF810E0CDF814C08DF824905BF082
:1039900079F9013D15F0FF05AED10DB0BDE8F08F0E
:1039A000D6F8A40E0368DB68CCE7D6F8A40E03684B
:1039B0001B69C7E7D6F8AC3E03F52A73C5E700BF1D
:1039C00078A70D08584C002013B50446074801910C
:1039D00008F046FF30B90199204602B0BDE810401A
:1039E0005CF02ABA042002B010BD00BF308600206F
:1039F000014808F011BD00BF3086002037B50446ED
:103A00000D460648019211468EF042FC019A294665
:103A1000204603B0BDE8304060F0EEB88059002089
:103A200010B588B004465DF005FC0C4BD3F8980245
:103A300038B90B4A0621204608B0BDE810405DF0B9
:103A4000E1BB69461E228DF011F9064A6B4606213C
:103A500020465DF0D7FB08B010BD00BF585C0020C9
:103A600098A40D085EF30D08034A92F8583E0133FE
:103A700082F8583E5CF0A2BC584C002007B50846BE
:103A8000019118F09BF838B10448019902F01EFF2B
:103A9000002003B05DF804FB0420FAE76C910020DD
:103AA000F7B58B8BCD2B06460C4617461DD1D1EDB5
:103AB000067AFCEEE77ACDED017A9DF80430022B10
:103AC00013D10E4D95F8BD1F05F6447065F01AF937
:103AD00058B195F8BD1F05F6447065F01BF920B983
:103AE00094ED020A064802F0D1FE3A4621463046DD
:103AF00003B0BDE8F0405CF0F3BC00BF586C0020A0
:103B00006C910020162A10B40C4605D0542A03D01C
:103B10005DF8044B5CF0ACB90323237001205DF821
:103B2000044B704710B5074B93F9582040F6CD343D
:103B300040F6CD13002A08BF1C465CF0F5FB20437D
:103B400010BD00BF587C002010B5044618F0ECFAF8
:103B5000204610BD10B50C4C94F96832002B0FDBD9
:103B6000D4F8740203681B6D984758B9D4F87402EE
:103B70000368DB6C984700280CBF0220032010BDAF
:103B80000120FCE70420FAE7585C002010B44C69DF
:103B9000012C05D101465DF8044B034803F030BA0F
:103BA0005DF8044B5CF024BC582C00202DE9F34157
:103BB000B1F90430002B06460C46154635DB4FF0B4
:103BC0000008CDE900281A4FB1F902209FED190A2B
:103BD000D7F85C1E4FF47A7360F0F6FA0123CDE952
:103BE00000539FED140AB4F90020D7F8601E4FF47B
:103BF0007A73304660F0E8FA9FED0F0AB4F90420BA
:103C0000D7F8641E43463046CDE9005860F0DCFA30
:103C1000CDE900589FED070AB4F90620D7F8681ED1
:103C20004FF47A73304660F0CFFA02B0BDE8F0810D
:103C3000584C00200000FA4400007A44044B1878E5
:103C400020B9044B93F86A02C0F38010704700BF9C
:103C5000E0920020585C00200B4B93F835287AB98D
:103C600093F88D2292060BD193F96822002A09DB82
:103C700093F8693213F0200F14BF0420012070471D
:103C80000520704703207047585C002008B5074B9B
:103C900093F9C834032B03D0BDE808405DF02ABB7C
:103CA000034A02215DF0AEFA042008BD584C002002
:103CB000B0A40D08094BD3F8FC24920701D45CF0A2
:103CC000CBB803F5005303F67C6393ED000ADFEDF8
:103CD000047AB8EEC00A20EE270A7047584C00203C
:103CE0000AD7233C10B594B0044603A817F05EFE33
:103CF0001C4BD3F87402036803A99B6D984778B3F3
:103D0000002103A817F01CFF50B3247C93F0D2FECF
:103D1000059BDDED047A0893069B09930023F8EEDA
:103D2000E77A9FED117A0B930C930D930E930F93FB
:103D30001093119312934FF6F853ADF84C300023C3
:103D4000962267EE877A8DF84E303323CDE9003224
:103D5000079007AA57212046CDED0A7A5AF092FF24
:103D600014B010BD585C00200AD7233C30B52DEDAF
:103D70000A8B774C0546D4F87402036899B05B6AE5
:103D8000984700285BD004F54054D4F85C31062BEA
:103D900000F2C980DFE803F00404045788AB530045
:103DA0006C489FED6D8A0BF0EBFB9FED6C0A016890
:103DB000426883680D930BA80B910C922DF058F973
:103DC000F0EE489AB0EE40CAF0EE60BAB0EE419A1A
:103DD000B0EE48AAF0EE488AF0EE48AAB0EE48BA33
:103DE00040F6F8542D7C93F065FE0023159316934E
:103DF00001238C228DF85E303323CDE900320B9005
:103E0000B1EE499AF1EE688AB1EE488A0BAA5521C3
:103E100028468DED0CCACDED0DBA8DED0E9A8DEDC7
:103E20000FBACDED10AACDED118A8DED12AACDED10
:103E3000139A8DED148AADF85C405AF023FF19B047
:103E4000BDEC0A8B30BD43480BF09AFB9FED430A53
:103E50000168426883680D930BA80B910C922DF0BA
:103E600007F93C48F0EE60BAB0EE419AB0EE40CAB5
:103E70000BF08AFB9FED390A2DF0FAF83548B0EEC9
:103E800040BAF0EE60AAF0EE418A0BF081FB9FEDA4
:103E9000330A2DF0EDF84FF44064B0EE40AAF0EE96
:103EA000609AB0EE418A9DE72A489FED2B9A0BF06D
:103EB0006BFB9FED2A0A2DF0DBF82648B0EE40BAE6
:103EC000F0EE60AAF0EE418A0BF062FB9FED230A50
:103ED0002DF0CEF8F0EE49BAB0EE40AAF0EE609ABE
:103EE000B0EE418AB0EE49CA40F607447AE7194875
:103EF000DFED198A0BF04CFB9FED180A2DF0B8F896
:103F0000F0EE68AAB0EE40AAF0EE609AB0EE418AF8
:103F1000B0EE68BAB0EE689AF0EE68BAB0EE68CA71
:103F200040F63F445EE79FED0C8A0024F0EE489A8D
:103F3000B0EE48AAF0EE488AF0EE48AAB0EE48BAD1
:103F4000B0EE489AF0EE48BAB0EE48CA4AE700BF71
:103F5000585C0020788D0020000000000AD7233C28
:103F60002DE9F0412DED068B3B4D95F86932990610
:103F70008CB004466AD505F580579FED380AD7F80E
:103F8000A40EDFED378A6C302DF072F88DED041A37
:103F900021EE281AD5F874628DED020ABDEEC11A21
:103FA000CDED030A11EE103A1DB2336894F810807B
:103FB000DB6D304660EE289A20EEA89A984707EE0F
:103FC000900AF8EEE77A304667EEA87AFDEEE77AD7
:103FD00017EE903A1CB233681B6E984707EE900AB2
:103FE000B8EE678AD7F8AC3EDFED1E7A93ED0FAAE4
:103FF000336828EE288A5B6EB4EEE78AF1EE10FA99
:1040000058BFB0EE678A30469847BCEEC88A002396
:10401000089318EE103AB7222AEE28AA20EE280AB2
:10402000ADF82C301A23CDE900323E2105AA4046D6
:10403000CDED059A8DED069A8DED07AA8DED090A55
:10404000ADF82850ADF82A405AF01CFE0CB0BDEC7B
:10405000068BBDE8F08100BF585C00209F0CB34583
:104060000AD7233C00FF7F472DE9F04F2DED028B4F
:104070001A4B047CD3F8A43E8DB0D3F88480D3F8D7
:104080008870D3F88C60D3F8905093ED258AD3F8DC
:1040900098B0D3F89CA0D3F8DC9093F00BFD0023EC
:1040A0008DF82C3016222523CDE90032029002AA89
:1040B000532120468DED078ACDF820B0CDF824A0FD
:1040C000CDF82890CDF80C800497059606955AF007
:1040D000D9FD0DB0BDEC028BBDE8F08F586C00200F
:1040E00070B58A7A4B7A43EA0223CA7A43EA0243DA
:1040F0009D2B06460C4621D1134D95F8BD1F05F6A4
:10410000447064F0FFFDC8B195F8BD1F05F644701A
:1041100064F00CFE022811D195F8BD1F05F644701D
:1041200064F0F8FD50B9D4ED057A9FED080A08480F
:10413000F8EEE77A27EE800A02F0A8FB2146304627
:10414000BDE870405CF03AB8586C00200AD7233CB8
:104150006C910020054BD3F898322BB193F8CA002C
:10416000002808BF0420704704207047585C0020D6
:1041700008B5034BD3F8740203681B68984708BD61
:10418000585C0020024B93F86902C0F3401070475E
:10419000585C002070B52C4E2DED028B0546D6F8EC
:1041A000740291ED018A036886B05B6A0C469847F9
:1041B00050B9BDEEC88A18EE103ADB0704D40220CD
:1041C00006B0BDEC028B70BDD4E904012AF0AAFD53
:1041D0000028F4D002A817F0E9FB02AA21462846DD
:1041E0005FF062FF0028EAD0184902A817F0F2FC3D
:1041F00003460028E3D1DFED160A00900246B0EE38
:10420000600A144802A90AF0F3FFD8B1D6F8740284
:1042100003685B6A9847044608B10020D0E70E485F
:104220000222042105F09AF860B1DFED090A09487D
:1042300000942346B0EE600A224602A90AF0D8FF95
:104240000028EAD10420BBE7585C0020D07A002087
:1042500000000000788D0020582C002008B591F84F
:104260002030032B1CD1D1ED027A9FED0E7A91ED17
:10427000060A0D4BF0EEE77AF4EEC77ADFED0B7A23
:10428000D3F87402F1EE10FA4CBF0121002120EEA8
:10429000270A0FF0F1FE002814BF0020042008BDFB
:1042A0000220FCE700000034585C00200000C842F7
:1042B00010B52DED028BD1ED007AF5EEC07AF1EE5E
:1042C00010FA82B00C4604DA042002B0BDEC028B76
:1042D00010BD9FED197AF4EEC77AF1EE10FAF3D81B
:1042E00091ED030A9FED158AF0EEC07AF4EEC87ADC
:1042F000F1EE10FA19D5D4ED037A1148D4ED010A84
:1043000094ED000AF4EEC87AD4ED027AFDEEE77A75
:10431000F1EE10FACDED017A9DF90410ACBF012247
:10432000002202F015FA0020CFE7F7EE000A29F08C
:104330001BFB0028C8D0DEE70000B44300000034B7
:104340006C91002091ED010AB5EEC00AF1EE10FA71
:1043500008B501DC042008BD9FED107A104BD1EDAB
:10436000007AD3F8740220EE070A9FED0E7A0368F4
:10437000F4EEC77AF1EE10FA05DD1B6F98470028BE
:10438000E8D00020E7E79FED087AF4EEC77AF1EE77
:1043900010FACCBFDB6E9B6EF0E700BF0000C84296
:1043A000585C00209A9939403333F33F08B5D1ED7A
:1043B000007A9FED157AF0EEE77AF4EEC77AF1EE27
:1043C00010FA1DD5D1ED017AF0EEE77AF4EEC77A56
:1043D000F1EE10FA14D50D480222032104F0BEFFBD
:1043E00080B10A480121FDF7F5FE094890F8183A16
:1043F000012B03D000F6142030F0B0F9002000E0CB
:10440000022008BD0420FCE700000034582C0020E6
:10441000587C002010B5D1ED007AFCEEE77A17EE5B
:10442000903A9CB2012C02D0022C06D04CB906481E
:10443000214669F0A3FA002010BD044802F0EEFF07
:10444000F9E70420F8E700BF707C0020582C00201A
:104450001FB5D1ED017A0B7CFCEEE77ACDED027A47
:10446000D1ED007A0093FCEEE77AD1ED030ACDEDB1
:10447000037A91ED020A9DF808309DF80C20014660
:1044800002480EF083FB05B05DF804FB582C0020B9
:1044900010B50A4C94F88D32DB070CD402220521AA
:1044A000A4F5405004F05AFF28B902221146A4F5A1
:1044B000405004F053FF002010BD00BF585C0020A6
:1044C00010B5D1ED007AFCEEE77A044617EE903A8B
:1044D00013F0FF030FD10F4BD3F874020368DB6FA7
:1044E000984708B1002010BD0B4A204606215CF019
:1044F00089FE0420F7E7012B0AD1064BD3F874029A
:104500000368D3F8803098470028EBD1034AECE7E2
:104510000220E8E7585C0020D4A40D08E4A40D08AC
:104520009FED0B7A01F10C03F1EC017AF4EE677A5E
:10453000F1EE10FA0AD6F0EEE77AF4EEC77AF1EE71
:1045400010FA03DC9942EFD1012070470020704738
:1045500000007A4430B52DED028B8DB00023054666
:1045600003930493059312F0E7F903A911F0C4FF34
:1045700058B312F0E1F900F55A7393E8070006AC5E
:1045800084E80700DDED060A9DED070A2D7CF1EEBB
:10459000600AB1EE400ABEF05FFA2046B0EE408AF3
:1045A0002DF064F9DFED0B7A089B0B93012228EEC6
:1045B000278A0C23CDE90032A82109AA28468DEDCF
:1045C000098A8DED0A0A5AF05DFB0DB0BDEC028B35
:1045D00030BD00BFE02E6542272938B5054613D00F
:1045E00008D81B290ED0242926D02846BDE83840FB
:1045F0005FF046BF282914D0402903D0A1F142031F
:10460000012BF2D8012405E0122159F039FD0446AE
:1046100010B90024204638BD297C0C4852F01EFBFE
:10462000F8E7162159F02CFD04460028F1D0297C2A
:10463000064852F0EDFBEDE70C2159F021FD044650
:104640000028E6D02846FFF785FFE3E7B07C00208E
:1046500038B5194C94F88D32DB070D460AD4D4F8DE
:10466000983293F8CB303BB901221146A4F1800077
:10467000FDF706FC002038BD94F96832002B4FF09E
:10468000020212DA0521A4F5405004F067FE00286A
:10469000F0D095ED000ADFED097AD4F8740220EE2F
:1046A000270A01210FF0E8FCE4E70921A4F54050B6
:1046B00004F054FEDEE700BF585C00200000C84252
:1046C00010B51B4C94F88D32DB070ED4D4F8983219
:1046D00093F8CB304BB194F96832002B07DA012202
:1046E0000821A4F18000FDF77FFC002010BDD1ED72
:1046F000007A9FED107AF0EEE77AF4EEC77AF1EEE9
:1047000010FA05D5022211460B4804F027FEECE70B
:10471000D4F8740203681B6898470428E5D0D4F8DD
:10472000740203681B6898471428EBD1DDE700BFCB
:10473000585C002000000034582C002073B58B8B8F
:10474000C12B05460C4644D8BB2B0DD8202B63D07B
:104750002ED8113B99B2052918D92146284602B016
:10476000BDE8704060F080BFBC3B052BF5D801A1CF
:1047700051F823F0B3480108BD4801085B47010820
:104780005B4701084B48010857480108052BE4D84E
:1047900001A151F823F000BF994801085B470108C7
:1047A0005B470108AD480108BF4701086D48010893
:1047B000732B2CD006D8542B58D0552BCDD1022298
:1047C00009216BE0B22BC8D102B0BDE87040FFF701
:1047D000B9BD4AF21146B34254D00BD8D12B40D0C8
:1047E000B3F5967F53D0D02BB7D102B0BDE870405F
:1047F000FFF710BE4AF21246B3423ED04AF21346C9
:10480000B342AAD102B0BDE87040FFF759BF02B071
:10481000BDE87040FFF74CBDD1ED007AF5EEC07AEF
:10482000F1EE10FA4FDD9FED297AF4EEC77AF1EE42
:1048300010FA48D8FCEEE77A254ACDED017A9DF8CA
:104840000430A2F82A3D00202EE0214602B0BDE847
:104850007040FFF79FBC214602B0BDE87040FFF7F3
:104860002FBE02B0BDE87040FFF7F2BD21462846DA
:1048700002B0BDE87040FFF7F1BC02B0BDE8704087
:10488000FFF7E6BE02B0BDE87040FFF701BE02B020
:10489000BDE87040FFF78ABD022205210D4804F0F3
:1048A0005DFD0028CFD1042002B070BD0222062198
:1048B000F4E70221084806F0F7F9F2E7022106487A
:1048C00006F0BCF9EDE70220EEE700BF00007F43F1
:1048D000584C0020582C00203086002008B591ED5F
:1048E000007AF6EE007AB4EEE77AF1EE10FA06DD21
:1048F000044801220521FDF777FB002008BD0420B4
:10490000FCE700BFD85B002030B52DED028BCD78E1
:1049100093B0272D28BF27250C462722002108A861
:10492000C0F02AFB2A4604F10C0108A8C0F0DAFA0C
:10493000424BD3F8740203685B6A9847002841D061
:104940009DF8465068063DD400244FF07E5329065A
:10495000049307940694059427D504A82BF032FEFF
:10496000EA0701940294039405F006032ED4002B69
:104970002ED10D9B01930E9B02930F9B0393304806
:104980000AF0E4F99DED100A044630B340F2ED4020
:10499000B7EE001AFFEE000A29F0EAF8284823468D
:1049A00001AA04A90AF0DAF90CE0099B04930A9B16
:1049B00005930B9B069304A80C9B07932BF008FE12
:1049C0000028CDD113B0BDEC028B30BD062BD6D064
:1049D00001211B480AF056F9F4E7DFED1A0A4FF4FB
:1049E0009E60B7EE001A29F0C3F8F6EE000AB0EEAA
:1049F000408A28F0B9FFE8B9B6EE000A124BB4EECF
:104A0000C08AF1EE10FAD3F8B03E08DD38EE400A65
:104A100030EE008A93ED070A28EE000ABEE730EE7A
:104A2000480AD3ED087A30EE000AF0EEE77A27EE76
:104A3000C00AB3E79FED030AB0E700BF585C00204F
:104A4000788D002000000000586C00202DE9F04314
:104A50009DB0814608460EA9FEF7DAFE844BD3F8D6
:104A6000740203685B6A984750B19DF86C30012B63
:104A700009D0DA1F022A06D97E4801210AF002F97C
:104A80001DB0BDE8F083BDF86840A20504F007063C
:104A900004F0380704F4E07501D5002DF0D04FF094
:104AA0000008CDF81480CDF81880CDF81C803EBBEE
:104AB0009FED716A9DED107ADDED117ADDED0F6AE3
:104AC00027EE067A67EEC67A66EE866A083B012B09
:104AD000CDED056A8DED067ACDED077A04D86748ED
:104AE00006AA05A9FDF7E8FC9DF86C30073B022BF0
:104AF00006D8634889F03AF9014605A82CF0D8FA9F
:104B0000CDF82080CDF82480CDF82880F7B9DDEDF0
:104B1000147A129B0893F1EE677A139B099308A904
:104B20004846CDED0A7AFFF7FBFC0028A4D09FEDA4
:104B3000520A08A82CF0F0FA9DF86C30083B012BC3
:104B400004D84E4809AA08A9FDF7B6FCCDF82C8078
:104B5000CDF83080CDF83480EDB99FED476A9DEDFA
:104B6000167ADDED177ADDED156A9DF86C3027EECB
:104B7000067A67EEC67A66EE866A083B012BCDEDB3
:104B80000B6A8DED0C7ACDED0D7A04D83B480CAA5A
:104B90000BA9FDF791FC14F4806233D1DFED397A73
:104BA0009DED180A9DF86C1020EE270ADFED327A91
:104BB0000839012920EE270A8CBF0021012114F4B5
:104BC000006305BFDFED2F7ADDED190ADFED2E0A58
:104BD00060EEA70A04BFDFED287A60EEA70AAEB93F
:104BE000002F35D1B3FA83F3B2FA82F25B0952098E
:104BF0000291019300920BAB08AA05A91D480AF087
:104C0000AFF93DE79FED200A0021D8E77FB9B3FA5D
:104C100083F35B0901200093B2FA82F3CDE901101E
:104C20005B0914480BAA08A90AF032FC28E7002DFA
:104C30007FF422AF0120B3FA83F3B2FA82F2CDE916
:104C400000105B090B4852090BA90AF0C9FB17E7D2
:104C5000002D3FF411AFB3FA83F3B2FA82F2CDE93B
:104C600000165B09520905A902480AF0FBF907E79B
:104C7000585C0020788D00200000C842582C00208D
:104C8000E07A0020E02E6542000000002DE9F047A8
:104C9000A2B08046084614A9FEF7BAFD7E4BD3F8B1
:104CA000740203685B6A9847C0B1BDF88040A305F1
:104CB00004F0070904F4E07700D57FB10CAE30466C
:104CC00016F074FEB9F1000F29D1DDE915012AF0C3
:104CD00029F830B97148012109F0D4FF22B0BDE8AC
:104CE000F0879DF8841009AA40465FF0C7F90028B4
:104CF000F0D0DDED177A9FED6A7A099B009367EE9D
:104D0000877A10ADFDEEE77ADDE9151217EE903ADD
:104D1000284616F06BFE95E80F0086E80F00002588
:104D200014F0380A06950795089514D1DDED1A7A26
:104D3000189B0693F1EE677A199B079306A94046E4
:104D4000CDED087AFFF7ECFB0028C3D09FED540AA5
:104D500006A82CF0E1F909950A950B959FB99FEDEE
:104D6000506A9DED1C7ADDED1D7ADDED1B6A27EEA4
:104D7000067A67EEC67A66EE866A8DED0A7ACDED22
:104D8000096ACDED0B7A14F4806805BFDFED457A32
:104D90009DED1E0A9FED440A20EE270A04BFDFEDB9
:104DA000407A20EE270A14F4006405BFDFED3D7A57
:104DB000DDED1F0ADFED3C0A60EEA70A04BFDFED60
:104DC000387A60EEA70AB9F1000F31D1BAF1000FBD
:104DD00052D13046CDED050A8DED040A16F016FECF
:104DE00003289DED040ADDED050A3FF473AF10A919
:104DF0003046CDED050A8DED040A109511951295FA
:104E000016F096FF00283FF465AFB4FA84F4640905
:104E1000B8FA88F3DDED050A9DED040ACDF804A08B
:104E200000945B0906AA10A91C480AF009F955E785
:104E3000BAF1000F0FD10123B4FA84F4CDE901A334
:104E40006409B8FA88F3154800945B0909AA06A911
:104E50000AF01EFB42E7002F7FF43CAF0123CDE9AF
:104E60000073B8FA88F2B4FA84F30C485B0952096B
:104E700009A90AF0B5FA31E7002F3FF42BAFB4FAD5
:104E800084F3B8FA88F2CDF800905B0952093146F4
:104E900002480AF0ADF921E7585C0020788D002027
:104EA0000000C842E02E65420000000030B48D7A58
:104EB0004B7A43EA0523CD7A43EA0543562B044651
:104EC0000A461BD008D8522B12D0542B13D02046A0
:104ED000114630BC5FF0A2BD03F18073863B23F026
:104EE0007F43012BF3D8017C064830BC52F058B800
:104EF00030BCFFF709BD30BCFFF7A8BD30BCFFF7E1
:104F0000C5BE00BFB07C00202DE9F0412DED028B25
:104F1000044690B000F5A0400023012269465830B5
:104F2000009352F0B3FD08B94D4B009304F5405681
:104F3000DFED4C8AD6F8740203685B69984704F584
:104F40008048002840F08780D8F8AC3ED3EDDE7A68
:104F500093EDD88AFDEEE77A28EE288A17EE903A8C
:104F60001DB204F53C57083701A938460EF0C6FBC0
:104F700018B955F0ADFB3A4B01933722002102A836
:104F8000BFF0FAFFA3238DF8083095238DF8093080
:104F900092F098FDD8F8A43ECDF80B00D6F8980210
:104FA000D3F8DC20D3F8E030CDF80F104430CDF842
:104FB0001320CDF8173058F045F80346DFED2A0AE4
:104FC00093ED000AB7EE001A9F2028F0D1FD10EEF5
:104FD000103AD6F89802CDF81B3003681B69984741
:104FE00010EE103A04F59D46CDF81F30083618EE45
:104FF000103A3046CDF8233088F0BCFE20EE280A67
:10500000384610EE103ACDF82730D8F8543ECDF897
:105010002B30019BCDF82F300EF092FB10EE103AA2
:105020003046CDF83330009BCDF83730ADF83B50EB
:1050300088F0ACFEBDEEC00A372210EE103A02A98D
:1050400004F58F50ADF83D3054F04AFB10B0BDEC84
:10505000028BBDE8F0819FED048A002581E700BF47
:105060002292CA7F0AD7233C0000000010B500F549
:105070008044D4F8A40E82F033F9D4F8AC1ED4F8EE
:10508000A40EBDE8104082F091B9000070B54FF455
:10509000805104460EF0A4FC00284ED004F5804652
:1050A00004F58F55D6F8A40E03689B6898476921CC
:1050B00000F19402284654F09FF9D6F8A40E036834
:1050C000DB6898476A2100F19402284654F094F96D
:1050D000D6F8A40E03681B6998476B2100F194026F
:1050E000284654F089F9D6F8AC2E6C21284602F5F2
:1050F0002A7254F081F9202120460EF071FCE0B1B3
:1051000004F54053D3F8740203681B69984778B1DB
:10511000D6F8AC2E284690326E2154F06DF9D6F8B0
:10512000AC2E2846BC32BDE870406F2154F064B903
:1051300020460AF017FF0028EAD170BD08B511F02B
:10514000FBFBBDE8084011F089B900007FB50E46B1
:105150004FF6FF71044615460EF042FCE0B11022F6
:1051600000216846BFF008FFA3238DF80030952387
:105170008DF8013003238DF8023092F0A3FC102249
:10518000CDF80300CDF8071004F58F5069468DF86F
:105190000B60039554F024FB04B070BD7FB50E4640
:1051A0004FF6FF71044615460EF01AFCE0B11022CE
:1051B00000216846BFF0E0FEA3238DF80030952360
:1051C0008DF8013004238DF8023092F07BFC102220
:1051D000CDF80300CDF8071004F58F5069468DF81F
:1051E0000B60039554F0FCFA04B070BD30B52DEDA2
:1051F000048B87B004460D46182200216846B0EEA5
:10520000409AF0EE608AB0EE418ABFF0B5FEA3236B
:105210008DF8003095238DF8013006238DF802308B
:1052200092F050FC1822CDF80300CDF8071004F5D9
:105230008F5069468DF80B508DED039ACDED048AA1
:105240008DED058A54F04CFA07B0BDEC048B30BDEF
:1052500010B54FF4801104460EF0C2FB30B104F5D6
:10526000A0501030BDE810400FF0D8BD10BD0000B8
:105270002DE9F0438FB014460546894631220021BE
:1052800001A8DDE916769846BFF076FEA3238DF8D7
:10529000043095238DF8053008238DF8063092F000
:1052A00011FC2368049363680593A36806933B6825
:1052B000CDF81D307B68CDF82130BB68CDF82530A6
:1052C0003368CDF829307368CDF80700CDF80B109E
:1052D000CDF82D303122B3688DF80F9001A905F576
:1052E0008F508DF81C80CDF8313054F0F9F90FB0A3
:1052F000BDE8F08370B52DED068B8CB014460546E5
:105300000E462C22002101A8B0EE409AF0EE608AF1
:10531000B0EE418AB0EE61AAF0EE429ABFF02CFEE8
:10532000A3238DF8043095238DF805300B238DF8D9
:10533000063092F0C7FBDFED1A7A94ED007ACDF8D3
:10534000070027EE277A29EE279A8DED077A94ED4C
:10535000017ACDF80B1027EE277A68EEA78A8DED3B
:10536000087A94ED027A8DF80F6028EE278A67EEAE
:10537000277A2C2201A905F58F508DED049ACDEDE9
:10538000058A8DED068ACDED097A8DED0AAACDED5F
:105390000B9A54F0A5F90CB0BDEC068B70BD00BFA4
:1053A000E02E6542A020704730B5154B89B0044609
:1053B0006946D3F8980204F58F551E228BF056FCEF
:1053C0006A461049284654F027FB04F54053D3F8A9
:1053D000740203681B68984704F50053014693F86C
:1053E0003424284654F03CFB04F5A050103011F052
:1053F00009FD04F590701FF0CDFA09B030BD00BF73
:10540000585C00205EF30D08274B70B543600446DE
:10541000183060F06DFE254E254BA361682560199C
:1054200061F01CF866513035B5F55A7FF7D1214D42
:1054300004F55A7062F0C8FC002104F27C708CF014
:1054400029F8C4F8305804F63800A5F644058CF065
:10545000F7FC9FED191ADFED190A9FED190AC4F840
:10546000C85804F6DC0082F095F89FED131A9FED02
:10547000150AF0EE410A04F6F40082F08BF89FED75
:105480000E1A9FED100AF0EE410A04F60C1082F09D
:1054900081F820460C494AF0B5FF20460B494AF0F6
:1054A000B1FF204670BD00BFB83A0020D0F10D0812
:1054B000E4F10D0888900020000000009A99993EC0
:1054C0000000B44300804A43B4E40D0814E70D081B
:1054D00070B5514D5149FAB0D022064646A8BFF0EA
:1054E00001FD0FCD0EAC0FC40FCD0FC40FCD0FC4F7
:1054F00095E80F0084E80F00002446AB181900213E
:10550000B7EE000A10344AF0B3FAD02CF5D1444B70
:105510000FCB02AC84E80F0001A920464AF05CFAE8
:1055200090B19DF90430DFED3F6AE06807EE103A74
:10553000B8EEC77AF0EE007AE7EE267AB7EE000A08
:1055400080EE270A4BF006FB00240EAB1819002151
:105550001034B7EE000A4AF08BFA402CF5D1324CE9
:1055600032480F214BF034FB0FCC1EAD0FC50FCCD2
:105570000FC50FCC0FC594E80F0085E80F0000227F
:1055800004211EA84AF020FB96F9DC69D6B9103434
:105590000FCC2EAD0FC50FCC0FC50FCC0FC594E8A7
:1055A0000F0085E80F00324604212EA84AF00CFBBC
:1055B0009FED1F0A1F484BF0CDFA1F48B7EE000AB7
:1055C0004BF0C8FA1D4C9FED1E0A0FCC06AD0FC55F
:1055D00094E80F0085E80F00002106A84AF048FA79
:1055E0009FED170A002128464AF042FA04F1100103
:1055F00060222EA8BFF076FC00242EAB18190021E3
:10560000B7EE000A10344AF033FA602CF5D162F09C
:1056100041F97AB070BD00BFCC920D08FC910D0825
:105620000C930D08CDCCCC3D1C930D0800EF0D085C
:105630000000000084E30D0893E30D089C930D081F
:10564000000034422DE9F04790B00DF106011D2015
:1056500062F0F0F9002800F09E809DF80630614A63
:105660000133DBB211210BA88DF8063091F082FADC
:1056700000220DF107010BA849F034FF9DF8063018
:10568000594A112105460BA891F074FA00220DF138
:1056900007010BA849F026FF9DF80630534A112157
:1056A00006460BA891F066FA00220DF107010BA83F
:1056B00049F018FF9DF806304D4A03F03F031121D1
:1056C00007460BA891F056FA00220DF107010BA82E
:1056D00049F008FF8046002D5DD0002E5BD0002FE2
:1056E00059D0002857D028464AF014F9002852D142
:1056F00030464AF00FF900284DD138464AF00AF9F1
:10570000002848D140464AF005F9002843D1394CD9
:1057100094E80F000DF10C0C10348CE80F0094E8A5
:105720000F000DF11C0989E80F0002A960464AF03C
:1057300053F998B3BDF8084002A948464AF04CF91D
:1057400000284AD0BDF8083054BB23B340F2E244ED
:105750009C420FFA84FA0FFA83F927D80DF10A0157
:105760003046ADF80A904BF001FD0DF10A012846D4
:10577000ADF80AA04BF0FAFC0DF10A013846ADF87D
:105780000AA04BF0F3FC00230DF10A014046ADF8EE
:105790000A304BF005FD10B0BDE8F0870024CBE7E0
:1057A00040F2D662002B08BF1346D1E70DF10A0183
:1057B0003046ADF80AA04BF0D9FC0DF10A0128469D
:1057C000ADF80A904BF0D2FC0DF10A013846ADF865
:1057D0000A904BF0CBFC0123D6E7002CDBD040F243
:1057E000D663B5E7A4E30D08B0E30D08BCE30D08EC
:1057F000C9E30D081C940D0837B500F51151782246
:105800003831044652F026FB00220C2126484AF08B
:10581000DBF92046FFF716FF04F512500022B7EE21
:10582000000A02210C304AF057FA012504F50C5108
:105830001E4A00950023203145204AF0C9F91C4A30
:105840001368D90709D41B49156004F50A5330338E
:105850000B6004F597531433CB6004F513501549CE
:105860000222303001254AF005FA134A0095002340
:1058700004F58F51FD204AF0ABF9104B1A68D2079E
:1058800005D40F4A1D6004F59B54083414600C487D
:1058900001214AF00BFA4AF0BBFF0A4A138843F091
:1058A0000103138003B030BDF4E30D086C260F082C
:1058B0006491002000220020809E0E086891002044
:1058C00018220020CC9300202DE9F04F2DED028B03
:1058D00000F50050D1B090F90435062B40F0BA80A5
:1058E0009549502228A8BFF0FDFA28AD002428468B
:1058F0000021B7EE000A01344AF0BAF8052C05F190
:105900001005F4D105A928A84AF066F806A9804632
:105910002CA84AF061F807A9074630A84AF05CF8BD
:1059200008A9064634A84AF057F8844B05460FCB21
:1059300018AC84E80F0003A920464AF04DF800286F
:1059400070D00021B7EE000A20464AF091F87C4959
:105950009FED7C8A802228A8BFF0C4FA28AC0025DD
:1059600020460021B0EE480A01354AF081F8082DA2
:1059700004F11004F4D1744D0FCD08AC0FC40FCD59
:105980000FC40FCD0FC495E80F00002584E80F0069
:1059900008AC20460021B7EE000A01354AF068F84D
:1059A000042D04F11004F4D16848002207A949F03D
:1059B00099FDB8B1B0F90030642B13DD07EE903AD1
:1059C000B8EEE70ADFED5F7A604820EE270ABCEE0A
:1059D000C00A10EE103A9BB200EE103AB8EE400A40
:1059E0004BF034F95A4D9FED578A0FCD18AC0FC4C8
:1059F0000FCD0FC40FCD0FC495E80F0018AD84E88C
:105A00000F00002428460021B0EE480A01344AF075
:105A10002FF8042C05F11005F4D151B0BDEC028B28
:105A2000BDE8F08FB8F1000F03D117B90EB9002D02
:105A30008DD04848002204A949F054FD002886D0A2
:105A400049F068FF002882D19FED430A41484BF09E
:105A5000FDF87CE70B2B7FF47AAFA0223F490DEBDA
:105A60000200BFF03FFA28AD002428460021B7EE1F
:105A7000000A013449F0FCFF0A2C05F11005F4D1AD
:105A800002A928A849F0A8FF03A983462CA849F039
:105A9000A3FF04A9824630A849F09EFF05A98146CC
:105AA00040A849F099FF06A9804634A849F094FF20
:105AB00007A9074638A849F08FFF08A906463CA861
:105AC00049F08AFF18A9054644A849F085FF044615
:105AD000BBF1000F08D1BAF1000F05D1B9F1000FE9
:105AE00002D1B8F1000F0ED01A4800220DF10701C3
:105AF00049F0F8FC38B149F00DFF20B99FED160AC6
:105B000014484BF0A3F827B91EB915B9002C3FF47F
:105B10001EAF134800220DF1070149F0E3FC0028F5
:105B20003FF415AF49F0F6FE00287FF410AF9FED6B
:105B30000A0A0B488BE700BF3C940D088C940D08B3
:105B40003C950D08CDCCCC3DBC950D08E7E30D0888
:105B5000FC950D0861DC0D08000000009C940D0808
:105B6000DCE30D080F299DBF302303FB01005030FB
:105B700000207047014B93F9BF047047584C002038
:105B8000024B93F88D0200F001007047585C002032
:105B9000044BB3F88434DB075ABF0069C0F34010EC
:105BA00000207047584C0020014BD3F8680E704716
:105BB000584C002008B503689B68984730B9044BDF
:105BC00093F98C02B0FA80F0400908BD0020FCE790
:105BD000585C002038B50D1E2DDB174C94F8742E40
:105BE000EBB29A4227D3D4F8703E0122595DA4F556
:105BF000005003F0B3FBF0B160F0FAFB032161F059
:105C0000FBFBC0B960F0F4FB0D2161F0F5FB90B92E
:105C100094F9A434EB40DB075CBF94F9BE14E9406F
:105C2000A4F5005048BF0221BDE8384058BF01F03C
:105C30000101FCF7E5BA38BD584C0020022A10B526
:105C40000C4605D1BDE810400948352203F086BB5B
:105C5000084BD3F8740203681B689847A04205D12B
:105C600060F0C6FBBDE8104060F04CBB10BD00BF4B
:105C7000582C0020585C002029B1022907D1044B80
:105C8000C3F86C127047024B0122C3F86C227047B4
:105C9000585C002031B1022907D1044B012283F85E
:105CA00070227047014B83F870127047585C0020D7
:105CB00010B500F50053DFED186AD3F8602ED3F865
:105CC0005C3EB2F90820B3F908309FED147A07EE74
:105CD000902AF8EEE77A0446C7EEA60A00F5A0502F
:105CE0000121103007EE903AF8EEE77A60EE870A6D
:105CF00087EEA60A20EE070A10F0BCFE54F0E8FC7E
:105D0000262154F07DFA04F54150054ABDE81040C3
:105D1000062157F083BF00BF0000C84235FA8E3C11
:105D200078EF0D0800F58042002382F8C03E044A57
:105D30000621137200F54150024A57F06FBF00BFB1
:105D40003D93002084EF0D0870B500F580450446B2
:105D500095F8C01E002956D02B4B2C4AD3F874025C
:105D6000904204D1D3F8983293F8CB3023B920462F
:105D7000BDE87040FFF7D6BF254E95F8C10E04F57B
:105D80004053012293F968323272C8BB002B3ADBD0
:105D900085F8C12E0139C9B204F5005385F8C01E3B
:105DA000D3F8602ED3F85C3EB2F90820DFED196A13
:105DB000B3F908309FED187A07EE902AF8EEE77AEB
:105DC000B1FA81F1C7EEA60A04F5A05049091030D6
:105DD00007EE903AF8EEE77A60EE870A87EEA60AB9
:105DE00020EE070A10F046FE95F8C03E5BB933720C
:105DF00004F54150094ABDE87040062157F00EBF36
:105E0000002BC7DAB3E770BD585C0020608F00201C
:105E10003D93002000007A4535FA8E3C98EF0D083E
:105E20006D2900F3E380012901DC61F029B98B1EA3
:105E30006B2BFAD80FF2040C5CF823F04B600108CE
:105E4000456001084B6001084B6001082B5E0108AA
:105E50004B6001082B5E01082B5E010845600108BC
:105E60002B5E01084B600108456001084560010890
:105E70002B5E01084B6001084B6001084B60010874
:105E80002B5E01082B5E0108456001084B6001088C
:105E9000456001082B5E0108456001084560010866
:105EA0002B5E01082B5E01082B5E01082B5E0108AA
:105EB0002B5E0108456001084B6001082B5E01085C
:105EC0002B5E01082B5E01084B6001082B5E010868
:105ED000456001082B5E01082B5E01084B6001083C
:105EE000456001082B5E01082B5E01082B5E01084E
:105EF0004B6001084B6001084B6001082B5E0108F4
:105F00002B5E01084B6001082B5E01082B5E010827
:105F10004B6001084B6001084B6001082B5E0108D3
:105F20002B5E01084B6001084B6001082B5E0108E5
:105F30002B5E01082B5E01082B5E01082B5E010819
:105F40002B5E01084B6001084B6001084B600108A3
:105F50004B6001084B6001084B6001082B5E010893
:105F600045600108456001082B5E01082B5E0108B1
:105F70002B5E01082B5E01082B5E01082B5E0108D9
:105F80004B600108456001082B5E01082B5E01088B
:105F90002B5E01082B5E01082B5E01082B5E0108B9
:105FA0002B5E01082B5E01082B5E01082B5E0108A9
:105FB0002B5E01082B5E01082B5E01082B5E010899
:105FC0004B6001082B5E01082B5E01082B5E010867
:105FD0002B5E01082B5E01082B5E01082B5E010879
:105FE0002B5E01082B5E010845600108A12921DC18
:105FF00096297FF71AAFA1F197030A2B3FF615AF49
:106000000FF2040C5CF823F04B6001084B600108B0
:106010002B5E01084B6001082B5E01082B5E010816
:106020002B5E01082B5E01084560010845600108F0
:106030004B600108B42908D0DB2903D0B2297FF4D2
:10604000F4AE7047002360F0EDBF704770B5632970
:106050008AB000F3D180012904DC0AB0BDE87040A9
:1060600060F06CBD8B1E612BF7D801A454F823F0AF
:106070007362010887620108A7620108AF62010824
:106080005B600108E36201085B6001085B60010876
:10609000956301085B6001085B6001089562010877
:1060A000BB6301085B60010891630108F5630108A7
:1060B000036401085B6001085B6001081364010868
:1060C000216401082F6401085B6001085164010824
:1060D000636401085B6001085B6001085B600108A4
:1060E0005B6001085B600108756401085B60010882
:1060F0005B6001085B6001085B600108CD6401081A
:106100005B6001085B6001085B6001085B6001087F
:10611000D1640108D56401085B6001085B60010877
:106120005B6001085B6001085B6001085B6001085F
:106130005B6001085B600108696501085B6001083C
:106140005B600108076401080B6401080F64010823
:106150005B6001085B6001085B6001085B6001082F
:106160005B6001085B6001085B6001085B6001081F
:106170005B6001085B6001085D65010861650108FD
:10618000656501086D65010871650108756501089F
:106190005B600108B7650108796501085B6001086B
:1061A0005B6001085B6001085B6001085B600108DF
:1061B0005B6001085B600108E96501085B6001083C
:1061C0005B6001085B6001085B6001085B600108BF
:1061D0005B6001085B6001085B6001085B600108AF
:1061E0005B6001085B6001085B6001085B6001089F
:1061F0005B600108F9650108A1291FDC97297FF779
:106200002CAFA1F19803092B3FF627AF01A454F856
:1062100023F000BFFD6501085B60010811660108FD
:106220005B6001085B6001085B6001085B6001085E
:10623000F16501085B6001089D640108B42900F064
:10624000DB80DB2917D0B2297FF407AF002A00F0EA
:10625000C381022A0FD1AB4BD3F874020368DB6F02
:10626000984740B95EF0BAFBA74A042157F0D6FC24
:1062700001E0022A01D0012430E035220E21A3489A
:1062800003F06CF8F7E7111E18BF01219F48FBF7D8
:10629000B7FFF0E7012A04D0022A14BF002102212F
:1062A000F4E71146F2E70621FFF7C8FCE3E7022A0C
:1062B000E1D1944DD5F874020368DB6A984704462F
:1062C0000028D8D0A5F58053D3F8643EB3F9083040
:1062D000002BD0D1A5F54050FFF7EAFC20460AB0CC
:1062E00070BD022AC7D1874E894AD6F874129142EE
:1062F000C1D0D6F8982292F8CB20002ABBD006F560
:106300000054A6F58056B4F9482A2AB9D6F8643E56
:10631000B3F90830002BAED01C22002103A805AD34
:10632000BEF02AFE284615F041FBB4F9483A794CF4
:1063300093B91623ADF80E30D4F87C3E7648642B22
:10634000B8BF642303A906932BF03CFE20B154F0A0
:10635000BFF9272153F054FF04F678630FCB85E88B
:106360000F00D6F8643E6C48B3F90830002BCCBF60
:106370001023152303A9ADF80E302BF023FE0028BF
:106380003FF479AF54F0A4F9272153F039FF72E7B5
:10639000032189E7022A04D0604B002283F8782E7B
:1063A00069E75F4819214BF0EBFA04460028F3D067
:1063B0005A4B012283F8782E90E7012A0BD0022A4B
:1063C00011D0002A7FF457AF544B83F8E82454F0DF
:1063D0007FF92B21D9E7514B019283F8E82454F03F
:1063E00077F92C21D1E74D4B83F8E82454F070F96C
:1063F0002D21CAE70F2157E74A4811468FF04EFC7E
:1064000039E7092150E704214EE705214CE7172120
:106410004AE7901E41424141434867F0AFFA2AE7FC
:10642000022A7FF428AF394800F0F8FF23E7012A59
:1064300006D0022A07D0002A7FF41DAF1146EBE7F1
:1064400011460192E8E73848012167F097FAEAE738
:10645000304B023AD3F8A43E5442544183F82040D2
:1064600009E7931E594259412A4BD3F8A40E82F0F2
:1064700047F900E7234BD3F8981291F8F51001295A
:106480003FF4F9AE541E012C93F86A228CBF00240D
:10649000012464F3041283F86A22ECE662B1022A52
:1064A0007FF4E9AE174BD3F8982292F8A13143F06C
:1064B000020382F8A131DEE6124BD3F8983293F84A
:1064C000A11162F3410183F8A111D4E61221EBE698
:1064D0001521E9E6002A38D0022A7FF4CCAE094D16
:1064E000D5F8740203681B6C98470446F0B105F5B3
:1064F00080550121D5F8A40E0368D3F8A030984741
:10650000ECE600BF585C0020FCEF0D08582C002082
:1065100030860020586C00206C860020584C0020EB
:10652000883B002044880020707C00205EF056FAF2
:106530000446D5F8740203685B6C98473D4A0346ED
:106540000421204657F06AFB95E63B4BD3F8A40E96
:1065500003681146D3F8A03098478CE60021A3E6E3
:106560001021A1E602219FE601219DE616219BE66E
:10657000072199E60B2197E6022A304B0ED1012420
:1065800083F8384954F0A4F84A2153F039FE5EF0FC
:1065900025FA2B4A062157F041FB9FE6002283F89B
:1065A000382954F095F84B2153F02AFE5EF016FA84
:1065B000244A06215AE6012A09D0022A0AD0002AD2
:1065C0007FF459AE012120480DF0D0F853E6019236
:1065D0000021F8E71146F6E71C4BD3F87402036874
:1065E000D3F88030984746E61146FFF745FB42E670
:1065F0001146FFF74FFB3EE61B2155E6022A7FF4CA
:106600003AAE1348FCF7A8FB5EF0E8F9114AD0E770
:10661000114660F0B5F910487EF0E0FD0446002810
:106620003FF429AE094A92F86B3243F0020382F834
:106630006B3253E6B0EF0D08586C0020587C0020F8
:10664000D9EF0D08EAEF0D08605B0020585C0020D0
:10665000582C002015F00D08D85B002010B504461A
:10666000044887F085FB04F10801BDE8104028F0DC
:10667000D7BA00BFE07A002038B504462DED028B72
:10668000114887F07BFB05462AF034FA0F48B0EE3C
:10669000408A0DF03FF990B1DFED0D7AB4EEE78A54
:1066A000F1EE10FA0BDDD5ED000A95ED010ABCF014
:1066B000D3F9DFED087A20EE270A84ED080ABDEC55
:1066C000028B94ED080A38BDE07A0020582C002097
:1066D00000401C46E02E6542074B93F9A5040228B2
:1066E00005D0032806D0003818BF0120704781F07C
:1066F0000100704704207047584C002003688B420B
:1067000016D00429C0E9001302D007290ED0704723
:10671000084B9FED097A03F5C263D3ED007AF8EEDA
:10672000E77A67EE877AC0ED087A704700238362C4
:10673000704700BF583C00200AD7233C08B50246EA
:10674000FFF7CAFFBDE8084001461046FFF7D6BF75
:1067500070B52DED048B0446F0EE408AB0EE608AF1
:106760000D46164691F0A6F99FED329ADFED329A6A
:10677000E06176B3236843B9304B03F5C263D3EDD0
:10678000007AF8EEE77AC4ED097A68EE898A002D7E
:10679000B7EE000AFFEE007AB8BFB0EE670A68EE07
:1067A000808AC4ED058A264BB4EEE98AF1EE10FA30
:1067B000D3F8A40E30DA80F081FF20EE090A84EDD0
:1067C000060ABDEC048B20460321BDE87040FFF7AC
:1067D00095BF94ED090A98EE890A27F073F9002D08
:1067E00084ED050A0BDAB4EEE90AF1EE10FADADB11
:1067F000DFED147A30EE670A84ED050AD3E7D2D0D4
:10680000DFED117AB4EEE70AF1EE10FACBD8DFED46
:106810000D7A30EE270AEFE780F050FFB4EE480A19
:10682000F1EE10FA48BFB0EE408A28EE098A84EDF6
:10683000068AC6E70000C84200000034583C002029
:10684000586C002000A00C47000000B410B52DEDDE
:10685000028B0446B0EE608AF0EE408A91F02AF98D
:10686000DFED090AE06168EEA08A68EE200AC4ED57
:10687000098ABDEC028BC4ED0A0A20460621BDE858
:106880001040FFF73BBF00BF0000C84210B52DED20
:10689000028B0446B0EE408A91F00CF994ED090A9F
:1068A000DFED097AE061A8EE270A27F0F5F8BDECE4
:1068B000028B002384ED090AA36220460621BDE86D
:1068C0001040FFF71BBF00BF0000C84270B54B6807
:1068D000154D06460C4673B98B6863B9C96851B942
:1068E0001248FFF72BFF95F8BD1F05F64470BDE871
:1068F000704062F06FBB95F8BD1F0D4862F00AFA58
:1069000048B906F10801204615F012FA18B10748F7
:106910000221FFF7F3FE95F8BD1F05482246BDE8AA
:10692000704062F04BBB00BF586C00206C9100209F
:106930009C7B002008B50721FFF7E0FE80ED0A0AE6
:1069400008BD000008B50368032B23D1D0ED057AFC
:106950009FED127AF0EEE77AF4EEC77AF1EE10FAD4
:106960001AD50F4B90ED090A03F5C263D3ED007AF7
:10697000F8EEE77A37EEC00A27F0A4F8DFED097ADF
:10698000B0EEC00AB4EEE70AF1EE10FA94BF0120AF
:10699000002008BD0120FCE70020FAE700000034D9
:1069A000583C00200000484330B50368023B85B0E6
:1069B0000446082B6DD8DFE803F0050D30374B6136
:1069C0003F616100FFF74AFE84ED090A94ED090A70
:1069D00005B030BD91F06EF8E369DFED310AE0619A
:1069E000C31A07EE903AF8EE677A94ED050A67EE5F
:1069F000A07AD4ED060AF12020EEA71A67EEE00A8D
:106A000027F0B6F8D4ED057A77EEC07AC4ED057AB2
:106A1000D4ED097A37EE800AD6E7FFF72DFEDFEDD9
:106A2000217A20EE270ACFE71F4BD3EDB07AF8EE9C
:106A3000E77AC0ED097AC9E71C4DD5F8B80E85F0A4
:106A4000CDFA0028C2D0D5F8B83E1B6B6362BDE713
:106A500091F030F8E3699FED127AD4ED0A6AE061B3
:106A6000C31A07EE903AF8EE677A67EE877A94EDEC
:106A7000097AA6EEA77A84ED097AA7E70B4B9FED7A
:106A80000C0AD3F8A40E6C302AF0F2FA84ED091A3D
:106A90009CE7064BD3F8AC3ED3F84433D6E700BFAF
:106AA0006F12833A0000C842585C0020586C0020E6
:106AB0009F0CB3450368092B08D8DFE803F0050AEB
:106AC00005050505070705100023836290ED0A0AF6
:106AD0007047044BD3F8AC3ED3F84833F5E7C36AAC
:106AE000F3E700BF586C0020F8B50023214FCB62BC
:106AF00097F88D32204E13F0010F04460D462DD12C
:106B0000D7F8740203689B6F984738B3D7F87402BC
:106B100003F00EF8DFED197A85ED0B0AB0EEC00A2E
:106B2000B4EEE70AF1EE10FA03D409213046FFF77C
:106B3000E5FD1148FFF738FF0F4884ED000AFFF725
:106B4000B9FF336884ED010A0A2B0FD8DFE803F0A0
:106B50000C1010101010100C100C0C003368092BC6
:106B6000E7D105480021E2E70223A3602046F8BDF3
:106B70000123FAE7585C00206C91002000000034EB
:106B8000034B01221A6000229A60DA601A61704792
:106B90006C91002013B501A904460CF02DFD04F5FD
:106BA000804320B9012283F8ED2F02B010BDDDED46
:106BB000017ADFED096A03F57E62B8EEE77AD2ED7D
:106BC000007A67EEA67AB4EEE77AF1EE10FA54BFD7
:106BD00001220022E7E700BF0000C8422DE9F04F84
:106BE0002DED068B00F500538DB000F5A0590193F3
:106BF00093F9FA34054600F5A04409F1100933B1C0
:106C000000F54058D8F8983293F8CB707FB900213E
:106C1000A4F82C19484610F01DF994F82D1948468F
:106C20000DB0BDEC068BBDE8F04F10F01DB990F033
:106C300041FF05F5804B0090DBF8AC0E9FED958A87
:106C400090EDDBAA83F0D2F909AE002800F0CD80E8
:106C5000DBF8AC3E03F55C7393E8070086E80700B9
:106C600030468DED0B8A2AF001FEB0EE409A2846A0
:106C70000CF050FE05F59D4A0AF1080A002800F0C4
:106C8000B780504687F07AF807C886E80700304694
:106C90008DED0B8A2AF0EAFDF0EE409AD8F87402E6
:106CA00003681B689847122840F0AB80002384F8E3
:106CB0002C39D8F8740203685B69984730B1019B9E
:106CC000D3F8643EB3F90830002B0DDC98F9683234
:106CD000002B09DA009BC4F83039504687F04AF897
:106CE00004F6341383ED000A94F82C395BB1009B51
:106CF000D4F83009181A41F28833984240F28F8054
:106D0000002384F82C39DBF8A40E9FED630A6C3065
:106D10002AF0AEF98DED090ACDED0A0A8DED0B1AB8
:106D200096E8070006AB03AE9FED5C0A83E8070018
:106D300086E8070030462AF09BF92846B0EE408AE4
:106D4000F0EE608A8DED060ACDED070A8DED081A8A
:106D50000CF0E0FD002874D0DFED517AF4EEE79AF4
:106D6000F1EE10FA94BF01250025DBF8AC0E83F09C
:106D70003DF930B1DFED4A7AB4EEE79AF1EE10FA60
:106D800009D9002D64D1D8F8740203681B689847AC
:106D9000022864D00027DBF8AC0E83F049FA0546E0
:106DA000002873D0B5EEC0AAF1EE10FA6DD5DFED74
:106DB0003D7AB4EEE7AAF1EE10FAACBF0126002648
:106DC000504686F0E3FF5EB9DFED377AB0EEC00AD9
:106DD000B4EEE70AF1EE10FA5AD8002D08BF0027EA
:106DE00094F82C1984F82D7914E7B0EE489A3EE710
:106DF00028460CF05FFD00287FF443AFDFED259AB5
:106E00004CE7D8F8983293F8CB30002B3FF451AFD1
:106E100098F96832002BBFF64CAF012347E7504684
:106E200086F0A8FF04F63413D3ED007A30EE670A3B
:106E3000DFED1E7AB4EEE70AF1EE10FA3FF760AF2D
:106E400061E728460CF036FD0546002884D18CE722
:106E5000DBF8AC0E83F0CAF8002894D19BE7B0EEC3
:106E6000680ABBF0D7FBF0EE408AB0EE480ABBF0F0
:106E7000D1FBDFED0F7A20EE280AB4EEE70AF1EE3F
:106E800010FACCBF0127002785E700252E4697E79B
:106E90003746A5E7000000009F0CB345D302373901
:106EA0000000FA420000C8C20000704200004842E0
:106EB00055CF7D3F38B504460CF02CFD04F5A055A8
:106EC000103548B920460CF0F5FC014620B928469B
:106ED000BDE838400FF01EBA04F54054D4F87402EF
:106EE0000368DB6C984720B9D4F8740203681B6D03
:106EF00098470146EBE7000030B5044689B0684684
:106F000004F5A05514F052FD103504A814F04EFD00
:106F1000694628460FF0B8FA98B104A928460FF040
:106F200003FB70B1059B019323680022DB6C69466B
:106F30002046984728B104F5315001212C308AF0C1
:106F400075FD09B030BD000000F5805292F88C2626
:106F5000D2070BD400F54052D2F8982292F8CB1009
:106F600009B1FFF7C9BF03689B6C18477047000061
:106F700030B587B0044602A8019114F017FD04F55E
:106F8000A05002A910300FF07FFA019A18B900251D
:106F9000284607B030BD236802A9DB6C204698471D
:106FA00005460028F3D004F5315001212C308AF039
:106FB0003DFDEDE7F0B5044685B004F5A056684602
:106FC00010360F46154614F0F1FC694630460FF0B6
:106FD000ABFA10B9002005B0F0BD394630460FF0CD
:106FE0000BF90028F6D0002DF5D004F58054284682
:106FF00094F88C3643F0020384F88C36EBE70000FB
:1070000003207047F0B5544FD7F8283EDA0785B013
:10701000044600F19E8000F54055D5F8983293F86B
:10702000C120002A40F0958093F8CB30002B00F06F
:107030008D8095F96832002BC0F2888000F5A0435E
:1070400093F83839002B40F0848000F580469FED9E
:10705000430AD6F8A40E6C302AF00AF8CDED020AE5
:1070600060EEA00ADFED3E7A8DED010AE0EE000A47
:107070008DED031AF4EEE70AF1EE10FA66DCD6F8AD
:10708000A43E9FED387AD3ED377AF4EEC77AF1EE6D
:1070900010FA04D5D5F898321B7A002B56D0B5EEED
:1070A000007AF4EEC77AF1EE10FA4FD404F59D4061
:1070B000083086F06BFEDFED2C7AB4EEE70AF1EED5
:1070C00010FA43D8D6F8A43E9FED287AD3ED367A4D
:1070D00067EE877AB3EE0E7AF4EEC77AF1EE10FA25
:1070E00034DA234AB4F9A410138801339BB2138015
:1070F00019B9B4F8A210A4F8A410B4F8A4109942D5
:1071000027D80026168053F0E3FA0122192153F004
:1071100097F8D5F8980203685B699847154A431CAD
:10712000314604F5415056F079FDD5F898320122E8
:1071300083F8C120D7F8283E5B070AD504F597509D
:10714000143005B0BDE8F0406AF00ABC084B0022DC
:107150001A8005B0F0BD00BF584C00209F0CB3450D
:107160004054094A6666663F000000B4E02E65425E
:10717000A691002000F20D08F0B52DED028B4A4BD0
:10718000D3F8283E9B0785B004461FD400F58046FF
:10719000DFED468AD6F8A40E03681B699847D0ED48
:1071A000017AF4EEE87AF1EE10FA0FDB04F54053C1
:1071B00004F5B245D3F8982292F8C1103C3549B194
:1071C000002303A92846039355F03EFF05B0BDEC0C
:1071D000028BF0BD92F8CB20002AF1D093F96832EF
:1071E000002BEDDB04F5A04797F83839002BE7D1E9
:1071F000D6F8A40E03681B699847D0F8A430D6F8D7
:10720000A40E039303681B69984704F58C7200F180
:10721000A401284656F020F8DDED037AB0EEC08ACE
:10722000F0EEE77AF4EEC87AF1EE10FA03D503A98E
:10723000284655F009FFD6F8A40E03681B69984745
:10724000D0ED040AF4EEE80AF1EE10FABEDBF6EE39
:10725000087A60EEA77AF4EEC87AF1EE10FA1CD53F
:1072600090F028FCD7F8483942F21072C31A9342C2
:10727000ACD9DFED0F7AC7F8480968EE277A04F534
:10728000415417EE900AF9F747F90A4ACDE900018F
:107290000021204656F0C2FC98E79DED030A26F037
:1072A00063FB0028DCD191E7584C0020000000343B
:1072B0000000C8421CF20D0810B5044600F5A040BD
:1072C000183066F06DFB04F5A0400121BDE81040C8
:1072D00038306EF00BBD00002DE9F04100F5A046FE
:1072E000044696F9183043B300F5405596F82C2023
:1072F00095F86832DB43C3F3C01363F3C30200F5B0
:107300009D4086F82C20083086F040FD3746DFEDA2
:107310003F7A183720EE670A384666F0C1FB96F8C8
:10732000383953B9384666F067FBD5F8983293F888
:10733000CB3023B9364B00221A80BDE8F08196F895
:107340002C30DB07F9D4D5F8740203689B6B98479F
:107350000028EFD095F96832002BEBDB2C4D2B8801
:1073600004F580484BB9B6F91E3033B1642213FBE3
:1073700002F3D8F87C2E9A42DFDB384666F0ACFB8D
:10738000D8F8A43E9FED237AD3ED367A67EE877A5C
:10739000B3EE0E7AF4EEC77AF1EE10FA05D82B8828
:1073A000002BCAD0013B2B80C7E7B4F9A4301BB92E
:1073B000B4F8A230A4F8A4302B88B4F8A420B4F90F
:1073C000A400154993423CBF01332B802B88D8F889
:1073D000542E012B01D10A60AFE709689142A9DD63
:1073E00018B9B4F8A220A4F8A420B4F8A4209A42B2
:1073F000A3D800232B8053F06BF902220C2152F00A
:107400001FFF2046BDE8F041FFF756BF0AD7233CD7
:10741000A4910020E02E6542A091002008B500F55F
:10742000A04393F918206AB300F5405292F96822FC
:10743000002A0DDA144A062100F5415056F0EEFB01
:1074400053F046F90322BDE808400F2152F0F8BE80
:10745000B3F91E3093B100F580426421D2F87C2E3E
:1074600013FB01F39A4209DA084A012100F5415061
:1074700056F0D4FB53F02CF90222E4E7BDE80840B3
:10748000FFF71ABF08BD00BF34F20D0846F20D0821
:1074900070B52DED028B00F540555A4ED5F8983257
:1074A00093F8CB308CB0044643B195F96832002B89
:1074B00004DB00F5005393F9CE342BB9002333805D
:1074C0000CB0BDEC028B70BD00F5A04393F83839C9
:1074D000002BF3D101F032FB00287AD1D5F87402E9
:1074E00003689B6B98470028E8D004F59C4058300F
:1074F00055F00AFE2AF0BAF9F0EE087AB4EEE70A7F
:10750000F1EE10FAF0EE408AD8DA04F5A053D3ED8C
:10751000977A93ED960A20EE270ABBF035FADFED55
:107520003A7A20EE270AB2EE0E7AB4EEC70AF1EEEE
:1075300010FAC3D904F58043D3F8A43E93ED368AFC
:1075400028EE278AF3EE0E7AB4EEE78AF1EE10FA0F
:10755000B4D904F5A050002309A9103009930A9367
:107560000B930EF0EDFF00283CD13388B4F9A42032
:1075700001339BB23380002A3FD0B4F8A420B3EB90
:10758000420F9DDB53F0A4F801220C2152F058FE6B
:107590001E4B002218EE900ACDE90623F8F7BCFF37
:1075A0001B4BCDE90401002218EE100ACDE902239D
:1075B000F8F7B2FF04F54154CDE90001154A204621
:1075C000002156F02BFB01220C211348FAF70CFD89
:1075D00076E7D5F8740203681B6D984700287FF49E
:1075E0007DAF6BE709A82AF041F9F2EE047AB4EE18
:1075F000E70AF1EE10FAB8DB60E7B4F8A220A4F8CD
:10760000A420BAE79C910020E02E654200000840CB
:1076100000003E405CF20D08D85B0020F0B52DED77
:10762000028B8BB0002307930893099305AB0446A4
:10763000019300F5A05007AB009302AA04AB03A985
:1076400010300EF095FE04F54057054687F83400DB
:1076500028B9002528460BB0BDEC028BF0BD90F098
:107660001DFABB6B9FED337AC31A07EE903AF8EE22
:10767000677A064667EE877A04F5405006AA02A9A3
:107680001030CDED067A55F0E7FD04F5405006AA1E
:1076900003A91C308DED020A55F0DEFD04F54050C3
:1076A00006AA04A9283004F500548DED030A55F00C
:1076B000D3FDBE6304F59A6393ED008AB5EEC08AEC
:1076C000F1EE10FAC5D9DDED080A9DED070ABBF011
:1076D00027F8DDED090ABBF023F8D4F8B82FDDED6B
:1076E000037AB4EEC08AF1EE10FA94BF01230023AE
:1076F0001AB194F8BC2FD20712D438EE087AB4EE3F
:10770000E77AF1EE10FA0BD80233DBB2DDED027A44
:10771000B4EEE78AF1EE10FA09D8002B99D099E778
:10772000B4EEE78AF1EE10FAF0D80133EDE7012B61
:1077300090D88EE7BD37863570B500F540550446C4
:1077400095F88D3243F0040385F88D3252F0C0FF76
:107750000122112152F074FDD5F8983293F8CB3004
:10776000002B42D0D5F8740203681B68984709289B
:107770000AD1204608F0F6FB30B104F5C24064306F
:10778000BDE8704008F0D6BB184BD3F8740203680C
:107790001B69984704F5005340B993F9CD34032B86
:1077A00023D10621204608F0C9FB0DE093F9CD1442
:1077B0000229F6D195F88D32DB07F2D40622204655
:1077C00001F0CCFD0028ECD0094BD5F87402012261
:1077D0005A7303685B6C9847064A0346022104F516
:1077E0004150BDE8704056F019BA70BD585C002099
:1077F0003D93002090F20D0808B500F5405292F834
:107800008D32590716D56FF3820382F88D320A4BF9
:107810005A7B3AB100225A730221084A00F54150BE
:1078200056F0FCF952F054FFBDE808400022112147
:1078300052F006BD08BD00BF3D930020B4F20D0814
:10784000F0B5054685B005F5A0576846103714F029
:10785000ADF8694638460EF067FE80B105F5135362
:10786000D3ED047A374CF5EEC07AF1EE10FA08D871
:10787000354A002328462380D373FFF7BDFF05B0A8
:10788000F0BD2846FFF7CAFE064628460CF012F85F
:1078900010B928460BF0E8FFA378002E18BF00208F
:1078A0000343DBB2A370002BE9D06378A0BB7BBBA2
:1078B00023780133DBB2082B237003D146B338465B
:1078C0000EF0C2FD2378092B02D138460EF0B4FD2C
:1078D0002378092B1CD94FF48573238052F0F8FECE
:1078E0000222102152F0ACFC90F0E4F86368C01A58
:1078F00047F23053984208D9144A022105F5415005
:1079000056F08CF990F0D6F860602846FFF714FF27
:107910000D4B6278DA73B2E72678002EF8D0013E7C
:10792000F6B22670002BF3D0002EF1D1667052F023
:10793000CFFE3246102152F083FC2846FFF75CFF51
:10794000E6E700BFA89100203D930020CCF20D088F
:1079500000F5405393F88D325B0701D5FFF7ECBE7D
:107960007047000073B5044600F5A05001A910301F
:1079700004F500560EF046FBD6F8FC3F8342054660
:107980000CD004F58043D3F8A40E81F0FFF8C6F8BC
:10799000FC5F52F09DFE3E2152F032FC04F5805611
:1079A00004F5405596F9202795F9001096F82037F0
:1079B000914218D0FF2B16D004F58043D3F8A40EC3
:1079C00081F0E4F896F820372B7052F081FE2A7887
:1079D000182152F035FC95F90030044A042104F5D1
:1079E000415056F01BF902B070BD00BFDCF20D082B
:1079F0002DE9F0438FB0054690F05CF80023059325
:107A000006930793089309930A930B930C930D9392
:107A100005F5A05804AB019308F1100803AB0093DF
:107A200006460BAB08AA05A940460EF081FCDFED27
:107A3000477A9DED077AB4EEE77AF1EE10FA074641
:107A400032DB9DED0A7AB4EEE77AF1EE10FAACBFC4
:107A50000124002405F54059404699F83430002BA4
:107A600008BF00270EF076FC8046FFB9444605F5B6
:107A7000005393F9C43D012B29D164B1D9F8983250
:107A800093F8CB403CB1D9F8740203685B6998471E
:107A900080F00100C4B299F80430C3BBCCB9C9F876
:107AA00008600FB0BDE8F0830024D3E7002CDDD0E0
:107AB00005F540501C3055F0C5FA90ED007AF7EE10
:107AC000007AB4EEE77AF1EE10FAD0DCCEE70024CB
:107AD000E1E7D9F80800301AB0F57A7FE1D9C9F8A2
:107AE0000C30012405F5804389F80440D3F8AC3EFE
:107AF00083F80C4452F0ECFD22461D2152F0A0FB0D
:107B0000134A022105F5415056F088F8C9E714B12F
:107B1000C9F80C60C5E7D9F80C0043F69823361A6B
:107B20009E42BED905F58043C9F8084089F8044053
:107B3000D3F8AC3E83F80C44C9F80C4052F0C8FDB1
:107B400022461D2152F07CFB024ADAE70000003495
:107B5000F4F20D080EF30D08704700000B46034ABF
:107B6000042100F5415056F059B800BF2CF30D0820
:107B700010B5044652F0ACFD0022052152F060FB26
:107B800004F54150024ABDE81040042156F046B8C1
:107B900038F30D0813B50B4642B100920421064A92
:107BA00000F5415056F03AF802B010BD02B0BDE801
:107BB0001040FFF7D3BF00BF50F30D0808B5074AC8
:107BC000042100F5415056F029F852F081FDBDE83E
:107BD00008400022082152F033BB00BF64F30D08B7
:107BE00038B504460D468FF065FF04F540533DB9A6
:107BF000D3F88422C3F888020AB9C3F8840238BDD6
:107C0000D3F88822801A642884BF0022C3E9A12205
:107C1000F5E7000037B5044600F59D40083086F0D2
:107C20009BF804F54052C0F3803592F86A32C3F3F2
:107C30004001A9421CD065F3410382F86A3204F581
:107C400041546DB152F044FD02220B2152F0F8FA7A
:107C5000084A0221204603B0BDE8304055F0DEBF9F
:107C600052F036FD2A460B2152F0EAFA024AF0E7BA
:107C700003B030BD7CF30D0898F30D0838B50A4603
:107C80000C460621054601F069FB28B1054A137828
:107C900043F00803137038BD21462846BDE838403C
:107CA00008F04CB95C93002038B50A460D46152102
:107CB000044601F053FB28B1084A137843F0080347
:107CC000137038BD04F541500421054A55F0A6FF54
:107CD00029462046BDE8384008F030B95C930020C2
:107CE000A8F30D0838B50A460D461521044601F0E3
:107CF00035FB28B1084A137843F00803137038BDE8
:107D000004F541500421054A55F088FF29462046D4
:107D1000BDE83840FFF7B2BF5C930020D0F30D08F8
:107D200038B50A460D461B21044601F017FB28B161
:107D3000084A137843F00803137038BD04F5415026
:107D40000421054A55F06AFF29462046BDE838401F
:107D5000FFF794BF5C930020E6F30D0838B5074A9F
:107D600004460D4600F54150042155F057FF2946C1
:107D70002046BDE8384008F0E1B800BFF8F30D0830
:107D800010B500F5405494F86A329A0623D4D4F81A
:107D9000740203681B689847032808D005D8022896
:107DA0000ED194F86802C00914E01B28F9D194F8A8
:107DB000680200F0A000A0F180035842584109E099
:107DC000B4F8680220F4FE4020F07F0080B2003852
:107DD00018BF012010BD0120FCE7000038B500F5F8
:107DE0004055194A95F88D3243F0080385F88D32D5
:107DF0000221044600F5415055F010FF52F068FC96
:107E00000122172152F01CFA2046FFF7B9FF38B1C2
:107E100004F53E500122BDE838401521FAF7E4B8D8
:107E2000D5F8740203681B689847062806D104F544
:107E3000C4407C30BDE8384009F08CBA20460B21A4
:107E4000BDE83840FFF71ABF0CF40D0870B500F517
:107E50004055D5E9A1239B1A41F288329342064648
:107E600011D9D5F8740203685B6D9847044695F8FC
:107E70008D32C3F3C003A34213D034B13046BDE802
:107E80007040FFF7ABBF0024F1E752F021FC22461F
:107E9000172152F0D5F995F88D3264F3C30385F8B4
:107EA0008D3270BD0B4610B511460446072B07D81E
:107EB000DFE803F029041316191C232608F03EF806
:107EC00004F50053D3F8C83D9B061CD504F5975024
:107ED0001430BDE8104069F043BDFFF7CFFEEFE777
:107EE000FFF700FFECE7FFF7DFFEE9E701221421CF
:107EF00000F53E50FAF778F8E2E7FFF711FFDFE709
:107F0000FFF72CFFDCE710BDF8B5044604F5005779
:107F100052F0DEFB0122052152F092F997F8B234BB
:107F2000072B98BF2F4A204694BFD55C0125FFF749
:107F300027FF60B12C4A2D492046FFF72BFE012276
:107F4000102104F53E50FAF74FF8002514E004F52F
:107F50004056D6F8740203681B6D984798B196F89E
:107F6000353883B196F93438012B0CDC204A21498D
:107F70002046FFF70FFE0125294620460322BDE8D3
:107F8000F840FFF78FBFD6F8740203681B6D98475F
:107F900018B1D7F8C83D190715D4D6F8740203688C
:107FA0001B689847032803D1D7F8C83DDA070DD4DA
:107FB000D6F8740203685B6A984768B90B49204693
:107FC000FFF7CCFDD8E70A4A0849D1E70A4A074932
:107FD0002046FFF7DFFDB8E7D7F8C83D5B07EDD5D2
:107FE000064AF4E7ECF40D082CF40D08CACC0E0890
:107FF00036F40D0849F40D0859F40D0869F40D081C
:1080000038B50446154652F063FB0122062152F0B2
:1080100017F92046FFF7B4FE90B10122072104F5BD
:108020003E50F9F7E1FF144A14492046FFF7B2FD2C
:108030000025294620460422BDE83840FFF732BF1C
:1080400004F54053EDB2D3F8740203681B6D9847F2
:1080500068B104F50053D3F8C83D1B0707D535B107
:10806000074A06492046FFF795FD0125E1E7034948
:108070002046FFF773FDDCE72CF40D0886F40D08AD
:1080800036F40D082DE9F041044604F5005752F08E
:108090001FFB0122082152F0D3F85EF0A9F897F8EF
:1080A000A134072B98BF384A04F5405698BFD55CD9
:1080B000D6F8983293F8CB8088BF0225B8F1000F2C
:1080C0000BD132492046FFF749FD002529462046BD
:1080D0000522BDE8F041FFF7E5BE2046FFF750FE60
:1080E00058B10122122104F53E50F9F77DFF284ACC
:1080F00026492046FFF74EFDE7E7D6F874020368ED
:108100001B6D984768B196F8353853B196F93438F5
:10811000012B06DC1F4A20492046FFF73BFD0125C5
:10812000D4E7D6F8740203681B6D984718B1D7F8E6
:10813000C83D190713D4D6F8740203681B68984722
:10814000032803D1D7F8C83D9A070BD4D7F8C83D08
:10815000DB0609D40D492046FFF700FDB6E70D4ABE
:108160000A49D9E70D4AC3E7D6F874020368DB6908
:10817000984706460028EDD1094A04492046FFF7F2
:1081800009FD3546A2E700BFF4F40D089FE00D0895
:108190002CF40D0836F40D0880F40D088EF40D084B
:1081A000A3F40D08F8B500F50055044695F9A1347F
:1081B000BBB300F54056D6F8F87197B38FF07AFC50
:1081C00005F5626595ED000ADFED167A9FED161A4A
:1081D000DFED160AC71B20EE270A8D2025F0C8FC0C
:1081E000BCEEC00A10EE103A9F420CD296F88D32C7
:1081F0009A0716D520460021FAF750F82046BDE828
:10820000F840FFF7DBBC0CD996F88D329B0708D4F9
:1082100020460121FAF742F82046BDE8F840FFF772
:1082200031BFF8BD00007A440000804F000000001C
:108230002DE9F341074600F59D40083085F08CFD9F
:1082400007F54054C0F3804801908FF033FC94F858
:1082500090324345454606460CD084F8908207F597
:108260004150002D40D03B4B3B4AC4F89462022160
:1082700055F0D4FC94F8903207F500583BB394F8CD
:10828000913223BBB8F9363E9FED340A9FED341A84
:10829000DFED340A07EE903AF8EEE77A40F2571035
:1082A00027EE800A25F064FCBCEEC00AD4F89402E4
:1082B00010EE103A361A9E4209D9012384F8913201
:1082C000294A244B022107F5415055F0A7FC98F9A3
:1082D000353E002B94F88D320DDC6FF3451384F896
:1082E0008D3202B0BDE8F0811A4B204AC4F8948266
:1082F00084F89182BBE7C3F34012AA42F1D065F340
:10830000451384F88D329B06EBD5194BD3F87402D4
:1083100003681B6998470028E3D052F0D9F901227D
:108320001F2151F08DFF3846FFF72AFD40B1012291
:10833000212107F53E5002B0BDE8F041F9F754BEE7
:1083400098F8351E3222384602B0BDE8F041FFF7FA
:10835000A9BD00BFBCF40D08CBF40D0800007A44A1
:108360000000804F00000000E1F40D08D6F40D0875
:10837000585C002008B5044B01221A708FF08EFB68
:10838000024B186008BD00BFB1910020B4910020DD
:10839000014B00221A707047B19100202DE9F04185
:1083A00004468FF07BFB2A4BB4F8BE201988294E77
:1083B000914205460ED01A80274B18603378A3B13E
:1083C0000024347052F084F922461321BDE8F041B4
:1083D00051F036BF3378214FDBB93B782BB11E4BC0
:1083E0001F4A1B68C31A934201D8BDE8F0810123DC
:1083F000337004F54053D3F8980290F8CB3013B1A2
:1084000003689B6A984752F063F90122132151F0E7
:1084100017FF3B78002BE8D03378002BE5D00E4ACD
:1084200010491368EB1A8B42DFD904F540541560EC
:10843000D4F8980290F8CB30002BD6D0002188F0E9
:1084400015FBD4F898020368BDE8F0415B6A184751
:10845000B2910020B0910020B4910020B191002091
:1084600080841E0040420F002DE9F84300F540557E
:1084700000F500580446D5F8740298F85C73036858
:108480001B6D9847014650B995F96832002BA5BF7E
:10849000D5F8983293F8CB00012180F0010104F562
:1084A0000C5909F1200948466AF062FAD5F8983269
:1084B00093F8CB300646002B7AD0002865D03D4B90
:1084C00093F96832002B04DB02463B49484669F0C9
:1084D00029FE98F926734FB195F96832002B0DDA11
:1084E00001220F2104F53E50F9F77EFD52F0F0F81D
:1084F0003246BDE8F843092151F0A2BED5F8740216
:1085000003685B69984758B195F96932002B07DA1F
:1085100095F88D32DA0703D498F85C33DB07DFD5A2
:10852000314648466AF08AFADFED247AB4EEE70A6B
:10853000F1EE10FA05DD0A220921204600F00EFFB7
:10854000D4E7023F032F12D801A353F827F000BF4E
:1085500037850108618501087F8501088585010847
:108560000A221521204600F0F9FE0028BED10A2279
:108570000621204600F0F2FE0028B7D1DBE70A22F0
:108580001121F6E70A221521F3E78FB198F85C3341
:1085900073B9084B93F96832002B05DB084A0521B3
:1085A00004F5415055F03AFB52F092F80022A0E752
:1085B000BDE8F883585C0020FCF40D080000C842B8
:1085C00005F50D0810B500F5A044B7EE001A94F8B3
:1085D000F638DFED080A43F0010384F8F638252069
:1085E000B0EE410A25F0C4FA04F6F40484ED010A61
:1085F00010BD00BF0000000070B500F540560446F5
:10860000D6F8983293F8A130032B00F5A04509D095
:10861000394B00221A7095F8283962F3000385F867
:1086200028391AE0D6F8740203681B6D98470028B1
:10863000EED120460BF06EF980B104F59D40083074
:1086400085F0A0FBDFED2D7AB4EEE70AF1EE10FA2B
:1086500021DB95F82829D1073CD570BDD6F89802C2
:10866000443054F0EFFC0346DFED250A93ED000A99
:108670009F20B7EE001A25F07BFADFED227AB4EEE8
:10868000E70AF1EE10FAE4DC04F58053D3F80C2687
:108690001D4B9A42DDDB04F5005393F8783E6BB135
:1086A00004F573641921204649F060F9042805D1C6
:1086B0001921204649F07AF9C828CAD895F82839EE
:1086C000DA07CAD50C4991F90020002A10DD013AD9
:1086D0000A70C2E708490B7801335BB2632B0B7059
:1086E000BBDD42F00102642385F828290B70B4E752
:1086F0006FF3000393E700BFB891002000007A43B6
:1087000000000000CDCC4C3F24FAFFFF2DE9F041E2
:1087100000F5405704460121D7F8980285F0E2FDA4
:1087200004F58046014604F5A045D6F8A40E0029BC
:1087300058D10368D3F890309847B7F8683213F4EB
:108740008142D7F8983206D093F8A02142F0200257
:1087500083F8A02105E093F8A01162F3451183F896
:10876000A01197F96832B5F82A09002B0CDBD7F86D
:1087700098329FED257AD3ED3E7AF0EEE77AF4EE6B
:10878000C77AF1EE10FA3DD5013800B2A5F82A09F2
:10879000B4F9A4301BB9B4F8A230A4F8A430B4F9E9
:1087A000A420002125F022FAA5F82A09D6F8A43E33
:1087B000B4F9A4101A6807EE900AD2F89420B8EE23
:1087C000E70A19B9B4F8A210A4F8A410B4F8A410D8
:1087D00007EE901AF8EE677ABDE8F04180EE270ABE
:1087E0001846104795F828190368C943D3F8903004
:1087F00001F001019847D7F8983293F8A0216FF360
:108800004512A5E70130C0E70000003438B500F597
:1088100040550446D5F8740203685B69984708B16F
:10882000002038BDD5F8740203681B6898470B28F0
:10883000F6D004F58043D3F8A40E0368D3F8A4302F
:1088400098470028ECD1D5F8740203681B6D98474F
:108850000028E6D195F9682295F86832002A09DBEC
:108860009B0607D504F5A04494F82809C04300F0FE
:108870000100D6E70120D4E710B55DF0B9FD202155
:108880005EF0BAFD044670B14FF47A715DF0F6FD0A
:10889000B4F90830DFED057A00EE103AB8EEC00A00
:1088A00020EE270A10BD9FED020AFBE76F12833A04
:1088B0000000000070B500F540540646D4F8983228
:1088C00093F8F520012A0AD0023A022A3AD81A6807
:1088D00093F8CC10D26E39BB9FED1B0A2EE0FFF748
:1088E000CBFFDFED1A7AD4F8985294F86A32B4EEDE
:1088F000E70AF1EE10FA0DDD43F0100384F86A3256
:108900002B68DC6E3046FFF7B7FF28462346BDE8EC
:10891000704018476FF3041384F86A322B689FED98
:108920000A0ADB6E2846F2E7B3F9DC109FED070A6E
:1089300007EE901AF8EEE77A27EE800ABDE870405D
:108940001846104770BD00BF000000000AD7233C46
:1089500038B500F54054B4F86832D4F8980203F4FE
:10896000814333B101220021BDE83840D03083F08B
:1089700047BA90F8CC5055B9D4F8740203685B69D3
:10898000984720B1D4F898022A460121ECE7D4F8A0
:1089900098020022E7E7000038B50D4604468FF044
:1089A00089F8002D084B06DD186004F5A04400236B
:1089B00084F8293938BD1B68C01AB0F5C87FF9D9C9
:1089C00004F5A0440123F3E7BC91002038B500F57D
:1089D00040530446D3F89852FFF718FF95F8A0319A
:1089E00060F3000385F8A03104F500532046D3F866
:1089F000643EB3F90810BDE83840FFF7CDBF000072
:108A000070B500F5405300F59D45083586B01979DD
:108A10000446284685F04EF902A812F0C7FF04F577
:108A2000A05002A910300DF02FFD04F58043049AE8
:108A3000C3F8802E059AC3F8842E284685F08CF959
:108A400082061AD5284685F095F904F59C45FDEE79
:108A5000C07A783504F5805417EE901A0222284621
:108A600017EE906A12F0A8FF94F88C36DB0706D454
:108A700001223146284612F09FFF06B070BD012149
:108A8000284613F05DF80028F2D0F6E770B500F53F
:108A9000A04486B0B4F854398B420D46164603D133
:108AA000D4F85039934221D08FF004F8D4F84C39DF
:108AB000C31A132B1AD9C4F85069A4F85459C4F82E
:108AC0004C0951F005FE04468EF0FCFF084B094AA4
:108AD0001B68CDE90453084B0193084B0093CDE983
:108AE0000201074B0749204651F034FA06B070BD29
:108AF000C09100201CF50D0834F50D088EC90D0835
:108B0000D8AC0D082FF50D0838B500F540540D46CA
:108B100094F86932C3F380138B420BD021B151F02A
:108B2000D7FD112151F06CFB94F8693265F386137F
:108B300084F8693238BD00007047000010B500F5B8
:108B400080430446D3F8A40E0368D3F8A4309847B2
:108B500018B904F5405494F8700210BD2DE9F041A5
:108B600000F54055064695F86832B1EBD31F0C4628
:108B700047D0254B00221A6000293ED051F0A8FDB5
:108B8000122151F03DFB95F8683264F3C71385F864
:108B9000683284F0010876F059FC414676F032FCE8
:108BA00006F50057B8F1000F06D097F836341BB918
:108BB0008EF080FFC7F8380487F836840CB3B7F816
:108BC00084345B071DD5D5F8983293F8CB30C3B108
:108BD000D5F8740203685B69984790B9D5F87402B8
:108BE000036820219B69984758B106F53E50012241
:108BF000BDE8F0410D21F9F7F7B951F069FD1C21ED
:108C0000BFE7BDE8F08100BFC09100202DE9F04F23
:108C10002DED088B00F540558DB0D5F89822C74F43
:108C200092F8CB9000F5A04382460193B9F1000F72
:108C300004D10121FFF792FF002424E095F9682276
:108C4000002A18DAD5F874020268D26C90470446FC
:108C50000028F1D1D5F8982292F8A01111F0400126
:108C600000F0688192F8A120032A0CD101465046F9
:108C7000FFF774FF07E0019B93F838390093002B4E
:108C800041D000243C6095F96822002AC0F254814A
:108C9000D7ED007ABAF9A420B8EE677A1AB9BAF813
:108CA000A220AAF8A420BAF8A430DFEDA56A07EE46
:108CB000903AF8EEE77A67EEA67AB4EEE77AF1EE4C
:108CC00010FAACBF012100215046FFF71DFF95F9B6
:108CD0006822002A95F86922B8BF44F001045306BF
:108CE000019B93F8382948BF44F002040AB144F0CC
:108CF00008043A68214650460DB0BDEC088BBDE82B
:108D0000F04FFFF7C3BED5F874020268126D9047AA
:108D1000061ED5F87402026852690CBF00240424B0
:108D200090470AF5804B002800F0D180D5F89822B2
:108D300092F9A021002A05DB019B93F82929002A3A
:108D400000F0C5800AF5A052D2ED857A9FED7D7ABC
:108D5000F0EEE77AF4EEC77AF1EE10FA40F1B78060
:108D600044F400744E460AF5A04808F1380840461D
:108D70006CF0DCFF0130DBF8A40E9FED730ADFED31
:108D800073BADFED738A0CBF012302236C3008EE47
:108D9000103A28F06DF90CABCDED0A0A8DED0B1AE7
:108DA0008DED090A13E907000DF10C0E0DF1180CF9
:108DB0008CE807008EE80700704627F0A5FE0AF54C
:108DC0008042DFED647AD2F8A42E92ED36AA2AEE24
:108DD00027AAB4EEEB0AB3EE0EBAF1EE10FA0AF5DA
:108DE0009C40B4EECBAACCBF44F4A06444F48064AD
:108DF0005830F1EE10FAC8BF44F48074F0EE40AA87
:108E000054F082F928F032FDB8EEC88A0AF59D4088
:108E1000B4EEC80AF1EE10FA00F1080098BF44F071
:108E20008004F0EE409A84F0B1FF68EE288AB0EE3C
:108E3000C09AB4EEE89AF1EE10FA504648BF44F0FA
:108E400040040AF04BFB00285AD144F02004CB46E2
:108E500040466CF06BFF012862D144F01004CDF85D
:108E60000090002E64D0F4EEEBAAF1EE10FA5FDC75
:108E7000B4EECBAAF1EE10FA5ADCF4EEC89AF1EE99
:108E800010FA55D8B4EEE89AF1EE10FA50D5BBF1CD
:108E9000000F4DD0009B002B4AD03A68BAF9A410BD
:108EA00007EE902AB8EE677A19B9BAF8A210AAF8B4
:108EB000A410BAF8A43007EE903AF8EEE77AB4EED0
:108EC000E77AF1EE10FA31D501323A60DBE650462E
:108ED000FFF734FE10B1002E3FF445AFD5F89822CD
:108EE000D679002E3FF43FAFDBF8AC2ED2EDDB7A23
:108EF000F5EEC07AF1EE10FA3FF532AF002632E718
:108F00000AF53A5054F09EF8DFED137A90ED007AAE
:108F1000B4EEE77AF1EE10FA97D44FF0000B97E732
:108F200040466CF003FF01309BD196E701219EE69D
:108F30000022CAE70C46A6E60121C5E6C091002042
:108F4000CDCC4C3EDB0FC93F9F0CB3450080BB44EA
:108F50000000C842E02E65420000484310B500F50D
:108F6000BB52044607CA88B002AB83E807009FEDF6
:108F70001D7ADDED047A77EE877A9FED1B7ACDEDD1
:108F8000047AD4ED2B7AF0EEE77AF4EEC77A04F5A2
:108F90009C40F1EE10FA00F158000BD5B4F9A22074
:108FA00007EE902AF8EEE77AF7EE006A86EEA77AE7
:108FB00084ED2B7AD4F8AC200192194601AA54F022
:108FC00089F92046FFF722FE2046FEF785F9204664
:108FD000FEF75EFA2046FEF715F82046FEF7CCF8BD
:108FE00008B010BD0AE81C410000003410B504466A
:108FF0002DED028B1D205EF097FD58B304F5405314
:10900000D3F8740200F030FC192108EE100A04F5C0
:10901000736048F0ABFC022819D00338012807D848
:1090200004F53A5054F00EF890ED008ABDEEC88A6F
:10903000B8EEC88A9FED090A28EE000ABDEC028B43
:1090400004F5A0403830BDE810406CF0F5BE9FED4F
:10905000048AEDE7BDEC028B10BD00BF0AD7233CAC
:1090600000000000124A0260124A426002F17801D8
:10907000816001F52751C160043101610839416106
:10908000243981610C49C1610C49016202F56261B8
:10909000416202F6E411816202F6E811C16202F651
:1090A000EC1102F51F624263054A01638263704757
:1090B000C4070E08D050002068400020FC7A002031
:1090C000702D002017294BD8DFE801F0100C141880
:1090D000231F2B1C4A274A2F4A4A4A32364A3A4A09
:1090E0004A3E424700F5B2405C30704700F5C6404A
:1090F0000830704700F5B3401C30704700F5B340AE
:109100005830704700F5C040EEE700F5C3402C3002
:10911000704700F5C2402030704700F5C24064300F
:10912000704700F5C4407C30704700F5C140E3E76C
:1091300000F5B7403030704700F5C34068307047E5
:1091400000F5C6404430704700F5C7401430704702
:1091500000F50050D0F8200D704700F5C140CFE772
:109160000020704773B50B6805465B6C08460C46DB
:10917000164698470F4A00960346042105F54150CC
:1091800054F04CFD51F0A4FA236805461B682046B4
:1091900098470A210246284651F052F8064B93F8A8
:1091A00069329B0641BF054A137843F004031370EC
:1091B00002B070BD38F50D08585C00205C930020AB
:1091C00038B50C4A182305460C464FF081FA78B1A1
:1091D00021462846FFF776FF30B10146064A284669
:1091E000FFF7C0FF002038BD28464FF0B9F9F9E776
:1091F0000120F8E7B8F50D0858F50D0810B500F591
:109200000053002283F8142F094B044693F8681288
:1092100000F5804304F54054D3F8A40EC9097EF04C
:10922000BDFAD4F874020368BDE81040DB68184743
:10923000585C00202DE9F0410446086803685B692A
:109240000D461646984790B1306803685B699847A9
:1092500068B904F54053D3F8982292F8CB2032B184
:1092600093F96832002B02DB2046F9F7F5F829481C
:109270000AF05EFF286803689B68984704F5B247C8
:109280002B685C37BB4211D104F580430022D3F830
:10929000A40E03681146D3F88C30984704F5405368
:1092A0000021D3F8980203681B6F98472868036869
:1092B0005B69984790B9326804F5C64308339A420F
:1092C0001CD1B7EE001ADFED140A2520B0EE410ADA
:1092D00024F04EFC04F5B14383ED1E0A30680368A8
:1092E0001B6C9847014698B904F58044D4F8A40E45
:1092F0000368BDE8F041D3F8A03018479742EDD19C
:10930000DFED050A2520B7EE001AB0EE600ADFE7B0
:10931000BDE8F0819C9200200000000070B500F5CF
:1093200040550446D5F874020B4E0368DB69984734
:109330003074D5F8740203681B689847F070D5F84C
:10934000740203689B6C9847014604F59E50BDE883
:10935000704043F01BBA00BF3D9300202DE9F74356
:1093600000F5A04300F5405893F8584983F8582970
:109370000546D8F8740203681B680F4616469847DE
:10938000B84221D105F500531A2E83F8346409D16F
:1093900040B905F5804503F6FC53D5F8A42E1B68AB
:1093A000C2F8FC30784B93F869329D0604D401244E
:1093B000204603B0BDE8F083B442F8D0734A137876
:1093C00043F002031370F2E7022E0AD01B2F10D1D4
:1093D00005F5B3403146583003B0BDE8F04301F025
:1093E00099BC39462846FFF7EBFE04460028EDD12C
:1093F000DEE739462846FFF765FE0446019018B9B6
:1094000028464FF0ADF8D3E7D8F8983293F8CB3030
:1094100083F0010943B90198036849465B6898479E
:109420000446A8B95A4A0EE003685B6998470446A7
:10943000002840F09B80D8F8983293F8A031980724
:1094400000F19480534A01992846FFF78BFEAFE75D
:1094500005F5495101AA3431284605F50054FFF7B6
:10946000E9FE0198C8F8740284F8346403681B6844
:1094700098473246014605F58F5050F0F1FA002129
:1094800005F541505CF0C8F894F9263323B105F591
:109490000C50203069F0F6FAD8F8740203681B68A3
:1094A0009847C21E05F580435042504104F6CC5106
:1094B00083F8340FD3F8A42E0968C2F8F81004F624
:1094C000FC51D3F8A42E0968C2F8FC10012F01D07A
:1094D0000B2F06D104F6E454D3F8A43E2268C3F857
:1094E000FC202846FFF71AFF274B93F869329B06AA
:1094F0003FF564AF5BE705F5005393F82023002A9E
:1095000089D0B3F83C23D10785D593F85C23002A92
:1095100081D0D8F8982292F8CB20002A3FF47BAF74
:1095200093F834340A2B7FF476AF98F96832002B25
:10953000FFF671AF184A01992846FFF713FE002481
:1095400036E716480AF0F8F90028D4D1D8F87402A2
:1095500003685B6998470028CDD0019803685B6970
:10956000984704460028C6D10D4A6CE70198036865
:109570001B6998470028E4D008480AF0CBF9044654
:109580000028DED1074A5EE7585C00205C9300208B
:1095900022780F0880F50D08A5F50D08582C00203D
:1095A00093F50D087E250F080148FFF7D7BE00BFD1
:1095B000582C002070B52DED028B244B93F88D3282
:1095C000DB0782B006460D461446B0EE408AF0EE48
:1095D000608A06D500232B60236002B0BDEC028BAD
:1095E00070BD5CF005FF037F002BF3D0F36A9FEDA5
:1095F000181A1B689FED170AB3F9083007EE103AE6
:10960000B36A1B68B3F9083007EE903AB8EEC77A30
:10961000F8EEE77A67EE000A68EE811A27EE800A14
:1096200028EE011A01A9684625F096F9DFED0A6ACD
:109630009DED007ADDED017A27EE267A67EEA67AB7
:1096400085ED007AC4ED007AC7E700BF585C0020C2
:109650000AD7233C530469390000C84270B52DED88
:10966000028B88B0002302930393364B93F88D321C
:1096700013F0010F0646B0EE408A06AD02AC03D1EE
:109680005CF0B6FE037F5BB994E8030085E8030055
:109690009DED060ADDED070A08B0BDEC028B70BD3A
:1096A000B36ADFED296A1B68B3F9083007EE903A18
:1096B000F36A1B68B3F9083007EE103AB8EEC77AC0
:1096C000F8EEE77A27EE267A67EEA67AF1EE476A99
:1096D000CDED026ADFED1D6ACDED037AB0EEC77AFB
:1096E000B4EEE67AF1EE10FA06D5F0EEE77AF4EE93
:1096F000E67AF1EE10FAC7D403AA21461448F8F727
:10970000DBFEDDED027A9DED037AF0EEE77AB0EE56
:10971000C77AF4EE477AF1EE10FACCBFB0EE670AE2
:10972000B0EE470A204627F03DF904A88DED040A63
:10973000CDED050A27F0E8F9204688EE000A27F06B
:1097400061F9A1E7585C0020530469390000003436
:10975000582C0020094B93F96822002A0CDAB5EE48
:10976000C00AF1EE10FA07D9D3F8983293F8A100A5
:10977000C31E58425841704700207047585C002073
:10978000436A1B6893F8CB3043B1054B93F86802EA
:1097900000F0A000203818BF01207047012070475A
:1097A000585C002010B5436A04461868D1B1022104
:1097B00087F06CF9236A9FED0C1A18680368F0EEC5
:1097C000410ADB6AB0EE410A9847236A074A1868E3
:1097D000D2ED000A03689FED040A5B6EBDE81040FD
:1097E000002118470121E3E700000000D8500020C5
:1097F00010B5436A04461868002930D0022187F06A
:1098000045F9236A18687DF099FF636A1B6893F82D
:10981000A130012B04D8236A012118687EF028FDAD
:109820006369186881F0D8FC6369186881F034FDB9
:1098300063699FED0C0A186881F05AFF6369186824
:1098400081F0C8FF236A9FED071A18680368BDE816
:109850001040DB6AF0EE410AB0EE410A18470121E0
:10986000CDE700BF0000000013B5044601A90C4875
:1098700009F0C2FE10B1019802B010BD636918680A
:1098800080F0B4FB18B9074BD3F87C0EF4E7064818
:1098900001AA032112F0C6F80028F4D0EBE700BFBC
:1098A000582C0020586C0020D07A002070B5044657
:1098B0002DED028B00296AD18368B3F92E58642DEF
:1098C000B8BF6425FFF7D0FFA8426268A4BF324B3F
:1098D00093F86952B2F93430ACBFC5F38015012555
:1098E000002BDBBF63691B685B4293EDC48AC8BF72
:1098F00007EE903AB2F93230C8BFB8EEE78A002BD3
:10990000B8BF5B429BB25B4207EE903AA368F8EEA9
:10991000E77AB3F92E68F4EEC87AF1EE10FAD8BF00
:10992000B0EE678A2046642EB8BF6426FFF79CFF1E
:109930006369A26B1B68D2ED001A93EDC61AD3EDD2
:109940000E0A311A00EE101AB8EEC00A24F0F2FB2B
:109950006368B3F93230002BB8BF5B429BB25B4205
:1099600001EE103A40F29720B8EEC11AF0EE480A24
:1099700024F0FEF863692946186880F0DBFBBDEC33
:10998000028B6369BDE87040186881F023BF9FEDCA
:10999000030A0025EEE700BF585C0020000000002D
:1099A000436A186803681B691847000038B52DED35
:1099B000028B03680446D3F884309847236B2A4807
:1099C0001B68F0EE408AB3F9085009F027FD4FF408
:1099D0007A72041E4FF000012846D8BF4FF4FA7483
:1099E00024F004F98442B6EE000A2ADD07EE900A5C
:1099F000B8EEE77A07EE904A27EE007AF8EEE77ABB
:109A000087EE278A4FF46D7038EEC00AF5EE087ABB
:109A1000B1EE400A80EE270AB7EE001AFEEE000A09
:109A200024F0A6F8F7EE007A77EEC07A28EE000A66
:109A300020EE080A20EE080AA7EE880ABDEC028B89
:109A400038BD031B07EE103AC4F57A74B8EEC77A36
:109A500007EE904A27EE007AF8EEE77A87EE278A3B
:109A600038EE008ACEE700BF582C002013B504461C
:109A70008DED010A6CF0F2F86369A26B1B6892ED40
:109A8000001A93ED0E0AD3EDC60A01A96AF074FF1D
:109A90009DED010A02B010BD436A186803685B6A55
:109AA0001847000038B5436A1C6894F8CB10054687
:109AB00061B9204686F0EAFF6B6A1B6893F8A10043
:109AC00018B1012814BF0320022038BD16480378BE
:109AD0003BBBFFF73FFE20BB144A92F8683203F00D
:109AE000A003202B17D0B5EEC00AF1EE10FA10D566
:109AF00092F86A325B070CD40121204686F0C6FF3B
:109B00006B6A1B6893F8A130012B0CBF0220032065
:109B1000DBE70221F1E72046022186F0B7FF0420AF
:109B2000D3E70120D1E700BF9C920020585C0020C1
:109B300010B52DED028B134B93F88D32DB070446E5
:109B400004D59FED110ABDEC028B10BD5CF050FCFA
:109B5000037F002BF5D0636B18685CF073FDA3687E
:109B6000DFED0A7A03F5116292ED008A03F6141311
:109B7000D3ED000A28EE278A24F0A8FE28EE000A7A
:109B8000E1E700BF585C0020000000000000C84270
:109B90000148F8F7BBBC00BF582C00200148F9F77A
:109BA0000BB900BF582C00200148FFF7D7BB00BFFE
:109BB000582C002070B52DED028B7D4D95F8693243
:109BC0008CB00026044658060496059603D56369B2
:109BD000186880F07FF895F88D32D9075DD46368F6
:109BE0009B899A071BD5734853F02CFADFED727AE4
:109BF00090ED007AB4EEE77AF1EE10FA0FDD50F056
:109C000067FD3D2150F0FCFA6C4809220521FFF761
:109C1000A5FB20B9092202212046FFF7C5FF636892
:109C200093F95430CBB365489FED658AF9F7C4F8D2
:109C3000E3689FED647A1B68D3ED0A7AF4EEC87A84
:109C4000F1EE10FAB8BFF0EE477AB6EE000A27EE52
:109C5000800A2046FFF702FD8DED040AB0EEC00A2F
:109C6000B4EEC80AF1EE10FACDED050A06D5F0EE15
:109C7000E00AF4EEC80AF1EE10FA0ED495F86A3252
:109C80001B0704D450F024FD492150F0B9FA95F88F
:109C90006A3243F0080385F86A3295F86B326FF345
:109CA000820385F86B32606909960A9609AD2A46E7
:109CB00004A90068012380F077F86369186881F0CF
:109CC000EBFA6369186880F0C3FBA3688DED060AA0
:109CD000CDED070A8DED081AD3ED007AF5EEC07AC6
:109CE000F1EE10FA52DD384B9FED388AB3F9743437
:109CF00000EE903AF8EEE00A2046CDED030AFFF7B9
:109D0000B3FDA368DDED030AD3ED001A9FED2A0A27
:109D1000B7EE002A07EE900A31EE822AB8EEE71A73
:109D200022EE082A61EE881A23F062FEDFED287A1F
:109D300020EE270ADFED277A20EE270AB8F0C0FDD3
:109D4000DFED257A20EE270A06A820EE088A26F005
:109D5000DBFEB4EEC08AF1EE10FA17D5C8EE006A49
:109D600063699DED067ADDED077A27EE267A67EEC8
:109D7000A67A8DED067ACDED077A1B68D3F8882395
:109D8000C3F89423D3F88C23C3F89823236A134988
:109D90001C682846FCF7A8FE0B9B009395E80C0076
:109DA00006A920467DF07CFD0CB0BDEC028B70BD99
:109DB000585C0020C47A002000002F44582C00205A
:109DC0000000003400007A43584C00200000C842D4
:109DD0000AD7233C35FA8E3C0AE81C416C910020DE
:109DE00013B504460191FFF7E5FE0199204602B044
:109DF000BDE81040FFF75ABD0148FEF7AFBE00BFF7
:109E0000582C002000487047985C00200148F8F763
:109E10006BBB00BF582C002030B50F4D87B000231E
:109E200004466946D5F8AC0E00930193029380F086
:109E300027FBD5F8AC0E02A980F076FB009B0393BC
:109E4000019B04930222029B059303A9204612F072
:109E5000EBF8204607B030BD586C0020014B0122C2
:109E60001A707047C491002000207047002070478E
:109E70000020704700207047002070470020704786
:109E80000020704700207047002070470020704776
:109E9000002070479FED010A704700BF00000000DE
:109EA0000020704700207047002070470120704755
:109EB0000020704700207047012070470020704745
:109EC0000120704701207047002070470120704733
:109ED000012070470020704700487047D0730F087A
:109EE00000487047D0730F0890F83C3043B983683E
:109EF00093F82439DB0742BF034B0122C3F86C22DD
:109F0000002380F83C307047585C00202DE9F04376
:109F10002DED0C8BF0EE409A20EE000A97B0002554
:109F2000A0EEA00A04468946B0EE41CAF0EE60AA4F
:109F300090461F4601950295039504950595069553
:109F4000B8F00AFFF7EE00CAB4EEEC0AF1EE10FA30
:109F5000C8BFCCEE807AA36803F50E6203F6E40373
:109F600092ED009A9FEDC5DAD3ED000AC4BF69EE09
:109F7000A79A6AEEA7AAB0EE690A24F0A7FCA36824
:109F800029EE0D9A03F50E6203F6E403D2ED008A82
:109F9000D3ED000A29EE009AB0EE6A0A24F096FC8E
:109FA000A36868EE8D8A03F6F80203F6FC03D3ED8E
:109FB000000A92ED008A68EE808AB0EE4C0A24F026
:109FC00085FC636828EE0D8A93F9703028EE008ACC
:109FD000002B00F0D980236A9FEDA90A18686C3025
:109FE00027F046F8B0EE60AACDED080A8DED091A0B
:109FF0008DED070A23F066FDBDEEC0BAA14940F61B
:10A00000B8321BEE100A23F0E1FD434207EE903A0E
:10A010006368F8EEE77A93ED1A7A67EE877AB0EE26
:10A020004A0ACDED017A23F04DFDFDEEC0BA40F6AF
:10A03000B83294491BEE900A23F0C8FD424263688F
:10A04000039507EE902A93ED1B7A93F97030F8EEA2
:10A05000E77A022B67EE877ACDED027A6ED18A4BD2
:10A06000B3F974340AEE103AB8EECBBAB8EECAAA15
:10A07000236AB4EECABAF1EE10FA1A683DDDA3689D
:10A08000DFED820AA16B92ED051AD1ED001A03F5FE
:10A090000E6393ED007A27EE0D7A3AEE4B0AC7EE87
:10A0A000200A24F047F8DDED017A37EE800A8DEDC5
:10A0B000010AB8EEEB0A236AB4EECA0AF1EE10FA0E
:10A0C0001A6834DDA368A16B92ED061AD1ED001A6F
:10A0D00003F50E63D3ED000A20EE8DDADFED6B0A97
:10A0E0003AEE400ACDEE200A24F024F8DDED027AA3
:10A0F00037EE800A8DED020A20E0B1EE4A0AB4EE96
:10A10000C0BAF1EE10FAD4D5A368A16BDFED5F0AF7
:10A11000D1ED001A92ED051A03F50E6393ED007A66
:10A1200027EE0D7A30EE4B0AC7EE200AB9E7B1EE02
:10A130004AAAB4EECA0AF1EE10FAC3D4236AD3F8DD
:10A1400000C00CF184030FCB12AD85E80F000EAEFA
:10A150000AAD86E80F0085E80F0004AB01AA294686
:10A1600060467EF039F8636893F97030022B16D19F
:10A17000DDED047A39EE279ADDED057A78EEA78ACF
:10A18000DDED067A38EE278A89ED009AC8ED008A5F
:10A1900087ED008A17B0BDEC0C8BBDE8F083F0EEC4
:10A1A000E99AF0EEEAAAF4EEE9AAF1EE10FA48BF55
:10A1B0006D46CDED009ACDED0AAAD5ED007ADFED22
:10A1C000340AB0EECCCAF4EECC7AF1EE10FAD8BF75
:10A1D00035468DED0ECA95ED007ADFED2E7A87EECD
:10A1E000270AAD20B7EE001A3CEEC00A23F0C0FCEF
:10A1F000E369D3ED937A04A820EE270A26F038FF0E
:10A20000F0EEC07A8DED061AB0EEC91A31EE671A7B
:10A210008DED040AB0EEC11A39EE000ACDED050A43
:10A22000B520F1EE410A23F0A3FCB0EE409A9DED7B
:10A23000050AB0EEE81AF0EEC07A31EE671A38EE91
:10A24000800AB0EEC11AF1EE410ABA2023F090FC68
:10A25000F0EE408A9DED060AB0EEC81AF0EEC07A24
:10A2600031EE671A38EE000AB0EEC11ABF20F1EEE7
:10A27000410A23F07DFCB0EE408A85E70000C84229
:10A280009F0CB34548F4FFFF584C002000007A446F
:10A290000000000000A08C45836893ED040AB5EE31
:10A2A000C00AF1EE10FA01DCFFF77ABB704700003C
:10A2B00073B5036A1D682B68D3F88C60436A044643
:10A2C000186803689B6E9847636A01901868036872
:10A2D0009B6F9847019902462846B047636A186801
:10A2E000036801211B6F9847044B93F8F62801205F
:10A2F0006FF3000283F8F62802B070BD587C00208E
:10A300002DE9F0412DED048B96B000241E46036A22
:10A3100001940294039404940594069405461868E5
:10A32000F0EE408A6C309FED2E0A88461746B0EE5C
:10A33000609A26F09DFEEB698DED070AD3ED7E7ADB
:10A34000CDED080AF8EEE77AB0EE608A30EE670AE3
:10A350008DED091A23F0B6FBEB6920EE490A8DED6D
:10A36000010A93ED7F0AB8EEC00A38EE400A23F0E6
:10A37000A9FB20EE680A2B6A03948DED020AD3F83C
:10A3800000C00CF184030FCB12AD85E80F000EACBA
:10A390000AAD84E80F0085E80F0004AB01AA294646
:10A3A00060467DF019FFD8ED007A9DED047A77EED6
:10A3B000877A9DED057AC8ED007AD7ED007A77EEC1
:10A3C000877A9DED067AC7ED007AD6ED007A77EEB2
:10A3D000877AC6ED007A16B0BDEC048BBDE8F0813B
:10A3E0009F0CB34530B52DED028B436A04461868C7
:10A3F00090F8CB1087B0002940F0858086F046FBAE
:10A40000636A186890F8A150012D7ED0032D00F0EA
:10A410009F8045B9236A294618687EF083FC236A29
:10A4200018687DF075F9636A186803689B6E984731
:10A43000A36A002840F0998018685CF003F9E36A89
:10A440001868B0EE408A5CF0FDF8636B8DED010A90
:10A4500018685CF0F7F805ABB0EE401A04AADDED21
:10A46000010A03A9B0EE480A2046FFF74FFD6368D2
:10A4700093F9702092B9534A92F96822002AB3BF27
:10A48000F0EE080AD3ED1A0A93ED1B0AB0EE600A4B
:10A4900005AB04AA03A92046FFF732FF636A1868D8
:10A4A00003689B6F984748B1636B18685CF080F84D
:10A4B00007EE900AF8EEE77ACDED057A236AA268F6
:10A4C000186892F8242903689DED030ADDED040A5B
:10A4D0009DED051A92074CBFDB6B9B6B9847236B76
:10A4E00039481B68B3F9081081F0D4FA236A62680E
:10A4F0001868D2ED020A036800215B6E984707B026
:10A50000BDEC028B30BD022178E70368DB6B984716
:10A5100068B92C4B93F96832002B84DA636A012105
:10A52000186883F0DFFE00287FF47DAF06E0636AE1
:10A530002946186883F0D6FE0028EAD0236A002155
:10A5400018687EF0EFFB236A18687DF0F7F86AE779
:10A550001C4B93F96832002BBFF665AF012183F0E5
:10A56000C1FE00287FF45FAFEDE718685CF020F8CB
:10A57000E36A07EE900A1868B8EEE78A5CF018F80C
:10A58000636A07EE900A186803689B6FF8EEE78A23
:10A59000984788B1636B18685CF00AF807EE900A78
:10A5A000B8EEE71A236A18680368F0EE680AD3F871
:10A5B0009C30B0EE480A91E72046FFF7B9FAB0EEBA
:10A5C000401AEFE7585C00204C85002070470000DF
:10A5D000002070470120704702207047002070471C
:10A5E00000207047012070470020704781F0010073
:10A5F000704700000120704701207047012070471C
:10A600000048704764F60D080048704770F60D0862
:10A6100038B54369044618687FF00AFE18B96369C3
:10A62000186880F089FF636920461D68FFF7EEFB1C
:10A630006368B3F93820B3F9363000EE903A4342FC
:10A6400001EE102A00EE103AB8EEC11AF8EEE00A58
:10A65000B8EEC00A28467FF0D7FC636920461D6823
:10A66000FFF7D4FB6368B3F93820B3F9363000EE56
:10A67000903A434201EE102A00EE103A2846B8EE16
:10A68000C11AF8EEE00AB8EEC00A7FF037FD0120EB
:10A6900038BD000030B52DED028B0446436985B00E
:10A6A0001D68FFF7B3FB6368B3F93820B3F93630A0
:10A6B00000EE903A434201EE102A00EE103AB8EE56
:10A6C000C11AF8EEE00AB8EEC00A28465B4D7FF0EA
:10A6D0009BFC2046FFF762FAB5F9743408EE103A95
:10A6E000236A186803689B6E9847B8EEC88AF0EE34
:10A6F000400A02AA01A9B0EE480A2046FEF75AFF16
:10A700002046FFF715FA236B1B68B3F90830F0EE0B
:10A71000408A00EE103A2046B8EEC00AFFF738FA39
:10A720002046B0EE408A8DED030AFFF76FFB6368A9
:10A73000B3F9363001EE103A434200EE903AB8EEEB
:10A74000C11AF8EEE00A2B20B0EE480A23F010FA06
:10A7500020468DED030AFFF7A5F9042813D8DFE89A
:10A7600000F0032F252A4B00236A18687CF0D0FFE5
:10A77000236A002118687DF07BFD63699FED300A34
:10A78000186880F0B5FF236ADDED020A18689DEDB8
:10A79000010A0368B0EE681ADB6A984763691868B3
:10A7A00081F018F805B0BDEC028B30BD236A0121A1
:10A7B00018687DF05DFD236A18687CF0BFFFDCE758
:10A7C000204D2B7863B963689FED1F1ADFED1C0ADB
:10A7D00093ED040A452023F0CBF9284609F090FCBC
:10A7E00020469DED030AFFF741F916488DED030A57
:10A7F00003A909F0BFFCC6E7636A0221186886F066
:10A8000045F9B5F97434114800EE103A02AA01A9CD
:10A81000B8EEC00A69F0E0FD20469DED030AFFF79F
:10A8200025F90B488DED030A08F004FF63699DEDDF
:10A83000030A18687FF06EFCA5E700BF584C0020A3
:10A84000000000009C92002000007A44207C002040
:10A85000605B00200020704790F8B931002B14BFD6
:10A860001B20032070470000002070470120704724
:10A8700090F89001062804D0A0F10A0358425841EC
:10A880007047012070470000012070470120704789
:10A890000120704790F8B901034A044B002814BF07
:10A8A00010461846704700BF0CF70D08CA390F084C
:10A8B00090F8B901034A044B002814BF104618460B
:10A8C000704700BF18F70D08CA390F0890F89001BB
:10A8D0000B3818BF0120704790F8B9312BB9044BE1
:10A8E000D3F8180E00F0010070470020704700BF39
:10A8F000584C002090F8903123B9034B187880F021
:10A9000001007047002070478092002038B590F811
:10A910009041012C054601D0002038BDC36818685D
:10A9200003681B6998470028F6D1EB681B6820462E
:10A9300083F8B848F1E70000C3681B68002283F879
:10A94000B82801207047000070B52DED028B002360
:10A9500080F8B931B0F87030012B84B004460D4650
:10A9600001D8002946D0636A254E1B6893F8CB3086
:10A9700073BB2448072384F890310368022B02D16B
:10A980000021FBF7BBFE9FED208AE368F0EE480A4A
:10A990001868B0EE481AF0EE481AB0EE480A0125E1
:10A9A00082F01AFC84ED738A84ED748A84ED758AD2
:10A9B00084F8B85104F59A7027F042F8134804F06F
:10A9C000D5FD96F86A326FF3C30386F86A3211E058
:10A9D00096F96832002BCCDA04F13C0029F020F91A
:10A9E00005460028C5D12046FFF70CFA084A022187
:10A9F00053F014F9284604B0BDEC028B70BD00BFC3
:10AA0000585C00206C91002000000000788D002030
:10AA100020F70D0810B50446094890F8183A012BA4
:10AA200003D100F6142027F073F8064890F8BD1FF4
:10AA300000F644705EF084F9002384F8B93110BD4B
:10AA4000587C0020586C002010B52DED028B094B6E
:10AA50000446D3F8B00EB0EE408A81F033FF9FED8C
:10AA6000060A28EE008A012084ED748ABDEC028B70
:10AA700010BD00BF586C00200AD7233C10B52DED47
:10AA8000028B094B0446D3F8B00EB0EE408A81F039
:10AA900029FF9FED060A28EE008A012084ED758AC1
:10AAA000BDEC028B10BD00BF586C00200AD7233CC0
:10AAB00010B52DED028B094B0446D3F8B00EB0EE65
:10AAC000408A81F01DFF9FED060A28EE008A0120D2
:10AAD00084ED738ABDEC028B10BD00BF586C002062
:10AAE0000AD7233CC3681B6818697FF0E3BD0000E8
:10AAF00038B5D0F8943104460D461BB98CF0DAFF16
:10AB0000C4F894018CF0D6FFD4F89431C01A4FF4F5
:10AB10007A73B0FBF3F0B4F89231984209D320462F
:10AB2000FFF770F92B88044A062153F077F80120CB
:10AB300038BD0020FCE700BF3CF70D0890F89031CD
:10AB4000052B05D1054BD3F8B83ED8687FF02ABD58
:10AB5000C36818680368DB68184700BF586C00209A
:10AB600008B590F89031052B0BD1094BD3F8B83EBE
:10AB7000D868243025F0C8FFBCEEC00A10EE100AD9
:10AB800008BDC368186803689B689847F4E700BF6E
:10AB9000586C002090F890318B4206D00B2B80F837
:10ABA000901102D10148FCF7D3BE7047582C002009
:10ABB00073B501231E4E80F87530D6F87432834287
:10ABC00005460A4614D1012485F8B941D6F8740225
:10ABD000019203681B689847019A014615484EF098
:10ABE0003FFF96F869329A061BD4204602B070BD2A
:10ABF00001910321FEF7D8FF019A04460028E2D113
:10AC000085F875004FF064FD1B220A214FF018FBF8
:10AC100096F869329B06E8D5074A137843F0040397
:10AC200003E0054A137843F002031370DDE700BF29
:10AC3000585C0020383E00205C93002030B585B081
:10AC400004460D4601466846FFF7E6F8694604F1FA
:10AC50003C0029F097FDC8B94FF03AFD1B220A21AC
:10AC60004FF0EEFA0D4B93F869329B0604D50C4A6F
:10AC7000137843F0040313702046FFF7C3F8094A22
:10AC8000042152F0CBFF002005B030BD29462046FC
:10AC900005B0BDE83040FFF78BBF00BF585C002017
:10ACA0005C93002050F70D0830B585B004460D4682
:10ACB00001466846FFF7B0F8694604F13C0029F008
:10ACC00085FDC8B94FF004FD1B220A214FF0B8FAE8
:10ACD0000D4B93F869329B0604D50C4A137843F068
:10ACE000040313702046FFF78DF8094A042152F03F
:10ACF00095FF002005B030BD2946204605B0BDE8CF
:10AD00003040FFF755BF00BF585C00205C93002027
:10AD10008CF70D087FB505460E4605F13C0401464B
:10AD20006846FFF779F86946204629F04FFDC0B91B
:10AD30002046694629F026FD044690B94FF0C8FC2C
:10AD40001B220A214FF07CFA0D4B93F869329B06C7
:10AD50000FD42846FFF756F80A4A042152F05EFF46
:10AD600004E031462846FFF723FF0446204604B09E
:10AD700070BD054A137843F004031370E9E700BF80
:10AD8000585C0020C4F70D085C93002030B50446E1
:10AD900085B00F4808F0BEFD0546B0B1072384F822
:10ADA00090310023019302930393E36801A918688B
:10ADB00081F022FDE3681868036801A95B6800223E
:10ADC000984704480021FBF799FC284605B030BDA0
:10ADD000582C00206C910020F0B5424FD7F8842EFB
:10ADE000D7F8803E2DED028B1343D7F87C2E13430A
:10ADF00087B005460C460CD14DF020FE40F275128E
:10AE00004FF4801107B0BDEC028BBDE8F0404DF06F
:10AE1000CDBD806982F0AEFF2046B0EE408A10F0D2
:10AE2000F5FD03283AD1EB6801A9186881F0C0FD4F
:10AE3000064698B3DDED017A6368009338EE678AC1
:10AE4000294BDFED2A7A93F968329FED290A2948C8
:10AE5000002BA8BFB0EE670A38EE008A009BBDEE5B
:10AE6000C88A002118EE102A9342ACBF00930092CA
:10AE7000FBF744FC6B69186880F05EFBDDED007A3F
:10AE80001D48B8EEE70A314609F0F4FB00212846D8
:10AE9000FFF780FE07B0BDEC028BF0BD94E80F0019
:10AEA00002AE86E80F00D7F8803E04936A46D7F8D2
:10AEB000843E05930221304610F0B4FD78B94FF07E
:10AEC00007FC022215214FF0BBF9DDED037AF8EE05
:10AED000E77A77EE887AFDEEE77ACDED007A002604
:10AEE000AEE700BF586C0020585C00200000000056
:10AEF0000000C8426C9100208092002030B52DEDFA
:10AF0000028BC36887B0044618680D4681F044FD83
:10AF100000284BD194F890210023009301930293D1
:10AF20006AB93148039303A90493059309F0D4FB4C
:10AF300028B1039B0093049B0193059B029394ED1E
:10AF4000730A9FED2A8AE368DDED000A9DED011A80
:10AF5000DDED021A1868B4EEC80AF1EE10FAAABFC5
:10AF6000DFED237A9FED230A20EE270A82F034F9E1
:10AF7000D4ED747AF4EEC87AF1EE10FA07DBE368E8
:10AF80009FED1B0A186827EE800A81F09BFCD4ED28
:10AF9000757AF4EEC87AF1EE10FA07DBE3689FEDFC
:10AFA000140A186827EE800A81F09CFCE3682946A1
:10AFB000186882F039F8054688B10F4B1B68022BE0
:10AFC00009D0032B03D10D4B93F9A5341BB10A48CB
:10AFD0000021FBF7B3FB01212046FFF7DBFD2846EC
:10AFE00007B0BDEC028B30BD809200200000003421
:10AFF0000000C842000000006C910020584C002066
:10B0000010B52DED028BC368DFED348A1B684269F1
:10B01000D3ED0A0A9FED328A93ED060AF4EEE80AB0
:10B020000446F1EE10FA1068B8BFF0EE480A7EF060
:10B03000D1FDE36862691B681068D3ED0A0A93EDDD
:10B04000060AF4EEE80AF1EE10FAB8BFF0EE480A8C
:10B050007EF038FE636918687EF0C8FF18B963692E
:10B06000186880F003F8E36862691B68106893ED64
:10B07000080A93ED0C1AD3ED070AB0EEC00A7EF071
:10B08000C3FFE36862691B68106893ED080A93EDDB
:10B090000C1AD3ED070AB0EEC00A7FF02FF86369EF
:10B0A00018687FF0C5F818B96369186880F044FA29
:10B0B00000210C48FBF722FB0B486AF055FF0B4AB6
:10B0C000B2F86A3223F48163A2F86A32BDEC028BD3
:10B0D00020460221BDE81040FFF75CBD00000034AF
:10B0E00000007A436C910020907C0020585C002086
:10B0F00010B50C4B0446D3F8B80E90ED0B0A90F83F
:10B10000502000F11C0181F07DF807480368022BF4
:10B1100002D00821FBF7F2FA20460521BDE81040D5
:10B12000FFF738BD586C00206C910020F0B52DED74
:10B13000028B4A4DDFED4A8AB0EE408A8FB004465A
:10B14000D5F8B80E0E46174680F0D2FEF0EEC87A5B
:10B15000F4EEE87AF1EE10FA07D49FED420AD5F842
:10B16000B80E28EE000A80F029FFD5F8B80E90ED51
:10B170000B0AB0EEC00A0FB1B1EE400A80F00EFF2C
:10B180000023D5F8B80E079302AA07A908930993DC
:10B1900080F030FFDFED347A9DED027AB4EEE77A8D
:10B1A000F1EE10FA56DD022207A90AA810F03CFFC2
:10B1B00071680191304610F029FC019902460AA8F5
:10B1C00010F0FAFBE3680AA9186881F02DFF10B9A6
:10B1D0002648FCF703FEA06982F0CAFD02684368B6
:10B1E000D5F8B80E049303A91C30039225F0BEFBDA
:10B1F00005A88DED050ACDED060A25F085FC1C4B52
:10B200001B68022B1BD0D5F8B83E1948D3ED0A7A3B
:10B21000F4EEE87AF1EE10FAB8BFD3ED047AF4EE6A
:10B22000C07AF1EE10FA4FF0000110D5DFED117A7F
:10B23000B4EEE70AF1EE10FA09DDFBF77FFA04211C
:10B240002046FFF7A7FC0FB0BDEC028BF0BDFBF76B
:10B2500055FAF4E72046FFF74BFFF4E7586C00205F
:10B26000000000340000C84200009643582C002023
:10B270006C9100200000FA4370B52DED028B294B34
:10B28000DFED298AD3F8B04ED3F8AC5ED4ED0A0ACC
:10B290009FED268A94ED060AF4EEE80AF1EE10FA24
:10B2A000B8BFF0EE480A064628467EF093FCD4ED7F
:10B2B0000A0A94ED060AF4EEE80AF1EE10FAB8BFB5
:10B2C000F0EE480A28467EF0FDFC28467EF08EFE11
:10B2D00010B928467FF0CAFE94ED080A94ED0C1AC6
:10B2E000D4ED070AB0EEC00A28467EF08DFE94ED3C
:10B2F000080A94ED0C1AD4ED070A2846B0EEC00AED
:10B300007EF0FCFE28467EF093FF10B9284680F0C0
:10B3100013F907480021FBF7F1F9BDEC028B01237B
:10B32000337070BD586C00200000003400007A4378
:10B330006C91002008B50748D0F8183E9B0704D54B
:10B340000121A0F50050F6F745FFBDE8084002488E
:10B3500008F0F0BF584C00208092002030B589B032
:10B360000446FEF70DFA30B10021204609B0BDE8D1
:10B370003040FEF73DBA636A0221186885F086FB0B
:10B38000E368186803685B69984701461048FCF752
:10B3900027FC6369186880F01DFA236A1D686369D9
:10B3A00018687FF055F805AC20460A498DED020A71
:10B3B000CDED030A8DED041AFBF796FB079B009376
:10B3C00094E80C0002A928467CF06AFA09B030BD66
:10B3D000582C00206C91002038B50446FEF7D0F9B7
:10B3E000054628B120460021BDE83840FEF700BAE6
:10B3F000636A0221186885F049FB29462046BDE8AA
:10B400003840FEF7EDBC00000148002106F0BCBB4F
:10B41000D48E002030B5174D9FED170A05F58043F7
:10B4200089B00446D3F8B80E80F086FF014628465E
:10B43000FCF7D6FB6369186880F0CCF9236A1D68B5
:10B44000636918687FF004F805AC20460B498DED60
:10B45000020ACDED030A8DED041AFBF745FB079BAD
:10B46000009394E80C0002A928467CF019FA09B070
:10B4700030BD00BF582C0020000000006C9100205F
:10B4800030B589B00446FEF77BF930B10021204683
:10B4900009B0BDE83040FEF7ABB9636A0221186815
:10B4A00085F0F4FAE368186803685B699847014619
:10B4B0001048FCF795FB6369186880F08BF9236AE4
:10B4C0001D68636918687EF0C3FF05AC20460A4911
:10B4D0008DED020ACDED030A8DED041AFBF704FB96
:10B4E000079B009394E80C0002A928467CF0D8F949
:10B4F00009B030BD582C00206C91002030B52DEDE6
:10B50000028B83B00446FEF73BF920B9636A1B68DF
:10B5100093F8CC3043B90021204603B0BDEC028B38
:10B52000BDE83040FEF764B994F89831DA071DD4CD
:10B53000E3681D682B6828469B689847D5ED097A13
:10B5400094F89831B4EEE70AF1EE10FA4CBF0122FC
:10B55000002262F3000384F8983107D4204603B038
:10B56000BDEC028BBDE83040FFF7F8BE94F898318F
:10B570009B0734D4E368DFED458A1B686269D3ED2D
:10B580000A0A9FED438A93ED060A1068F4EEE80A72
:10B59000F1EE10FAB8BFF0EE480A7EF01BFBE3684C
:10B5A00062691B681068D3ED0A0A93ED060AF4EE8F
:10B5B000E80AF1EE10FAB8BFF0EE480A7EF082FB1E
:10B5C000636918687EF012FD18B9636918687FF026
:10B5D0004DFD94F8983143F0020384F898312D4BD7
:10B5E000D4F8A021D3F87C3E9B1A07EE903AB8EE2F
:10B5F000E78AF1EE047AB0EEC87AB4EEE77AF1EEBB
:10B6000010FA38D594F8983143F0040384F898314F
:10B61000204684ED678AFEF7CDFA6369A26B1B684A
:10B62000D2ED001A93EDC61AD3ED0E0AB1EE480A18
:10B6300022F080FD63691B6840F2AA4093EDC31AB3
:10B64000D3EDC40A22F094FA2046FEF70FFA12480E
:10B650008DED010A07F0EEFF63699DED010A1868A0
:10B660007EF058FD6369186803B0BDEC028BBDE83D
:10B67000304080F0AFB8D4ED677A68EE277AF5EE07
:10B68000C07AF1EE10FAC3D5BCE700BF0000003469
:10B6900000007A43586C0020605B002030B52DED2F
:10B6A000028B83B00446FEF76BF820B9636A1B680F
:10B6B00093F8CC3043B90021204603B0BDEC028B97
:10B6C000BDE83040FEF794B86369DFED347A1B685B
:10B6D00094ED710A93EDC31AD3EDC40A20EE270A44
:10B6E00040F2C44022F044FA2046FEF7BFF9236A34
:10B6F000186803689B6EB0EE408A9847284BB3F9F0
:10B70000743407EE903AB4F8BC316425F8EEE77A69
:10B7100013FB05F3B4EEE70A07EE103A94F9BE31D5
:10B72000F1EE10FAD8BFF0EE407A13FB05F39FED6F
:10B730001D0AF8EEC76A07EE103AF4EE407AB8EE4A
:10B74000C77AF1EE10FA58BFB0EE670A6846CDED41
:10B75000006A8DED017A25F029FA236ADDED010AF0
:10B760001868B4F8C03102689DED000A126B13FB33
:10B7700005F301EE103A0121B8EEC11A9047636952
:10B78000B0EE480A18687EF0C5FC6369186880F05E
:10B7900021F803B0BDEC028B30BD00BF0000C842F1
:10B7A000584C002000007A442DE9F0432DED028B27
:10B7B000B64F85B00446D7F87402FDF7E1FF48B1F3
:10B7C000D7F87402002105B0BDEC028BBDE8F04350
:10B7D000FEF70EB807F58056D7F89802022185F0DB
:10B7E00055F9D6F8A43E93ED378A8CF063F9B7F893
:10B7F000683203F4814305467BB1D6F8AC0E7EF087
:10B8000069FA2378022B08D159F0E8F8A04BA14A35
:10B81000062152F003FA0323237066F0C7F866F09E
:10B82000B1F848B166F0C2F866F0B6F820B12378F6
:10B83000012B10D9022B1DD02378082B00F2858113
:10B84000DFE813F02100390063000A013E014501E1
:10B850005A015C012A0059F0C1F88D4B8E4A06212D
:10B8600052F0DCF9D6F8AC3ED3F8543363610823C8
:10B870002370E1E759F0B2F8854B884A062152F06F
:10B88000CDF90323F4E7D6F8B00E03681B69984797
:10B8900010B12046FFF7F0FC2378082B00F27381EB
:10B8A000DFE813F05C01640164017A017A017A0136
:10B8B0007A0182018201A560D6F8AC3E9FED787ACC
:10B8C000D3F854336361774B03F65462D2ED007AB8
:10B8D000F4EEC77AF1EE10FA4EDB9FED737A67EE65
:10B8E000877AD6F8B03E93ED087AB0EEC77AF4EED8
:10B8F000477A4FF07E53F1EE10FA48BFB0EE677A08
:10B900002361022384ED067A2370D4ED016A9FED52
:10B91000647AD6F8AC3EF0EEE67AF4EEC77AF1EE51
:10B9200010FA0AD4D4ED057A93EDD56A77EEC67A8B
:10B93000F4EEE76AF1EE10FA29D4DFED5C6AD4ED9B
:10B94000067A67EEA67AD3EDDB6AF4EEE76AF1EEEB
:10B9500010FA26DCA368D4ED047AEB1AB3F5FA6F7B
:10B9600021D2B4EE678AF1EE10FAC8BFB0EE678A52
:10B9700084ED048AE5608FE7B3F9AA34002BB8BFE1
:10B980005B429BB207EE903AF8EEE77AA9E706230E
:10B99000237059F023F83E4B454A042152F03EF9FA
:10B9A0007AE7A56078E7DFF8FC8008F64863D3ED16
:10B9B000006A67EEA67AF4EEC87AF1EE10FAD9D4EE
:10B9C00008F64C69D9ED007AF4EEC77AF1EE10FA78
:10B9D00022DB98F8783E33B90623237058F0FEFF37
:10B9E0002B4B344AD9E7A8F5005007F077FD98B102
:10B9F00098F98E3E83B9B8F97A3ED9ED007ADFED39
:10BA00002A6A07EE103A67EEA67AB8EEC77AB4EE65
:10BA1000E77AF1EE10FAADDCE068281AB0F5FA7FAB
:10BA20007FF63AAF0323237008F6486858F0D6FF34
:10BA300098ED007AD4ED047A67EE277A054617EE82
:10BA4000900AF4F769FD124B1B4ACDE9000106216B
:10BA5000284652F0E3F81FE7D6F8AC0E7FF0E8FD79
:10BA600065F0A4FF65F08EFF68B158F0B7FF084B92
:10BA7000124A062152F0D2F865F098FF65F070FF87
:10BA80000423237008E70523FBE700BF585C002070
:10BA900010F80D081EF80D0828F80D083FF80D08DD
:10BAA00000000034584C00200000C842333373BFFC
:10BAB00051F80D086CF80D089CF80D08C4F80D0835
:10BAC00065F074FF65F05EFFC0BB05232370404B3B
:10BAD000E068DFED407AD3ED006A9FED3F7A2D1AE2
:10BAE000A6EEA77A07EE905AF8EE677AF4EEC77AD8
:10BAF000F1EE10FA3FF5D0AE07232370D6F8AC3E36
:10BB00009FED367AD3EDC37AD3EDC66A67EE877AB6
:10BB1000B6EE007A67EEA77A67EE877A87EEA67AA6
:10BB2000D4ED057A77EEC77A93EDD57AF4EEC77A3D
:10BB3000F1EE10FA3FF6B0AE0823A2E765F036FF4B
:10BB400065F02AFF0028C0D1A6E64CF077FF40F24E
:10BB50009C524FF480114CF029FF9DE6204805B01F
:10BB6000BDEC028BBDE8F043FFF7F8BBD7F87402D9
:10BB7000FEF720F894ED060A0121B1EE400AD6F84E
:10BB8000AC0E7EF0D7FAD6F8AC0E05B0BDEC028B49
:10BB9000BDE8F0437FF01EBED7F87402FEF70AF846
:10BBA0009FED100A0021EAE79FED0E8AD7F8740294
:10BBB0008DED038AFDF7FEFFD6F8AC0E0123B0EE43
:10BBC000480A03AA04F114017FF0BAF8DBE700BFCA
:10BBD000A85A002000007A440000FA43CDCCCC3DA6
:10BBE000308600200000000030B590F8B83185B0F4
:10BBF0000446F3B168460FF0D9FE424869460AF0A0
:10BC000093FC50B104F13C0028F0A8FD002384F817
:10BC1000B83104F59A7025F013FF94F890310B2B8E
:10BC20002DD8DFE803F0294C50544C582C5C60644C
:10BC30002C6800F59A7025F003FF04F13C0590B1E3
:10BC400094F84030012B0ED194F89031012B0AD199
:10BC5000284628F0F1FB50B12046FEF7D3F82A4AD7
:10BC6000022151F0DBFF284628F014FCD5E72046DE
:10BC7000FEF7C8F8254AF3E72046FFF75BFB94F888
:10BC800044303BB994F8463023B994F840309A1EBA
:10BC90005342534194F8B9218AB383BB84F8B93134
:10BCA0001B4CD4F8740203681B6898472D22014688
:10BCB000A4F5F15005B0BDE830404DF0D1BE2046AE
:10BCC000FFF74CFBDBE72046FFF786FBD7E7204674
:10BCD000FFF79AFBD3E72046FFF79CFBCFE7204610
:10BCE000FFF7CEFBCBE72046FFF708FCC7E7094884
:10BCF000FFF75AFDC3E72046FFF7D0FCBFE705B0CA
:10BD000030BD00BF68400020E0F80D0808F90D08BC
:10BD1000585C0020C49100202DE9F0412DED028BEC
:10BD2000074684B008460E460FF070FE0328804692
:10BD30006D4628D1FB68186880F08CFC012822D160
:10BD40002148294607F058FC0446B0B17B69DDED77
:10BD5000007A1B68F8EEE77A93EDF27A77EEC77A0D
:10BD60004246FDEEE77A17EE901AC829CDED007A2B
:10BD7000B8BFC82130460FF01FFE204604B0BDEC0E
:10BD8000028BBDE8F081114B0FCB85E80F003046E8
:10BD90000FF03CFE014628460FF0D2FE0446002874
:10BDA000EBD07B69DDED017A1B68B8EEE78AD3ED55
:10BDB000F27A284638EE678A0FF028FEBDEEC88A70
:10BDC000024618EE101AD5E7582C0020D07A002031
:10BDD00010B543699FED126A1B68D3EDF06A93EDCD
:10BDE000F17AD3EDF27A86B066EE866A27EE067AAD
:10BDF00067EEC67A68460C46CDED006A8DED017A95
:10BE0000CDED027A25F0F8F803A920468DED030A5E
:10BE1000CDED040A8DED051A10F05AF906B010BDEB
:10BE20000AD7233C30B5083204461D460FCA84E8C1
:10BE30000F00134301BFAB68A360EB68E360636866
:10BE400085B093B920460FF0E1FD03AA01462846CC
:10BE50000FF0E8FD60B10399019120460FF0D6FD87
:10BE60000199024620460FF0A7FD204605B030BDDF
:10BE7000696801912846F1E730B50B6985B0044641
:10BE80000BB94B6953B30023C4F8B43108310FC95F
:10BE90006D4685E80F0029462046FFF73DFF98B91B
:10BEA000124B0122D3F87C1E28460FF085FD4EF080
:10BEB0000FFC022215214EF0C3F92046FDF7A2FF28
:10BEC0000B4A022151F0AAFE29462046FFF716F838
:10BED00010B90848FBF782FF05B030BD0123C0F858
:10BEE000B43105B0BDE83040FFF78AB8586C002087
:10BEF0003CF90D08582C002070B51A4B04460E462C
:10BF00000FCB88B06D4685E80F0020462946FFF725
:10BF10005FFFE368186880F03FFD98B1E368186838
:10BF200003681B69984768B1E3682946186880F080
:10BF3000A5FB38B94CF082FD40F295624FF48011B8
:10BF40004CF034FD214604A82B463246FFF76AFF29
:10BF500004A92046FEF7D2FF10B90348FBF73EFFC5
:10BF600008B070BDD07A0020582C002070B5154B59
:10BF70000C4606460FCB88B06D4685E80F00294673
:10BF80003046FFF725FF2B462246314604A8FFF72F
:10BF900049FF6288A388122A4FEA132305D1227E23
:10BFA000D20744BF03EB83035B00227A07EE903A8B
:10BFB000C2F34002B8EE670A04A93046FFF7B6F8AC
:10BFC00008B070BDD07A002038B504460D46FFF7A2
:10BFD00093FF0023C4F89431AB88A4F8923138BDA4
:10BFE0007FB50D460446FFF787FF05F108010FC92D
:10BFF0006E4686E80F00134306D1234BD3F8802EFC
:10C00000D3F8843E0292039304F5D07201213046A6
:10C010000FF008FD94F8983170B923F0050343F050
:10C02000050384F898312046FDF7ECFE174A0621F7
:10C0300051F0F4FD04B070BD23F0070384F898318B
:10C040000023C4F89C31E36862691B68106893EDB3
:10C05000080A93ED0C1AD3ED070AB0EEC00A7DF082
:10C06000D3FFE36862691B68106893ED080A93EDDB
:10C070000C1AD3ED070AB0EEC00A7EF03FF8082193
:10C080002046FEF787FDD5E7586C002068F90D08BB
:10C090002DE9F0438DB06D4688461C460746134691
:10C0A0000A4601462846DDE91469FFF7BBFE95E81C
:10C0B0000F0084E80F0007A80FF078FCB8F80430F0
:10C0C000F3B9B8F80010013105AA89B207F13C00B4
:10C0D00027F05EFDA0B1234605AA39462846FFF7A2
:10C0E000A1FE95E80F0086E80F00BDF81630A3F119
:10C0F00052025342534189F800300DB0BDE8F0833D
:10C1000094E80F0086E80F000023F4E770B58B88F1
:10C1100092B004460D461646002B47D10DA80FF0ED
:10C1200045FC298801310BAA89B204F13C0027F0B3
:10C130002FFD00283AD0BDF82E1052291CD019D856
:10C14000112913D80F2913D933462A46214603A8AB
:10C15000FFF768FE03AB214607A80BAAFFF762FEB4
:10C16000E36807A9186880F09FFF01E01329EBD06E
:10C1700012B070BD5E29FAE707AD03A80FF016FCF8
:10C1800028460FF013FC0DF10B03CDE900533246A6
:10C1900003AB0BA92046FFF77BFFE0689DF80B304F
:10C1A00000682A4603A980F055FFE1E70120DFE798
:10C1B00070B5214B04460E460FCB88B06D4685E81E
:10C1C0000F0020462946FFF703FEE368186880F059
:10C1D000E3FB98B1E368186803681B69984768B186
:10C1E000E3682946186880F049FA38B94CF026FC13
:10C1F00040F216624FF480114CF0D8FB214604A89F
:10C200002B463246FFF70EFE04A92046FEF776FEC7
:10C2100020B90A48FBF7E2FD08B070BD0023C4F85E
:10C220009431B388A4F8923104AA31462046FFF72E
:10C230006DFF0028F0D1ECE7D07A0020582C0020C8
:10C24000F0B5324B04460E460FCB91B004AD85E8F5
:10C250000F0020462946FFF7BBFDE368186880F011
:10C260009BFB98B1E368186803681B69984768B13D
:10C27000E3682946186880F001FA38B94CF0DEFB13
:10C280004FF4DF624FF480114CF090FB0CAF08A824
:10C290000FF08CFB38460FF089FB0DF10F03CDE951
:10C2A00000732A4608AB31462046FFF7F1FEE068EE
:10C2B0009DF80F3000683A4608A981F011FA20B9BC
:10C2C0001348FBF78BFD11B0F0BD0023C4F8943187
:10C2D000B388A4F8923108AA31462046FFF716FF2A
:10C2E0000028EDD00B4B1B68022B09D0032B03D188
:10C2F000094B93F9A5341BB106480021FAF71EFA41
:10C3000001212046FEF746FCDDE700BFD07A002081
:10C31000582C00206C910020584C002037B5044662
:10C320000D468BF0C7FBC4F8A801D5ED027AF5EEF7
:10C33000C07AF1EE10FA17DD9FED137A67EE877A77
:10C34000FCEEE77AC4ED697A2046FDF75BFDD4F890
:10C35000A4214FF47A73B2FBF3F30C4A062103B025
:10C36000BDE8304051F05ABC65F010FE0023009348
:10C3700095F90D2095F90E3095F90C1065F0A2FD98
:10C38000C4F8A401E0E700BF00007A4480F90D087A
:10C3900010B5B1F90A30A0F8BC3191F90C3080F831
:10C3A000BE31B1F90D30A0F8C031B1F90F3007EE50
:10C3B000903AF8EEE77A0446C0ED717A8BF07AFB9A
:10C3C0000B21C4F8C8012046BDE81040FEF7E2BBCF
:10C3D00038B504460D468BF06DFBC4F8B001D5EDC1
:10C3E000027A9FED047A67EE877AFDEEE77AC4ED74
:10C3F0006B7A38BD00007A444A7C06480B46003A06
:10C4000091F91010D3ED030A93ED020A18BF01222F
:10C41000FAF79EB96C91002070B51B4E0446D6F811
:10C420007402036886B01B680D469847042806D13D
:10C430006B88102B0FD0732B20D000201CE0D6F877
:10C44000740203681B6898470328F6D194F890316A
:10C45000062BF2D1ECE705F108010FC902ACDFEDC4
:10C460000B0A84E80F00002309480093B0EE600A2D
:10C470001A46214602F0BCFE06B070BD2046294691
:10C48000FFF7BAFF0120F7E7585C0020000000002A
:10C49000788D002038B5D1F8093007EE903AF5EEE6
:10C4A000C07AF1EE10FA05460C4605DD0B7A022B38
:10C4B00003D01ED9032B0ED038BD154B9FED150AA6
:10C4C000D3F8B00E27EE800A80F0FCF9D4F80930DA
:10C4D000C5F8D031F0E70E4B9FED0E0AD3F8B00E41
:10C4E00027EE800A80F0FEF9D4F80930C5F8D4317F
:10C4F000E2E7074B9FED070AD3F8B00E27EE800A5C
:10C5000080F0FEF9D4F80930C5F8CC31D4E700BF8B
:10C51000586C00200000C84238B5114D0C4605F695
:10C52000447095F8BD1F5CF0EDFB58B195F8BD1F48
:10C5300005F644705CF0EEFB20B994ED040A09485E
:10C54000FAF7A4F994ED041AD4ED020A94ED030A63
:10C5500095F8BD1F0448BDE8384000225CF012BCCD
:10C56000586C00206C9100209C7B0020F0B50B697A
:10C57000214F85B005460E460BB94B6953B30023D6
:10C580003B7006F108030FCB6C4684E80F00214690
:10C590002846FFF7C1FB98B9184B0122D3F87C1E3F
:10C5A00020460FF009FA4EF093F8022215214DF0C3
:10C5B00047FE2846FDF726FC114A022151F02EFBCA
:10C5C00021462846FEF79AFC38B90E48FBF706FCD0
:10C5D00005B0F0BD3846FEF74FFEB38807EE903A3F
:10C5E000F8EE677A09212846C7ED017A05B0BDE863
:10C5F000F040FEF7CFBA00BFC4910020586C002075
:10C6000090F90D08582C002010B5044C237813B174
:10C61000034869F0A3FC207810BD00BF8092002081
:10C62000907C00200078072894BF002001207047EC
:10C6300013B5094B01910446D3F8B00E03681B698A
:10C64000984730B10199204602B0BDE81040FEF78E
:10C650004FBA02B010BD00BF586C002090F898315E
:10C6600013F0010018BFC3F380007047094A034666
:10C6700092F8B90268B192F8B822043A012A07D8B0
:10C680005B6A1B6893F8A100431E584258417047EB
:10C6900000207047588C002010B504468BF00AFA31
:10C6A000D4F8B031C01AD4F8AC3123EAE37398421D
:10C6B0004FF0000084BFC4F8AC01012010BD0000A1
:10C6C00010B5036804461B6E9847D4F8AC3123EAD2
:10C6D000E37398424FF000003CBFC4F8AC01012066
:10C6E00010BD000008B504480321FAF707F8BDE8BB
:10C6F00008400148FAF726B96C91002070B51C4B30
:10C700000446D3F8B00E03681B690E4698470546E9
:10C7100010B90025284670BDD4F894315BB98BF070
:10C72000C9F9B4F89231C4F8940123B1114A53788D
:10C7300043F0010353708BF0BDF9D4F89421B4F8A1
:10C740009231801A4FF47A72B0FBF2F09842E0D343
:10C7500023B9084A537843F0010353702046FDF78C
:10C7600051FB3388044A062151F058FAD2E700BF42
:10C77000586C00205C9300203CF70D0810B590F831
:10C780009031042B0446164B0AD1D3F8B00E03683F
:10C790001B69984718B12046FEF7AAFC002010BD7F
:10C7A0000A79D3F8B83EDFED0F6A93ED0E6A07EE13
:10C7B000902A0A7E920748BF9FED0B7AF8EE677ABF
:10C7C00048BF67EE877A86EE267AB0EEC77AB4EE77
:10C7D000E77AF1EE10FAACBF01200020DFE700BFDE
:10C7E000586C0020DB0FC9400000803B13B5094B9B
:10C7F00001910446D3F8B00E03681B69984730B125
:10C800000199204602B0BDE81040FEF771B902B0B0
:10C8100010BD00BF586C002010B504468BF04AF9DB
:10C82000D4F8A831C01AD4F8A43198424FF00000CF
:10C8300084BFC4F8A401012010BD000038B505462E
:10C840000C468BF037F9D5F8C831C01A23894FF45C
:10C850007A725343984294BF0020012038BD0000F3
:10C86000C368186808B190F8B808704710B501217E
:10C8700004460A4804F008FD28B120460321BDE81B
:10C880001040FEF787B94CF0D9F8BDE8104040F2EF
:10C890006B124FF480114CF089B800BFD48E002089
:10C8A00090F89031022B04D0032B04D1034804F0FC
:10C8B000BBBC012070470020704700BFD48E002011
:10C8C00038B50C4BD3F8185E90F89031032B044622
:10C8D00005F004050AD1084804F0BEFC94F8903134
:10C8E00035B110B9023B5842584138BD0020F5E738
:10C8F0000120FAE7584C0020D48E002010B50F4AD2
:10C90000137843F0800313700D4B93F96822002ACB
:10C91000044609DBFEF73AFA70B920460822BDE862
:10C9200010400921FDF740B9BDE8104001220E2159
:10C93000A3F18000F5F758BB10BD00BF5C93002049
:10C94000585C0020F8B5D0F8B44105465CB1012C24
:10C950001AD04CF073F840F643024FF480114CF0BB
:10C9600025F8012407E0184BD3F8B00E03681B69C3
:10C97000984710B900242046F8BD2846FEF740FB32
:10C980000123C5F8B431F6E7104F97F96832002B50
:10C99000F0DA436A1B6893F8A160012EEAD13C30BB
:10C9A00027F04CF904460028E5D1D7F8983293F8DF
:10C9B000CB3033B132460D21A7F18000F5F714FBDF
:10C9C000D9E73446D7E700BF586C0020585C0020F8
:10C9D00038B56E4BD3F874226D4B9A4204460D461F
:10C9E00001D0002072E04B885E2B55D8512B0CD81B
:10C9F000103B9AB20F2A29D92046FDF703FA6B881B
:10CA0000644A042151F00AF959E0523B0C2BF3D847
:10CA100001A252F823F000BF6FCB0108F9C9010849
:10CA200031CB010845CB0108F9C90108F9C9010852
:10CA3000F9C90108F9C90108F9C90108F9C90108CA
:10CA4000F9C9010875CB01084DCB01080F2BD3D8CC
:10CA500001A252F823F000BF3FCB0108E3C901084F
:10CA600055CB01085BCB010869CB010845CB010818
:10CA700031CB0108F9C90108F9C90108F9C9010850
:10CA8000F9C90108F9C90108F9C90108F9C901087A
:10CA9000F9C9010861CB0108732B74D006D8702B3B
:10CAA0006ED0722BA8D1FFF70BFE44E04AF2CF62A2
:10CAB000934262D0A0D8B32B09D8B12B9CD9204681
:10CAC000FDF7A0F9298855F0A1FA012038BDBC3B3B
:10CAD0009AB2132A90D8132B8ED801A252F823F0C1
:10CAE000BFCA0108BFCA0108F9C90108F9C901088C
:10CAF000F9C90108F9C90108F9C90108BFCA010843
:10CB0000F9C90108BFCA0108F9C90108F9C9010832
:10CB1000F9C90108BFCA0108F9C90108F9C9010822
:10CB2000F9C90108BFCA0108F9C90108BFCA01084B
:10CB30002046FFF769FD00283FF453AFBFE7FFF73A
:10CB4000DDFDF8E72046FFF7FDFEF4E71248FFF7AA
:10CB500069FDF0E7FFF712FEEDE7FFF769FDEAE791
:10CB6000BDE83840FFF77ABDFFF780FDE3E7FFF748
:10CB70003DFEE0E7FFF750FEDDE7FFF75FFEDAE797
:10CB8000FFF78AFDD7E7FFF7ADFDD4E7585C00203B
:10CB900030860020C4F90D08C491002090F890312F
:10CBA000032B0BD0062B06D0012B0AD1C3681868C3
:10CBB00003681B681847044801F00CBF034804F0E1
:10CBC000BDBB0020704700BF788D0020D48E0020B0
:10CBD0008B88012B05D00B693BB94B692BB9CB680E
:10CBE0001BB904480021FAF7C3B9024800220831F2
:10CBF000FAF7E0B9582C002010B54B885E2B04469C
:10CC00000A464DD8512B05D8103B99B20F2921D98E
:10CC100000209DE0523B0C2BFAD801A151F823F0E3
:10CC20008BCD010811CC010845CD01085BCD010871
:10CC300011CC010811CC010811CC010811CC01085C
:10CC400011CC010811CC010811CC010893CD0108C9
:10CC50009BCD01080F2BDBD801A151F823F000BFB9
:10CC600053CD010865CD01086DCD010875CD0108D2
:10CC700085CD01085BCD010845CD010811CC010827
:10CC800011CC010811CC010811CC010811CC01080C
:10CC900011CC010811CC010811CC01087DCD01088F
:10CCA000B32B00F0848016D8732B7DD00ED8702B58
:10CCB00077D0722BACD1D1ED027A9FED447A67EE3A
:10CCC000877AFDEEE77AC0ED6B7A40E0B22B9FD118
:10CCD000FFF7E0FB3BE0CD2B2CD8BB2B98D9BC3B1E
:10CCE000112B95D801A151F823F000BF4FCD0108B9
:10CCF0004FCD010811CC010811CC010811CC01085D
:10CD000011CC010811CC0108B5CD010811CC0108E6
:10CD1000B5CD010811CC010811CC010811CC0108D6
:10CD2000B5CD010811CC010811CC010811CC0108C6
:10CD3000C1CD01084AF2CF6293427FF469AFFFF799
:10CD400027FB04E002F108012046FEF745F8012028
:10CD500010BD1146FFF72CFAF9E711462046FFF700
:10CD60008BF8F4E71146FFF7C7F8F0E71146FFF735
:10CD7000FDF8ECE71146FFF727F9E8E71146FFF762
:10CD80002FF9E4E7FFF772FDE1E71146FFF758FAE4
:10CD9000DDE71146FFF7C2FAD9E71146FFF7E6FBD8
:10CDA000D5E7FFF715FBD2E7FFF726FBCFE7FFF745
:10CDB0000FFFCCE7064802F10801F9F787FDC6E747
:10CDC00011462046FFF7A8FBC1E700BF0000C8429C
:10CDD0006C910020704700007047000090F8280018
:10CDE0007047000090F8A802704700000F207047BD
:10CDF00000207047002070470020704700207047D7
:10CE00000048704774FA0D080048704780FA0D0812
:10CE100008B5094800F50053D3F8643EB3F908306B
:10CE200000EE103AB8EEC00AF5F770FBBDE8084016
:10CE30000248FCF71BBE00BF582C002008880020C9
:10CE400010B514482DED028B1C4600F5005300F57B
:10CE50008040B3F97434D0F8A40E08EE103A036899
:10CE600082B09B6ECDE900219847B8EEC88AF0EEFB
:10CE7000400ADDE90021B0EE480A0748FCF79AFBBA
:10CE80000548FCF755FE84ED000A02B0BDEC028BAC
:10CE900010BD00BF582C002008880020F8B51C4D9C
:10CEA00005F5005405F580462846D6F8AC7EF5F722
:10CEB0001BFBB4F9B03401EE103AB4F9AE3400EE15
:10CEC000903A434200EE103AB8EEC11AF8EEE00A8A
:10CED000B8EEC00A38467DF097F82846D6F8AC6E12
:10CEE000F5F702FBB4F9B03401EE103AB4F9AE3400
:10CEF00000EE903A434200EE103A3046B8EEC11AC6
:10CF0000BDE8F840F8EEE00AB8EEC00A7DF0F6B8E9
:10CF1000582C002038B5144C04F5804504F58F5486
:10CF2000D5F8A40E03689B689847692100F1940224
:10CF300020464CF061FAD5F8A40E0368DB689847E8
:10CF40006A2100F1940220464CF056FAD5F8A40E5E
:10CF500003681B6998476B2100F194022046BDE8E5
:10CF600038404CF049BA00BF582C0020014806F068
:10CF7000D1BC00BF582C00203C3088F07BBE0000A4
:10CF800073B51F4D0646D5F8740203681B6B9847AE
:10CF9000044680B395F96932002B2FDBD5F898321F
:10CFA00093F8CB403CB395F8683203F0A003202BF4
:10CFB00024D1D5F8740203681B689847052808D067
:10CFC000D5F8740203681B689847A0F110035C420F
:10CFD0005C410C4A02F688630193A2F50053214696
:10CFE000D3F87C3F0093D2F8AC3ED2F8A42E304662
:10CFF00088F0EEFD0446204602B070BD0024FAE73A
:10D00000585C0020586C00203C30FFF7B9BF00008E
:10D0100038B5114D04461148F5F7CEFE95F9683242
:10D02000002B14DA236A93F8A120012A06D0D5F840
:10D0300074020021BDE83840FCF7DABB0D21A5F1F0
:10D040008000F4F7D1FF95F96832002BEFDB204622
:10D05000BDE8384089F0F8B8585C0020582C002012
:10D060003C30FFF7D5BF000001207047012070471A
:10D07000012070470120704707207047012070474A
:10D08000002070470020704701207047004870471B
:10D09000C8FB0D0800487047D0FB0D0870B52DED9A
:10D0A000028B0025C36880F83C501B68DFED488A7E
:10D0B000D3ED0A0A42699FED478A93ED060AF4EE22
:10D0C000E80A0446F1EE10FA88B01068B8BFF0EE36
:10D0D000480A7CF07FFDE36862691B681068D3ED45
:10D0E0000A0A93ED060AF4EEE80AF1EE10FAB8BF68
:10D0F000F0EE480A7CF0E6FD636920461E68FCF706
:10D1000085FE6368B3F93820B3F9363000EE903A03
:10D11000434201EE102A00EE103AB8EEC11AF8EEC2
:10D12000E00AB8EEC00A30467CF06EFF6369204624
:10D130001E68FCF76BFE6368274CB3F93820B3F91F
:10D14000363000EE903A434200EE103A01EE102ADB
:10D150003046B8EEC11AF8EEE00AB8EEC00A7CF02C
:10D16000CDFFD4F8B80E7FF069F8D4F8B86E338BE1
:10D170001B0723D504A80EF019FC09F0DDFB9FED79
:10D18000170A044606F11C0023F072FF01AA04A945
:10D1900020468DED010ACDED020A8DED031A09F04E
:10D1A000ADFB80B10322294604A80EF005FC0C4B10
:10D1B000186804AA90F879105BF000FF094808216C
:10D1C000F9F79CFA012008B0BDEC028B70BD00BFDE
:10D1D0000000003400007A43586C00200AD7233C3A
:10D1E000DC9C00206C91002030B52DED048BC368D1
:10D1F0009FED898A1B684269D3ED0A7ADFED870AC1
:10D2000093ED060AF4EEC87AF1EE10FA0446A8BFD0
:10D21000F0EE670A106889B07CF0DCFC6369204698
:10D220001D68FCF7F3FD6368B3F93820B3F93630B5
:10D2300000EE903A434200EE103A01EE102A2846E2
:10D24000774DB8EEC11AF8EEE00AB8EEC00A7CF0ED
:10D25000DBFED5F8B80E7FF06DF9A5F5805393F895
:10D260008D32D90747D4D5F8B83E1A8BD20742D5AC
:10D2700093ED0A9AB4EEC89AF1EE10FAB8BF93EDA6
:10D28000049AE36A186859F0DDF9D5F8B03ED3ED99
:10D29000067AA36B20EE270AD3ED007AF0EE498AD6
:10D2A000E0EE278AB0EE490AF5EEC08AF1EE10FAF8
:10D2B000D8BFDFED5C8AF0EE680A20F055FB28B994
:10D2C000D5F8B80EB0EE680A7EF078FE636893F980
:10D2D0005130272B0FD0A36A186859F0B3F9F0EE3C
:10D2E000C07AF4EEC87AF1EE10FAB0EE407A20D5AA
:10D2F000002384F83C30236B1B68B3F9083000EE40
:10D30000103A2046B8EEC00AFCF742FC2046FCF773
:10D31000ADFB2046B0EE408AFCF732FA002848D038
:10D320000021204609B0BDEC048BBDE83040FCF77D
:10D330005FBAD5F8B83E9FED3C0AD3ED0F7AD3ED36
:10D340000B6AA36B27EE800AF4EEC86AD3ED007A6D
:10D35000F1EE10FA67EE277A10DB9FED341ADFED5D
:10D36000310A552037EE800A20F002FC012384F8B0
:10D370003C30D5F8B80E7EF011FEBCE79FED2C7A5C
:10D38000F4EEC76AF1EE10FA05D89FED261ADFED2C
:10D39000290A5920E6E7F0EEE66AF4EEC86AF1EEF3
:10D3A00010FAE3D594F83C30002B08BFB0EE670AC2
:10D3B000DCE7636A0221186883F068FB1E4806F008
:10D3C00039F9B0EE480AD5F8B80E7EF0B5FF01463F
:10D3D0001A48FAF705FC636918687EF0FBF9236ABE
:10D3E0001D68636918687DF033F805AC2046144960
:10D3F0008DED020ACDED030A8DED041AF9F774FBE9
:10D40000079B009394E80C0002A928467AF048FA9A
:10D4100009B0BDEC048B30BD0000003400007A433D
:10D42000586C002000000000E02E65420000B4426D
:10D43000000000B40000B4C2605B0020582C002043
:10D440006C91002008B5064BD3F8B83ED86824305C
:10D4500023F05AFBFCEEC07A17EE900A08BD00BF1D
:10D46000586C0020024BD3F8B83ED8687DF09AB8CB
:10D47000586C00200B207047012070470020704737
:10D480000120704700207047004870476CFC0D0871
:10D490000048704774FC0D080120704708B5DFEDA7
:10D4A000237AF4EEE70AF1EE10FA2DED028BF0EE9E
:10D4B000408AB0EE608A35DDDFED1D7AF4EEE70AD2
:10D4C000F1EE10FA2ED5F6EE007A70EEE77ADFED87
:10D4D000196A9FED190ADFED190AF0EEE77A87EE77
:10D4E000A67A8720B7EE001A30EE470A20F040FBFC
:10D4F000DFED137A9FED131ADFED130A20EE270AF2
:10D500008A2020EE280A20F033FB30EE080ABDEC1A
:10D51000028BDFED0A0ABDE808408D20B7EE001A45
:10D5200020F026BB9FED050AEFE700BFAC1C5A3E7A
:10D53000D578493F8FC2753E9A99993F0000000007
:10D54000FAEDEBBA9A99993E9A9999BE30B52DEDBC
:10D55000048B7D4BB3F9743400EE903AF8EEE00A98
:10D5600083B0044601AA6946B0EE600AFCF722F8CF
:10D57000A06980F003FCE369D0ED008AD3ED946AE2
:10D58000D3ED977A90ED016AA3689FED701ADFEDF5
:10D59000700A27EEE80A68EEA68A03F6F803E6EEBC
:10D5A000278A05463B20DFED6B7AB0EEE87AB4EED1
:10D5B000E77AF1EE10FA58BFB0EE677ADFED667ADF
:10D5C000C7EE275AF7EE007A77EEE57A9DED007AFE
:10D5D00067EE877A93ED007A67EE877A9FED5F7A40
:10D5E000A6EE260A87EE879A20F0C2FA3C209FED2D
:10D5F000571ADFED570AB0EE408AB0EE680A20F005
:10D60000B7FA626B564B1268DFED567AB2F9082012
:10D61000D3ED006A9FED541ADFED540A07EE102A8D
:10D62000B8EEC77AF0EE408A27EE277ADFED507A1F
:10D63000A6EEA77A4520F4EE007AA7EE678ABAEE46
:10D64000000A28EE000A83ED007A8DED000A20F032
:10D650008FFADDED017A9FED477A474B8DED000A99
:10D66000F0EEE77AF4EEC77AF1EE10FA51D593EDC9
:10D67000007ADFED427A77EE277AB2EE007AF4EEA6
:10D68000C77AF1EE10FA58BFF0EE477AC3ED007A90
:10D6900067EEA87ACDED017A636A186890F8CB102E
:10D6A000002939D183F0F2F9636A1B6893F8A1105D
:10D6B000012939D0032940D039B9236A18687AF092
:10D6C000D7FD236A18687AF023F8236ADDED010A92
:10D6D00018689DED000A0368B0EE491ADB6A9847A6
:10D6E000204695ED028AFCF761F92046F0EE400AEB
:10D6F000B0EE480AFFF7D2FE236A62681868D2EDDE
:10D70000020A036801215B6E984703B0BDEC048BED
:10D7100030BD00221A60BFE7194B93F96932002B24
:10D72000B4BF01210221BDE7236A18687AF0A0FD89
:10D73000236A18687AF002F8C7E7D9790029C4D1BA
:10D740002046FCF759FBC0E7584C002000000C4471
:10D7500000000CC40000FA4400409C450000344224
:10D76000E09100200AD7233D00A08C4500A08CC585
:10D770008FC2753F00000034E49100208FC2F53C59
:10D78000585C00201620704700207047002070472A
:10D79000012070470020704781F0010070470000B1
:10D7A000012070470048704710FD0D080048704781
:10D7B00088DF0D0803681BB1007900F00100704795
:10D7C00018467047F0B5494D95F9BD6F85B00446D0
:10D7D000A5F50055002E00F085804548FFF7EAFFCB
:10D7E000064600287ED0636920461F68FCF70EFBC2
:10D7F0006368B3F93820B3F9363000EE903A43420B
:10D8000001EE102A00EE103AB8EEC11AF8EEE00A66
:10D81000B8EEC00A38467CF0F7FB636920461F6803
:10D82000FCF7F4FA6368B3F93820B3F9363000EE48
:10D83000903A434200EE103A01EE102A3846B8EE14
:10D84000C11AF8EEE00AB8EEC00A7CF057FC05F504
:10D850008043D3F8AC0E7CF0EBFC18B96369186810
:10D860007DF06AFEB5F9A43004F13C001BB9B5F8AF
:10D87000A230A5F8A430B5F8A43007EE903AF8EE3F
:10D88000677A04F1980203A90027CDED037A4FF0DF
:10D8900075FC04F15C00C4F8A070019070F07EFE8D
:10D8A000002384F8A530B5F9A43001981BB9B5F868
:10D8B000A230A5F8A430B5F8A43007EE903AF8EEFF
:10D8C000E77AB7EE000A80EE270A70F08BFE09486F
:10D8D00080F050FAC4F8C870DFED077A20EE270A0E
:10D8E00084ED310A304605B0F0BD00BF584C002031
:10D8F000105C0020E07A00200AD7233C10B50446D3
:10D90000FBF7B0FB2046154B40F83C3B4FF0B8FB13
:10D91000134B2365134B9FED142A9FED141ADFED73
:10D92000140A9FED140A6365F1EE041A04F15C0019
:10D9300070F06EFE002320460F49C4F8A830C4F8EA
:10D94000AC30C4F8B030C4F8B430C4F8B830C4F85F
:10D95000BC3042F057FD204610BD00BF18FE0D0838
:10D96000CDCCCC3D000040400AD7233B00803B4556
:10D970009A99993ECDCC4C3EB0FD0D082DE9F0436F
:10D980002DED028B9BB0914604460D468AF092F82D
:10D99000B8499FEDB98A0646A1F1080022F0E6FFDA
:10D9A00094ED161ACDED110A7E20F1EE410A8DEDAF
:10D9B000100A20F0DDF894ED161A8DED100AF1EE44
:10D9C000410A7F209DED110A20F0D2F810A904F140
:10D9D0003C008DED110A4FF0EFFBA848CDED130A86
:10D9E0008DED120A80F0C6F9D4ED327AD4ED140A26
:10D9F00094ED151AE0EE087A892004F15C074FF0E7
:10DA00000008B0EE670A20F0B3F812A822F0FAFF7F
:10DA10009B4812A909F0E2F914A938468DED140AC1
:10DA2000CDED150A70F09AFC3846CDF85880CDF847
:10DA30005C8070F0D7FC8DED160ACDED170AB9F1B8
:10DA4000000F00F001810123C4F8D06084F8CC30CD
:10DA50008C4E04F1A80116A822F0B0FFB6F9743478
:10DA600000EE103A16A8B8EEC00A22F0CBFF16A9B5
:10DA7000A6F53F6009F09EF918A928468DED180A11
:10DA8000CDED190A22F09AFFB6F9743495ED007ABB
:10DA900007EE903AF8EEE77AB0EEC77AB4EEE77A9E
:10DAA000F1EE10FA00F3CE8095ED017AB0EEC77A70
:10DAB000F4EEC77AF1EE10FA4CBF0123002384F88C
:10DAC000A530B6F9743495ED000A5A4207EE903A43
:10DAD00000EE902AB8EEE71AF8EEE00ACA2020F02D
:10DAE00047F885ED000AB6F9743495ED010A5A42FB
:10DAF00000EE902A07EE903AF8EEE00AB8EEE71A48
:10DB0000CB2020F035F885ED010A94F8A4305A1C9A
:10DB100084F8A4201422B3FBF2F102FB1133DBB230
:10DB2000002B34D14CF0D4FD064689F0CBFF804663
:10DB3000D4F8AC000F46F2F7EFFCCDE90E01D4F8B3
:10DB4000A800F2F7E9FCCDE90C01D4F8A000F2F747
:10DB5000E3FCCDE90A016868F2F7DEFCCDE90801D3
:10DB60002868F2F7D9FCCDE906011398F2F7D4FC46
:10DB7000CDE904011298F2F7CFFCCDE90087CDE999
:10DB80000201414B414A424930464CF0CDF91BB0AD
:10DB9000BDEC028BBDE8F08312A822F0B5FFDFEDEB
:10DBA0003D7AB4EEE70AF1EE10FA57D494F8CC308F
:10DBB00063B956E0384670F075FC94F8CC3084EDCB
:10DBC0002A0AC4ED2B0A002B3FF442AFDFED325A94
:10DBD000DFED324A9FED324ADFED323A12AA2B4690
:10DBE00005F10801B2EE0E5AB7EE003AB2EC016A46
:10DBF00094F99D00B0EEC67A67EE256A07EE900AAA
:10DC000076EE842AF8EEE77AB0EE647AA7EE857AAB
:10DC1000C3EEA27A27EE087A77EE837A27EE267A89
:10DC2000B5EEC06A67EE877AF1EE10FA48BFF1EE02
:10DC3000677AE3EC017A9942D8D1CDF85C80CDF8CF
:10DC4000588005E701233AE794F8CC304BB1D4F87B
:10DC5000D00040F6B833361A9E429DD9002384F88E
:10DC6000CC3094F8A530002BA4D1384670F080FC5D
:10DC7000A3E700BF3C5C00200AD7233CE07A0020E9
:10DC800068400020584C0020C3C80D081CFD0D083A
:10DC900088DF0D089A99993E0000C8420000BE42F4
:10DCA000000070420000FA432DE9F04F2DED048B87
:10DCB0000446A5B0BD4880F05DF8BD4BDFEDBD7AF0
:10DCC0001B68DB6A93F89C3060EE278A33B9F1EE6B
:10DCD000687AC4ED327AC4ED318A47E0B64D05F575
:10DCE0004053D3F8983293F8A090B9F1020FEED1D7
:10DCF00089F0E0FE05F58043D3F8BC3EC01A40F23F
:10DD0000DB539842E3D99FEDAD8A95F8B41D8DEDB4
:10DD1000218A18AB21AA05F6C8008DED228A8DED67
:10DD2000238A1EF0CDF808B3A54821A921F020F8D8
:10DD3000D4ED2C7A8DED210A37EE800AD4ED2D7AC0
:10DD4000CDED220A77EEA00A9E4884ED2C0AC4EDA0
:10DD50002D0A8DED231AFFF72DFD60B989F0AAFE7B
:10DD600084ED2D8AC4F8C00084ED2C8A25B0BDEC6A
:10DD7000048BBDE8F08F05F5005BD4F8C020DBF81C
:10DD8000EC3F42B9C4F8C03084ED2D8A84ED2C8A72
:10DD900084ED328AEAE79A42E8D08B4804F1B00178
:10DDA00009F008F889498DED190AF1EE607AA1F1C0
:10DDB000080010EE108A17EE907ACDED1A0ACDED1C
:10DDC0001B7A8DED1C0A22F0D1FDDBF8EC3FD4F874
:10DDD000C0208DED1D0AA3EB020ABAF5FA7FCDED46
:10DDE0001E0A04F1B8051DAE0CD996E80300C4F86C
:10DDF000C03084ED2D8A84ED2C8A85E80300C4EDC3
:10DE0000318AC5E72946304622F0B0FD96E8030086
:10DE100085E8030094ED329ADBF8EC3F9FED6C6AE5
:10DE2000C4F8C03039EE285A8DED1F0ACDED200A16
:10DE30001FA91BAA0023F0EE489AF1EC017AF0EE3C
:10DE4000E76AF4EEC66AF1EE10FA1FD4D2ED005A7A
:10DE5000B0EEE57AB4EEC67AF1EE10FA16D485EE9D
:10DE6000A77AB5EEC07AF1EE10FA0FD907EE903A24
:10DE7000F8EEE77A37EE457A77EEA67AE7EE269A5D
:10DE8000FCEEE77ACDED177A9DF85C30B9F1010F21
:10DE900002F1040240F087802BB107EE903AF8EED1
:10DEA000E77AC9EEA79A4FF4EC70F5EEC09AF1EE5E
:10DEB00010FA48BF79EEA99AB5EE001AFDEE000AF5
:10DEC000B0EE690A1FF054FE39EE009A9FED410A48
:10DED00094ED327ADFED407A29EE009AA7EE279A88
:10DEE000D4ED147A84ED329A39EE289AB4EEE79A9A
:10DEF000F1EE10FA44BF77EEE87AC4ED327A94ED91
:10DF0000329A4CF0E5FB054689F0DCFD8146D4F8F9
:10DF1000C400CDF850A00E46F2F7FEFACDE912018A
:10DF200018EE900AF2F7F8FACDE91001D4F8C8001B
:10DF3000F2F7F2FACDE90E0119EE900AF2F7ECFAD7
:10DF400038EE899ACDE90C0119EE100AF2F7E4FADD
:10DF5000CDE90A014046F2F7DFFACDE9080138467B
:10DF6000F2F7DAFACDE906012098F2F7D5FACDE911
:10DF700004011F98F2F7D0FA184B194ACDE90201B3
:10DF8000CDE90096174928464BF0CEFF2046FBF717
:10DF900039FF1549B0EE490A50F0CCF884ED2D8ACE
:10DFA00084ED2C8A97E64FF0010946E7E07A0020DD
:10DFB000609100200AD7233C582C0020000000006C
:10DFC00088430020105C0020684000203C5C00205A
:10DFD0000AD7233DCDCC4C3ECDCC4C3F3CFD0D086B
:10DFE00048FD0D087FFD0D0884FD0D082DE9F04169
:10DFF0002DED048B044688B0FFF756FE636920467A
:10E000001D68FBF703FF6368B3F93820B3F93630B6
:10E0100000EE903A434200EE103A01EE102AF8EE7C
:10E02000E00AB8EEC11AB8EEC00A28467BF0ECFF51
:10E0300004F13C052046FBF7B1FD28464FF0B8F847
:10E04000D4ED260A1FF090FCB74BA0B9B3F9A42079
:10E050001AB9B3F8A220A3F8A420B3F8A43007EEAD
:10E06000903AF8EE677A04F1980206A92846CDEDB9
:10E07000067A4FF083F8AD4DDFEDAD8AD5F8643EFA
:10E08000B3F9083000EE103AA5F50050B8EEC00A1A
:10E09000F4F73CFA2046B0EE408A8DED030AFBF718
:10E0A000B5FEB5F9AE3401EE103A434200EE903AB7
:10E0B000B8EEC11AF8EEE00AF820B0EE480A1FF0F8
:10E0C00057FD20468DED030AFBF732FD2046B0EEEA
:10E0D000409A9DED030AFBF7E5FC074605F6B8708C
:10E0E000FFF768FBD8B195F8D83F9FED927AD4ED51
:10E0F000286A07EE903AF8EEE77A67EE877A9FEDA6
:10E100008E7AE6EE877A8D4EC4ED287A042F22D8D7
:10E11000DFE817F00800BF00E200E700F200F0EED1
:10E12000687AF0E7864B0021D3F8980282F0AEFCC3
:10E13000D6F8A40E79F0ECFAD6F8A40E01217AF004
:10E1400097F8D6F8AC0E9FED7A0A7DF0D1FA04F17B
:10E150005C0070F023FAD5F85C3ECDED048AB3F98B
:10E160000880D5F8603ECDED058AB3F90870B5F9A1
:10E17000743408EE103A236A186803689B6E984757
:10E18000B8EEC88AF0EE400A05AAB0EE480A04A923
:10E190002046FBF70FFA94F99C3094ED287A07EEAD
:10E1A000903AF8EEE77AF1EE489AB4EEE77AF1EEBB
:10E1B00010FA37DB89F07EFCD6F8BC3EC01A40F678
:10E1C000B83398422ED958EA070306A914BF012292
:10E1D00000222046CDED068ACDED078AFFF7CEFB63
:10E1E000F6EE007A69EEA70A28EE271A4FF4A5701A
:10E1F0009DED060A8DED011ACDED000A1FF0B8FC69
:10E2000040F24B108DED060A9DED011ADDED000A7E
:10E210009DED070A1FF0ACFC06A904A88DED070AC6
:10E2200022F0CCFBB0EE481AF0EE690A9DED040A2C
:10E230004FF4A7701FF09CFCB0EE481AF0EE690A8C
:10E240008DED040A40F24F109DED050A1FF090FC81
:10E25000B5F974348DED050A00EE103A05AA04A94B
:10E26000B8EEC00A374866F0B7F8D6F8A40EDDED70
:10E27000050A03689DED040ADB6AB0EE491A984767
:10E28000636918687DF0A6FA08B0BDEC048BBDE8A0
:10E29000F0812B4B2C4FD3F89802022182F0F6FB31
:10E2A0003B786BB963689FED291ADFED210A93ED86
:10E2B000040A4FF48C701FF05BFC384605F020FF19
:10E2C00020469DED030AFBF7D1FB1F488DED030AA5
:10E2D00003A905F04FFF3EE7236A0121186879F092
:10E2E000C7FF236A186879F029FA63699FED100A5D
:10E2F00018687DF0FDF92EE7114F0221D7F898023A
:10E3000082F0C4FB20469DED030AFBF7AFFBA7F1AB
:10E31000F8008DED030A05F08DF963699DED030AA0
:10E3200018687BF0F7FE16E7582C0020584C0020A8
:10E3300000000000D0CC4C3D3333733F586C0020BC
:10E34000585C0020207C00209C92002000007A4431
:10E350001720704701207047002070470020704749
:10E360000120704700487047A4FE0D080048704720
:10E370008DDF0D0883689FED067A03F63803D3ED31
:10E38000187A67EE877AFCEEE77A17EE900A704704
:10E390000000C84283689FED067A03F63803D3ED88
:10E3A000197A67EE877AFDEEE77A17EE900A7047E2
:10E3B0000000C842806800F6380083F06FBD00009E
:10E3C00010B5836803F63803D3ED180A93ED190AE4
:10E3D000044B0C460FCB84E80F0020460DF054FE92
:10E3E000012010BDD07A002070B5836893F9386899
